:100000000C94E50D0C94160E0C94160E0C94160E12
:100010000C94160E0C9489380C9441550C94FD4A9E
:100020000C94160E0C94160E0C94160E0C94160EC0
:100030000C94160E0C94160E0C94160E0C94160EB0
:100040000C94160E0C943A7F0C94D55B0C94160EFF
:100050000C94160E0C94160E0C94160E0C940C495F
:100060000C94160E0C942F7D0C94067D0C94160E99
:100070000C94160E0C94160E0C94160E0C94160E70
:100080000C94FC870C94160E0C94160E0C94160E01
:100090000C94DD7C0C94B47C0C94160E0C94160E0F
:1000A0000C94160E0C94160E0C94160E0C94160E40
:1000B0000C94160E0C94B43C0C94160E0C94160E64
:1000C0000C94160E0C94160E0C94160E0C948B7C3D
:1000D0000C94627C0C94160E0C94397C0C94107C5D
:1000E0000C94160E431946194D19501953195619E7
:1000F0005D19641967196E1975197C193B1F691F01
:10010000A01FD71FB220E920172145210B220B2267
:100110000B220B220B220B220B220B220B220B2277
:100120000B220B220B220B220B220B220B220B2267
:100130000B220B220B220B220B220B220B220B2257
:100140000B220B220B220E2046207D207321AB2197
:10015000E2210C24122418241E2424242A243024CE
:1001600036243C24422448244E24602466246C24F3
:10017000722478247E2484248A24902496249C2427
:10018000A224A824AE24B424BA24C024CC24D82485
:10019000DE24E424EA24022508250E2514251A2548
:1001A00020250A261026162628262E263426462600
:1001B0004C26522658265E26642676267C26A626BF
:1001C000AC26B226B826D026D626DC26E226FA268B
:1001D000002706270C27122718271E272427282741
:1001E0002C27302736273A273E27422746274A27FB
:1001F0004E275427722778277E27F02426252C2582
:10020000322538253E254425BE26C426CA26E826A2
:10021000EE26F42684278A2790276A2670264A2508
:10022000502556255C25622568251C263A26D224B1
:1002300054245A24F624FC2496279C27A227C6245B
:10024000822688268E2694269A26A0266E25742538
:100250007A25802586258C25922598259E25A425FE
:10026000AA25B025B625BC25C225C825CE25D4256E
:10027000DA25E025E625EC25F225F825FE250426DD
:10028000662760275A276C2722264026842E612E57
:100290003A2EA12EF82EC02EEF2EDE2EA92F8C2F57
:1002A000652FF92FC62FC62FE82FD12F7F357F3529
:1002B00099357F35A635BF35DA35F535E13CE93C72
:1002C000F03C033D143D253D2F3D1B441E440D4491
:1002D000114417445544224426442C4430443444A9
:1002E0003A443E444244554448444C4450449F465A
:1002F000A446A946B346BD463647C746CF46D7466D
:10030000E146EB46F54604470E4736471847224775
:100310002C4729725D729272B272E7724F735F73EB
:100320008974D373DD7311744674547489741B73A8
:10033000BC8DD38DEA8D018E188E468E5D8E748EA7
:100340008B8EAA8EC28ED98EF88E0E8F2F8E340091
:10035000330032004E6F6E650053746F70706564C9
:10036000004E65757472616C205475726E004D6F2D
:1003700076696E672052657665727365004D6F769B
:10038000696E6720466F7277617264004272616BBA
:10039000696E670054414E4B20524553544F5245AD
:1003A000440025004865616C7468204C6576656C76
:1003B0003A200056454849434C4520524550414952
:1003C0005220434F4D504C4554450054414E4B2014
:1003D00044455354524F5945440025004865616CCB
:1003E0007468204C6576656C3A20002900564548B3
:1003F00049434C45205245504149522053544152A3
:10040000544544202800524550414952204F504500
:10041000524154494F4E2043414E43454C4C454474
:100420000029004D414348494E452047554E20483C
:10043000495421202800524550414952204F5045EF
:10044000524154494F4E2043414E43454C4C454444
:1004500000290043414E4E4F4E2048495421202848
:100460000054757272657420726F746174696F6E76
:10047000206973206E6F74206F6620747970652018
:10048000536572766F2E204E6F20736574757020E1
:10049000617661696C61626C652E004E6F207374C9
:1004A000656572696E6720736572766F206173731C
:1004B00069676E65642C2072652D636865636B20C7
:1004C00076656869636C6520747970652E00547573
:1004D0007272657420656C65766174696F6E2069EF
:1004E00073206E6F74206F66207479706520536579
:1004F00072766F2E204E6F20736574757020617652
:1005000061696C61626C652E00546F70204C656689
:100510007400546F702043656E74657200546F7080
:10052000205269676874004D6964646C65204C658D
:100530006674004D6964646C652043656E74657211
:10054000004D6964646C6520526967687400426F8D
:1005500074746F6D204C65667400426F74746F6DB7
:100560002043656E74657200426F74746F6D205223
:1005700069676874004649524D57415245205645B7
:100580005253494F4E3A20006942757300534275E9
:10059000730050504D004E6F6E6520446574656366
:1005A00074656400417A696D7574682020202000AC
:1005B000456C65766174696F6E2020005475726EAB
:1005C00020202020202020005468726F74746C65F5
:1005D00020202000537469636B20202020202020DD
:1005E0004D696E2020202043656E746572202020A6
:1005F0004D6178202020204465616462616E642032
:1006000020526576657273656400524144494F20FB
:10061000494E464F202D20004E4F5420444554450E
:10062000435445440049474E4F52454400416E6192
:100630006C6F67004469676974616C00417578206C
:100640004368616E2E2020204D696E2020202020DE
:100650004D61782020202020547970650043686126
:100660006E6E656C73207574696C697A65643A2086
:10067000004368616E6E656C7320646574656374B5
:1006800065643A2000202844697361626C656429BE
:10069000002028456E61626C656429004D656368C1
:1006A000616E6963616C207265636F696C0041699A
:1006B00072736F6674004D656368616E6963616C27
:1006C0002042617272656C3A200020284D31290069
:1006D00020284D322900202842290042617272658B
:1006E0006C20456C65766174696F6E3A202000203D
:1006F000284D30290020284D31290020284129008B
:1007000054757272657420526F746174696F6E3AB9
:100710002020200020416D7073290020284375722D
:1007200072656E74204C696D69743A200044726978
:100730007665204D6F746F72733A20202020202040
:10074000004D4F544F522054595045530054616E40
:100750006B202854616D69796120444D442900540F
:10076000616E6B2028444B4C4D2047656172626F6F
:100770007829004361720048616C66747261636B32
:100780000054616E6B00554E4B4E4F574E005965ED
:1007900073004E6F002900252C20446563656C654D
:1007A000726174696F6E20666163746F72200020DD
:1007B000284B69636B6261636B20737065656420AD
:1007C00000547261636B205265636F696C20456EE3
:1007D00061626C65643A202020004E2F4120666FD4
:1007E000722076656869636C652074797065005461
:1007F00075726E204D6F64653A20202020202020E5
:1008000020202020202020004E2F4120666F7220C3
:1008100076656869636C65207479706500596573E5
:10082000202854616D69796129002500202D200060
:100830004E65757472616C205475726E20416C6CDB
:100840006F7765643A20202000207365630054723E
:10085000616E736D697373696F6E2044656C617945
:100860003A2020202020002073656300456E6769D0
:100870006E652050617573652054696D653A20205E
:10088000202020200020736563005368696674206F
:1008900054696D653A20202020202020202020202F
:1008A0002020004175746F6D61746963004D616E45
:1008B00075616C005472616E736D697373696F6EEC
:1008C00020547970653A20202020202000250059EE
:1008D0006573202D20005265766572736520537014
:1008E000656564204C696D697465643A2020002553
:1008F00000596573202D2000466F72776172642065
:100900005370656564204C696D697465643A202094
:1009100000206D73290025207468726F74746C65F3
:1009200020666F7220002028004D6F746F72204E79
:100930007564676520456E61626C65643A202020AD
:10094000200029004E6F6E65004E6F6E65002C20F2
:100950005072657365743A20002900202841646A4A
:10096000757374656420746F200020284C6576656B
:100970006C3A2000446563656C2052616D702045BF
:100980006E61626C65643A20202020200029004EB0
:100990006F6E65004E6F6E65002C2050726573653A
:1009A000743A20002900202841646A7573746564D4
:1009B00020746F200020284C6576656C3A20004139
:1009C0006363656C2052616D7020456E61626C6579
:1009D000643A202020202000416374697665204419
:1009E000726976696E672050726F66696C653A202D
:1009F0000056656869636C6520547970653A2020FB
:100A0000202020202020202020004452495645202C
:100A100053455454494E4753002073656300526553
:100A2000636F696C2064656C61793A202020202016
:100A300020202020202020202020202020200025D1
:100A400000596573202D200042617272656C20454B
:100A50006C65766174696F6E205370656564204CB7
:100A6000696D697465643A20002500596573202D0D
:100A7000200054757272657420526F746174696FCE
:100A80006E205370656564204C696D697465643AC5
:100A90002020005455525245542053455454494E39
:100AA000475300556E6B6E6F776E004865617679BF
:100AB000004D656469756D004C6967687400437525
:100AC00073746F6D00556E6B6E6F776E004E6F6E48
:100AD00065004F70656E2050616E7A6572005461DA
:100AE0006D697961205370656300207365632072BE
:100AF00065636F766572792900207365632072657E
:100B00006C6F61642C2000204D4720686974732C41
:100B100020002063616E6E6F6E20686974732C20F4
:100B200000280057656967687420436C6173733AE5
:100B300020202020200044616D6167652050726F85
:100B400066696C653A2020200059657320280041B1
:100B50006363657074204D472044616D6167653A39
:100B6000200059657320280053656E64204D47208E
:100B7000495220436F64653A2020004E2F410052B5
:100B8000657061697265642062793A2020202020B6
:100B900020004E2F41004869742050726F746F63BB
:100BA0006F6C20323A2020200029002028546561F3
:100BB0006D2000466972652050726F746F636F6CB0
:100BC0003A2020202000466972652050726F746FB1
:100BD000636F6C3A202020200049732052657061B9
:100BE00069722054616E6B3F2020200049522026FC
:100BF0002054616E6B20426174746C696E6720448E
:100C0000697361626C656400424154544C452049EB
:100C10004E464F00554E4B4E4F574E0042656E6547
:100C200064696E6920544253204D6963726F0042BB
:100C3000656965722055534D2D52432D3200546124
:100C40006967656E20536F756E642043617264003E
:100C50004F70656E2050616E7A657220536F756EAD
:100C60006420436172640042656E6564696E692048
:100C7000544253204D696E6900536F756E64206352
:100C80006172643A2000534F554E44204341524410
:100C90000048696C6C205068797369637320456EF5
:100CA00061626C65643A20202020202020202000F2
:100CB00042617272656C2053746162696C697A6119
:100CC00074696F6E20456E61626C65643A200053F2
:100CD000656E736F722064657465637465643A2031
:100CE0002020202020202020202020202059657333
:100CF0000053656E736F72206E6F74206465746547
:100D0000637465642100494E45525449414C204D5D
:100D10004541535552454D454E5420554E4954007A
:100D2000556E6B6E6F776E0042617272656C204516
:100D30006C65766174696F6E20436F6D6D616E6472
:100D40000054757272657420526F746174696F6EAD
:100D500020436F6D6D616E64005374656572696EDA
:100D60006720436F6D6D616E640056656869636CE2
:100D70006520537065656400456E67696E65205334
:100D800070656564005468726F74746C6520436F9D
:100D90006D6D616E64005370656564206465637297
:100DA00065617365732062656C6F772000537065B1
:100DB000656420696E637265617365732061626F3B
:100DC000766520005475726E2053746F7070656480
:100DD000004C656674205475726E20537461727491
:100DE0006564005269676874205475726E2053748C
:100DF00061727465640056656869636C652053743C
:100E00006F70706564004D6F76696E67205265760D
:100E100065727365004D6F76696E6720466F7277F5
:100E200061726400456E67696E652053746F70006F
:100E3000456E67696E652053746172740043616E1C
:100E40006E6F6E2052656C6F6164656400566568F4
:100E500069636C652044657374726F7965640043DF
:100E6000616E6E6F6E20486974004272616B6573CB
:100E7000204170706C696564005661726961626CD2
:100E80006500290020286F662000506F7320004104
:100E90007578204368616E6E656C200056617269DA
:100EA00061626C65004F6E004F6666004200410053
:100EB00045787465726E616C20496E70757420009F
:100EC000070809090B0C0C0B0C0C54757272657435
:100ED00020537469636B202D200046756E6374691E
:100EE0006F6E202300202D3E200020736563005488
:100EF0007572726574206D6F76656D656E742064B1
:100F0000656C61793A2020004E6F6E6500596573FB
:100F10000054757272657420737469636B20667512
:100F20006E6374696F6E733A200046554E435449A0
:100F30004F4E20545249474745525300762063751F
:100F4000746F666629002028004C564320456E6168
:100F5000626C65643A202020202020007600566FC5
:100F60006C746167653A20202020202020202020FA
:100F700000596573004E6F00426174746572792088
:100F800044657465637465643A2000424154544575
:100F900052590053657269616C20332054782042A5
:100FA0006175643A2020004175782053657269614B
:100FB0006C20426175643A202020004D6F746F727E
:100FC0002053657269616C20426175643A20005556
:100FD00053422053657269616C20426175643A2006
:100FE00020200042415544205241544553002120C5
:100FF00000464143544F52592052455345542120F5
:10100000003A200042697420004761703A2000498C
:101010004F20506F72742042202D2050756C7365E4
:101020006400494F20506F72742042202D20537469
:1010300061727420426C696E6B696E6700557365EE
:10104000722046756E6374696F6E2031005573654A
:10105000722046756E6374696F6E203200466F723F
:10106000776172642047656172004E6575747261C4
:101070006C20476561720052657665727365204722
:101080006561720053657420416363656C20526131
:101090006D70204C6576656C3A2000536574204471
:1010A0006563656C2052616D70204C6576656C3AA5
:1010B00020005365742042617272656C2053656E26
:1010C00073697469766974793A20005365742048AD
:1010D000696C6C2053656E73697469766974793ACA
:1010E0002000416E616C6F672055736572204675F4
:1010F0006E6374696F6E2031202D2000416E616C2B
:101100006F6720557365722046756E6374696F6EE4
:101110002032202D20002D00202D200020005452B0
:1011200055450046414C5345002500576169746997
:101130006E6720666F7220726164696F2E2E2E209A
:101140000000002100240027002A002D0030003379
:101150000001010000040107010A0100002200252E
:101160000028002B002E0031003400020100000591
:101170000108010B01000020002300260029002C9B
:10118000002F0032000001000003010601090105E3
:10119000050505070508080808020202020A0A08F0
:1011A0000804040404010101010101010103030316
:1011B0000303030303040707070C0C0C0C0C0C0CB3
:1011C0000C0202020206060606060606060B0B0BBA
:1011D0000B0B0B0B0B0102102020080810204010F5
:1011E00020408002010201080402010102040810EB
:1011F0002040808040201008040201800402018009
:101200004020100804020108040201010204081031
:10121000204080010204081020408000000A0B02D8
:10122000090C0D0E08070304010000000000000077
:1012300000000000000000000000000000000000AE
:10124000000000000000001211100000000000006B
:10125000000000000000000000000000000000008E
:1012600000202D2053746172742052657065617482
:10127000696E6700202D2053746F7000557365727E
:1012800020536F756E64200041202D200042202DD8
:101290002000536F756E642042616E6B2000506CAD
:1012A00061792F53746F7000506C61792052616EB8
:1012B000646F6D00506C61792050726576696F754E
:1012C0007300506C6179204E6578740046697265D0
:1012D0002043616E6E6F6E004669726520526570C4
:1012E000616972205369676E616C00416972736F46
:1012F0006674202D204D616E75616C205472696793
:10130000676572004D656368616E6963616C205248
:1013100065636F696C202D204D616E75616C205482
:1013200072696767657200536572766F20526563F4
:101330006F696C202D204D616E75616C205472694F
:1013400067676572004869676820496E74656E73E7
:1013500069747920466C61736820556E6974202D1C
:10136000204D616E75616C2054726967676572000B
:101370004D47205374617274004D472053746F7051
:1013800000417578204F757470757420466C6173D8
:1013900068656400417578204F75747075742049D4
:1013A0006E766572736520466C6173686564005380
:1013B000746F7020417578204F7574707574204279
:1013C0006C696E6B696E670053746F70205265763E
:1013D0006F6C76696E6720417578204C6967687418
:1013E00000494F20506F72742041202D2050756CA1
:1013F00073656400494F20506F72742041202D2086
:10140000537461727420426C696E6B696E6700552B
:101410006E6B6E6F776E0044657461636865642FF0
:101420004E41005265636F696C20536572766F00A0
:1014300050616E20536572766F00536572766F2F20
:10144000455343004F6E626F617264204D6F746F3D
:101450007220447269766572004F70656E2050612B
:101460006E7A65722053636F75742053657269617B
:101470006C20455343005361626572746F6F7468EA
:101480002053657269616C00506F6C6F6C752053EE
:10149000657269616C00536572766F203100536527
:1014A00072766F203200536572766F203300536579
:1014B00072766F203400536572766F203500536565
:1014C00072766F203600536572766F203700536551
:1014D00072766F2038005475726E20456E67696EA3
:1014E00065204F6E004D616E75616C207472616E87
:1014F000736D697373696F6E202D20707574206928
:101500006E206E65757472616C2067656172206211
:1015100065666F7265207374617274696E672065A9
:101520006E67696E6521005475726E20456E67693D
:101530006E65204F666600456E67696E6520417571
:10154000746F2053687574646F776E00456E6761C1
:101550006765205472616E736D697373696F6E0095
:10156000446973656E67616765205472616E736D5F
:10157000697373696F6E00536574205475726E20C1
:101580004D6F64653A203100536574205475726E56
:10159000204D6F64653A2032005365742054757293
:1015A0006E204D6F64653A203300456E61626C6554
:1015B000204E65757472616C205475726E730044B0
:1015C000697361626C65204E65757472616C20543C
:1015D00075726E730042617272656C205374616241
:1015E000696C697A6174696F6E3A205475726E65C0
:1015F00064204F4E0042617272656C2053746162C8
:10160000696C697A6174696F6E3A205475726E659F
:1016100064204F46460048696C6C205068797369B5
:1016200063733A205475726E6564204F4E004869AA
:101630006C6C20506879736963733A205475726ECC
:101640006564204F464600494F20506F7274204118
:10165000204F7574707574202D204F6E00494F20F7
:10166000506F72742041204F7574707574202D2056
:101670004F666600494F20506F72742042204F75AC
:1016800074707574202D204F6E00494F20506F727A
:10169000742042204F7574707574202D204F66663B
:1016A000004C56432045786974202D20566F6C7489
:1016B00061676520526573746F72656400762900F6
:1016C0004C5643207468726573686F6C6420726551
:1016D0006163686564212028004C69676874203163
:1016E000204F6E0052657665727365643A20200063
:1016F0004D61782050756C73653A20004D696E20FD
:1017000050756C73653A2000456E642056616C75A7
:10171000657300456E64205265636F696C20536584
:1017200072766F20536574757000456E6420526F39
:10173000746174696F6E20536572766F205365749F
:10174000757000456E6420456C65766174696F6ED6
:1017500020536572766F20536574757000536572FF
:10176000766F20756E2D72657665727365640053B1
:101770006572766F20726576657273656400526576
:101780007665727365643A2020004D61782050754B
:101790006C73653A20004D696E2050756C73653A24
:1017A000200053746172742056616C756573004932
:1017B0004E56414C494420534552564F2E204E4FD1
:1017C0002053455455502E00536574757020526552
:1017D000636F696C20536572766F00536574757022
:1017E0002054757272657420526F746174696F6EE3
:1017F0002050616E20536572766F0053657475706A
:10180000205374656572696E6720536572766F2028
:10181000284F757470757420322900536574757083
:10182000205374656572696E6720536572766F2008
:10183000284F757470757420342900536574757061
:101840002054757272657420456C65766174696F99
:101850006E20536572766F00401F7017D007A00F7F
:10186000A00FDC05D007C40910278813983A102769
:1018700058026C0258026C0258026C0258026C0248
:1018800058026C0258026C0258026C0258026C0238
:101890005802B0366C023A026C023A026C023A020A
:1018A0006C02B036384A5C121C255C125C121C2596
:1018B0005C12BC7FC7F2C07887A5B7C5A00F88139C
:1018C000B80B401FB80BB80B7017401F5461696705
:1018D000656E2056322F563300536F6E7900524397
:1018E0005441204D616368696E652047756E004301
:1018F0006C61726B204D616368696E652047756E1F
:10190000005243544120526570616972004942554A
:101910002052657061697200436C61726B20526580
:1019200070616972004F70656E50616E7A65720009
:10193000567354616E6B00464F560054616967657B
:101940006E2056310048656E67204C6F6E670054FC
:10195000616D69796120312F33350054616D69798A
:101960006120322D53686F740054616D6979610094
:10197000556E6B6E6F776E004C696768742031200E
:101980004F6666004C696768742032204F6E004CC9
:10199000696768742032204F666600326E64204D9D
:1019A000472053746F7000326E64204D472053748B
:1019B0006172740052756E6E696E67204C6967685B
:1019C0007473204F6E0052756E6E696E67204C699D
:1019D00067687473204F666600417578204F757490
:1019E000707574204F6E00417578204F7574707556
:1019F00074204F66660053746F70205265766F6C6A
:101A000076696E6720417578204C69676874005369
:101A1000746F7020417578204F7574707574204212
:101A20006C696E6B696E6700417578204F757470D4
:101A30007574205072657365742044696D00537429
:101A400061727420417578204F75747075742042EE
:101A50006C696E6B696E6700416972736F667420A2
:101A60002D20456E61626C6564004D656368616E32
:101A70006963616C205265636F696C202D20456E2F
:101A800061626C656400416972736F6674202D2019
:101A900044697361626C6564004D656368616E6979
:101AA00063616C205265636F696C202D20446973FB
:101AB00061626C656400436F6D6D73206368616E75
:101AC00067656420746F2055534200436F6D6D73DA
:101AD000206368616E67656420746F205365726966
:101AE000616C20310044726976696E672050726FB4
:101AF00066696C652073657420746F20230025006F
:101B00005370656564207265647563656420746FE5
:101B10002000537065656420726573746F7265642C
:101B200000536D6F6B657220656E61626C65640059
:101B3000536D6F6B65722064697361626C656400DC
:101B400053657420766F6C756D653A20002900200E
:101B50002D2041646A757374656420746F200020C1
:101B60002853656E73697469766974792000290059
:101B7000202D2041646A757374656420746F2000A1
:101B8000202853656E7369746976697479200053EF
:101B900074617274205265766F6C76696E6720414D
:101BA0007578204C6967687400524144494F20465B
:101BB00041494C5341464500526164696F2052656A
:101BC000616479202D200000EDA911241FBECFEF04
:101BD000D1E2DEBFCDBF00E00CBF16E0A0E0B2E076
:101BE000E7EEF7E901E00BBF02C007900D92A031CC
:101BF000B107D9F723E1A0E1B6E001C01D92AB39EE
:101C0000B207E1F71DE0C5EEDDE000E006C0219778
:101C10000109802FFE010E9478B5C43ED10780E003
:101C20000807A9F70E94AB970C9438BB0C940000EE
:101C30002F923F924F925F926F927F928F929F92DC
:101C4000AF92BF92CF92DF92EF92FF920F931F93CA
:101C5000CF93DF93CDB7DEB7E6970FB6F894DEBF2C
:101C60000FBECDBF8091B4069091B5060E94ED7B6A
:101C70000E94E24365E775E08091B4069091B50655
:101C80000E948F7A62EF75E0CE0101960E94507A31
:101C90000091B4061091B506D801ED91FC914D81EB
:101CA0005E8169817A810280F381E02DC8011995F6
:101CB000C8010E94ED7BCE0101960E94207A0E940D
:101CC000E1948091B4069091B506DC01ED91FC9110
:101CD0000284F385E02D19958091B4069091B506A4
:101CE0000E94ED7B0E94E2436AE076E08091B406B8
:101CF0009091B5060E948F7AE091010BE4300CF0D0
:101D0000E0E086E995E09A83898382E995E09C8307
:101D10008B838DE895E09E838D8388E895E0988796
:101D20008F83EE0FFF0B81E090E08C0F9D1FE80F7B
:101D3000F91F608171818091B4069091B5060E946F
:101D4000007C0E94E24364ED75E08091B4069091BE
:101D5000B5060E94007C0E94E24368EC75E0809129
:101D6000B4069091B5060E948F7AE091DB11F09154
:101D7000DC1181819281883E934014F40E94D24309
:101D8000E091DB11F091DC11618172818091B406E8
:101D90009091B5060E94D77584E00E948995E091E4
:101DA000DB11F091DC11658176818091B406909110
:101DB000B5060E94D77585E00E948995E091DB11F8
:101DC000F091DC11638174818091B4069091B50625
:101DD0000E94D77584E00E948995E091DB11F09113
:101DE000DC1167818091B4069091B5060E94AD74B4
:101DF00088E00E948995E091DB11F091DC118085EB
:101E00000E94BE436CEB75E08091B4069091B506DC
:101E10000E948F7AE091E511F091E6118181928123
:101E2000883E934014F40E94D243E091E511F09172
:101E3000E611618172818091B4069091B5060E948D
:101E4000D77584E00E948995E091E511F091E61143
:101E5000658176818091B4069091B5060E94D77510
:101E600085E00E948995E091E511F091E61163818A
:101E700074818091B4069091B5060E94D77584E074
:101E80000E948995E091E511F091E61167818091BA
:101E9000B4069091B5060E94AD7488E00E948995C1
:101EA000E091E511F091E61180850E94BE4360EB60
:101EB00075E08091B4069091B5060E948F7AE0910A
:101EC000EF11F091F01181819281883E934014F4DA
:101ED0000E94D243E091EF11F091F0116181728183
:101EE0008091B4069091B5060E94D77584E00E9457
:101EF0008995E091EF11F091F011658176818091E3
:101F0000B4069091B5060E94D77585E00E94899528
:101F1000E091EF11F091F011638174818091B4062A
:101F20009091B5060E94D77584E00E948995E09152
:101F3000EF11F091F01167818091B4069091B50690
:101F40000E94AD7488E00E948995E091EF11F091B4
:101F5000F01180850E94BE4364EA75E08091B4066A
:101F60009091B5060E948F7AE091F911F091FA11E3
:101F700081819281883E934014F40E94D243E09183
:101F8000F911F091FA11618172818091B4069091FA
:101F9000B5060E94D77584E00E948995E091F911F9
:101FA000F091FA11658176818091B4069091B50621
:101FB0000E94D77585E00E948995E091F911F09112
:101FC000FA11638174818091B4069091B5060E94E4
:101FD000D77584E00E948995E091F911F091FA118A
:101FE00067818091B4069091B5060E94AD7488E037
:101FF0000E948995E091F911F091FA1180850E9473
:10200000BE438091B4069091B5060E94ED7B0E947C
:102010001F82C82E6CE376E08091B4069091B506DD
:102020000E94007C0E94E2430AE711E1E12CF12CBE
:10203000D12C57012FEFA21AB20AB5018091B40634
:102040009091B5060E94D77549E0E416F10410F4AA
:102050008BE001C08AE00E948995D8012C91809183
:10206000B4069091B5062223C9F11596ED91FC9125
:102070001697618172810E94D775D8011596ED91EE
:10208000FC91169781819281883E934014F40E94BE
:10209000D24384E00E948995D8011596ED91FC9178
:1020A0001697638174818091B4069091B5060E9461
:1020B000D77584E00E948995D8011596ED91FC9121
:1020C000169727818091B4069091B506222319F0C6
:1020D00064E376E00BC06DE276E008C0EC14FD042A
:1020E0001CF465E276E002C068E176E00E94007CC4
:1020F000095F1F4F7501BCE0AB16B10409F099CF21
:102100000E94E24361E776E08091B4069091B506C3
:102110000E948F7A0E941F82682F8091B40690914E
:10212000B5060E9498746DE576E08091B4069091B2
:10213000B5060E948F7A6091FE0A7091FF0A809125
:10214000B4069091B5060E940A760E94E1948091AF
:10215000B4069091B506DC01ED91FC910284F38503
:10216000E02D19958091B4069091B5060E94ED7B03
:102170000E94E24361E477E08091B4069091B50655
:102180000E94007C0E94E2436DE277E08091B406F9
:102190009091B5060E948F7A809120100E94C757B7
:1021A000BC018091B4069091B5060E948F7A80910F
:1021B00020108A30C1F46BE177E08091B4069091F1
:1021C000B5060E948F7A6091D4108091B4069091E8
:1021D000B5060E94AD7464E177E08091B4069091F9
:1021E000B5060E948F7A8091B4069091B5060E9440
:1021F000ED7B60E077E08091B4069091B5060E9497
:102200008F7A809121100E94C757BC018091B4063B
:102210009091B5060E948F7A209121108091B4068A
:102220009091B5062B303CF4293054F4283069F4F1
:102230006FEE76E007C02B3041F46BEF76E002C022
:1022400065EF76E00E94007C02C00E94ED7B6BEDA2
:1022500076E08091B4069091B5060E948F7A8091C5
:1022600022100E94C757BC018091B4069091B50618
:102270000E948F7A209122108091B4069091B50629
:102280002B303CF4293054F4283069F46AEC76E0C1
:1022900007C02B3041F466ED76E002C060ED76E0D9
:1022A0000E94007C02C00E94ED7B66EB76E080918C
:1022B000B4069091B5060E948F7A209134108091D7
:1022C000B4069091B506222319F06EEA76E002C0BA
:1022D0006CE976E00E948F7A2091F20D8091B4062D
:1022E0009091B506222319F061E976E002C065E815
:1022F00076E00E948F7A8091B4069091B5060E9494
:10230000ED7B0E94E1948091B4069091B506DC01CA
:10231000ED91FC910284F385E02D199580910002E6
:10232000823011F00C947A1AF090511000915410F0
:1023300010E08091B4069091B5060E94ED7B0E945A
:10234000E2436AE07AE08091B4069091B5060E947B
:10235000007C0E94E24361EF79E08091B4069091A5
:10236000B5060E948F7AE0916110E6300CF0E0E053
:1023700086E897E09A83898381E897E09C838B8342
:1023800087E797E09E838D8383E797E098878F8325
:102390008FE597E09A8789878DE497E09C878B8704
:1023A000EE0FFF0B81E090E08C0F9D1FE80FF91FEF
:1023B000608171818091B4069091B5060E94007C85
:1023C00068ED79E08091B4069091B5060E948F7A0D
:1023D000609100028091B4069091B5060E949874B5
:1023E0006FEB79E08091B4069091B5060E948F7AE8
:1023F0008F2D0E94A943FF2009F44BC065EB79E0C3
:102400008091B4069091B5060E948F7A8091B406AF
:102410009091B506112339F060914C100E94AD7473
:1024200090914C1006C0609152100E94AD74909132
:1024300052108091511398130C94811A69E979E034
:102440008091B4069091B5060E948F7A8091B4066F
:102450009091B506112339F060914D1061110CC0B7
:1024600064E979E006C060915310611105C06FE81E
:1024700079E00E948F7A05C0062E000C770B0E942F
:10248000D7756DE879E08091B4069091B5060E9409
:102490008F7A8091B4069091B5060E94ED7B64E737
:1024A00079E08091B4069091B5060E948F7A802FD2
:1024B0000E94A943002309F44BC06AE679E08091A9
:1024C000B4069091B5060E948F7A8091B4069091DF
:1024D000B506112339F060914F100E94AD749091B0
:1024E0004F1006C0609155100E94AD749091551028
:1024F0008091531398130C949B1A6EE479E08091A9
:10250000B4069091B5060E948F7A8091B40690919E
:10251000B506112339F06091501061110CC069E4C7
:1025200079E006C060915610611105C064E479E05D
:102530000E948F7A05C0062E000C770B0E94D7757B
:1025400062E479E08091B4069091B5060E948F7A9A
:102550008091B4069091B5060E94ED7B69E279E026
:102560008091B4069091B5060E948F7A80916A108E
:10257000811103C00E94B74335C06EE877E08091B7
:10258000B4069091B5060E948F7A66E279E0809158
:10259000B4069091B5060E948F7A60916A1080917E
:1025A000B4069091B5060E94AD7466E179E0809121
:1025B000B4069091B5060E948F7A40916B105091AD
:1025C0006C1060E070E02AE08091B4069091B5064E
:1025D0000E94C87A61E179E08091B4069091B506D5
:1025E0000E94007C68EF78E08091B4069091B50677
:1025F0000E948F7A809162108436C8F461EF78E08F
:102600008091B4069091B5060E948F7A6091621015
:102610008091B4069091B5060E94AD746FEE78E09B
:102620008091B4069091B5060E94007C03C080E0C2
:102630000E94B74366ED78E08091B4069091B506AC
:102640000E948F7A809163108436C8F46FEC78E032
:102650008091B4069091B5060E948F7A60916310C4
:102660008091B4069091B5060E94AD746DEC78E04F
:102670008091B4069091B5060E94007C03C080E072
:102680000E94B74364EB78E08091B4069091B50660
:102690000E948F7A2091AD068091B4069091B50684
:1026A000222319F06DEA78E002C063EA78E00E9424
:1026B000007C6AE878E08091B4069091B5060E94AB
:1026C0008F7A6091581070915910072E000C880B6A
:1026D000990B0E9498B920E030E04AE754E40E9448
:1026E000F1B5AB01BC0121E08091B4069091B50633
:1026F0000E94107B65E878E08091B4069091B50661
:102700000E94007C6CE678E08091B4069091B5065A
:102710000E948F7A60915A1070915B10072E000C06
:10272000880B990B0E9498B920E030E04AE754E406
:102730000E94F1B5AB01BC0121E08091B4069091FB
:10274000B5060E94107B67E678E08091B406909110
:10275000B5060E94007C6EE478E08091B40690910A
:10276000B5060E948F7A60915C1070915D10072E03
:10277000000C880B990B0E9498B920E030E04AE7E2
:1027800054E40E94F1B5AB01BC0121E08091B40694
:102790009091B5060E94107B69E478E08091B406C0
:1027A0009091B5060E94007C60E378E08091B406C9
:1027B0009091B5060E948F7A90916110913011F03E
:1027C0009430F9F480915E100E94A94380915E10CC
:1027D000882329F16CE278E08091B4069091B506E7
:1027E0000E948F7A60915F108091B4069091B50637
:1027F0000E94AD746AE278E08091B4069091B506CB
:102800000CC02091B4063091B506953019F46DE1F5
:1028100078E002C068E078E0C9010E948F7A809178
:10282000B4069091B5060E94ED7B6FEE77E0809143
:10283000B4069091B5060E948F7A909161102FEFA7
:10284000290F8091B4069091B506223028F460914A
:1028500012060E94987404C06AED77E00E94007C22
:1028600061EC77E08091B4069091B5060E948F7A72
:1028700080916E100E94A94380916E10882341F1CF
:102880006FEA77E08091B4069091B5060E948F7A46
:1028900060916F108091B4069091B5060E94AD745E
:1028A00067E977E08091B4069091B5060E948F7A2F
:1028B000609170108091B4069091B5060E94AD743D
:1028C00065E977E08091B4069091B5060E948F7A11
:1028D0008091B4069091B5060E94ED7B0E94E19430
:1028E0008091B4069091B506DC01ED91FC910284D3
:1028F000F385E02D19958091B4069091B5060E945C
:10290000ED7B0E94E24363E97AE08091B406909106
:10291000B5060E94007C0E94E24362E77AE0809163
:10292000B4069091B5060E948F7A80912910843662
:10293000C8F46BE67AE08091B4069091B5060E94E7
:102940008F7A609129108091B4069091B5060E940B
:10295000AD7469E67AE08091B4069091B5060E9464
:10296000007C03C080E00E94B74368E47AE0809175
:10297000B4069091B5060E948F7A80912810843613
:10298000C8F461E47AE08091B4069091B5060E94A3
:102990008F7A609128108091B4069091B5060E94BC
:1029A000AD746FE37AE08091B4069091B5060E9411
:1029B000007C03C080E00E94B7436EE17AE0809122
:1029C000B4069091B5060E948F7A6091361070918E
:1029D00037101616170614F50091B4061091B506B7
:1029E000072E000C880B990B0E9498B920E030E06C
:1029F0004AE754E40E94F1B5AB01BC0122E0C801F2
:102A00000E94107BC8010E94ED7B69E17AE0809111
:102A1000B4069091B5060E94007C03C080E00E943D
:102A2000B7430E94E1948091B4069091B506DC0111
:102A3000ED91FC910284F385E02D19958091B40607
:102A40009091B5060E94ED7B0E94E24368E07CE035
:102A50008091B4069091B5060E94007C0E94E243EA
:102A6000209134068091B4069091B506222309F492
:102A7000C3C169ED7BE00E948F7A0E94E5610E94EC
:102A8000B7430E94E5612091B4063091B5068823D2
:102A900089F066EC7BE0C9010E948F7A809137064D
:102AA0000E943D83BC018091B4069091B5060E94BE
:102AB000007C4FC063EB7BE0C9010E948F7A80915C
:102AC00034060E943D83BC018091B4069091B50606
:102AD0000E948F7A809135068823A9F16BEA7BE00A
:102AE0008091B4069091B5060E948F7AE0913506E8
:102AF000E4300CF0E0E084E593E09A83898382E59A
:102B000093E09C838B8380E593E09E838D838EE4AA
:102B100093E098878F83EE0FFF0B81E090E08C0F9E
:102B20009D1FE80FF91F608171818091B40690911B
:102B3000B5060E948F7A69EA7BE08091B406909195
:102B4000B5060E948F7A8091B4069091B5060E94D6
:102B5000ED7B66E97BE08091B4069091B5060E941A
:102B60008F7A809136060091B4061091B5068823BD
:102B700021F00E943D83BC0102C062E97BE0C801F4
:102B80000E94007C6FE77BE08091B4069091B506CF
:102B90000E948F7A809137060091B4061091B50695
:102BA000882321F00E943D83BC0102C06BE77BE0DB
:102BB000C8010E94007C68E67BE08091B406909199
:102BC000B5060E948F7A809139068823E1F062E68B
:102BD0007BE08091B4069091B5060E948F7A809137
:102BE00038060E943D83BC018091B4069091B506E1
:102BF0000E948F7A6AEF75E08091B4069091B506D5
:102C00000E94F07B03C080E00E94B7436FE47BE04A
:102C10008091B4069091B5060E948F7A80913A0611
:102C20008823E1F069E47BE08091B4069091B506D9
:102C30000E948F7A809138060E943D83BC0180916A
:102C4000B4069091B5060E948F7A6AEF75E0809184
:102C5000B4069091B5060E94F07B03C080E00E940C
:102C6000B74366E37BE08091B4069091B5060E947D
:102C70008F7AE0913B06E3300CF0E3E08EED9AE0D2
:102C80009A83898382ED9AE09C838B838DEC9AE012
:102C90009E838D8385EC9AE098878F83EE0FFF0BE0
:102CA000A1E0B0E0AC0FBD1FEA0FFB1F6081718196
:102CB0008091B4069091B5060E94007C63E27BE0AF
:102CC0008091B4069091B5060E948F7AE0912D060E
:102CD000E4300CF0E4E08EEB9AE09A83898388EB91
:102CE0009AE09C838B8381EB9AE09E838D838BEAB1
:102CF0009AE098878F8383EA9AE09A878987EE0F14
:102D0000FF0B81E090E08C0F9D1FE80FF91F6081A1
:102D100071818091B4069091B5060E94007C61E2B9
:102D20007BE08091B4069091B5060E948F7A609105
:102D300032068091B4069091B5060E94AD7462E1AE
:102D40007BE08091B4069091B5060E948F7A8091C5
:102D50002D06811110C0609133068091B4069091C8
:102D6000B5060E94AD7467E07BE08091B406909157
:102D7000B5060E948F7A60912E0670912F06072E5D
:102D8000000C880B990B0E9498B920E030E04AE7CC
:102D900054E40E94F1B5AB01BC0121E08091B4067E
:102DA0009091B5060E94107B69EF7AE08091B4069D
:102DB0009091B5060E948F7A60913006709131062D
:102DC000072E000C880B990B0E9498B920E030E088
:102DD0004AE754E40E94F1B5AB01BC0121E08091C7
:102DE000B4069091B5060E94107B6AEE7AE080915D
:102DF000B4069091B50602C06CEE7BE00E94007CA8
:102E00000E94E1948091B4069091B506DC01ED91A9
:102E1000FC910284F385E02D19958091B406909180
:102E2000B5060E94ED7B0E94E24366E87CE080915B
:102E3000B4069091B5060E94007C0E94E24369E7C7
:102E40007CE08091B4069091B5060E948F7AE09163
:102E50007710E5300CF0E5E087E69CE09A83898303
:102E600080E59CE09C838B838EE39CE09E838D8336
:102E70008FE29CE098878F838CE19CE09A8789871A
:102E800084E19CE09C878B87EE0FFF0B81E090E054
:102E90008C0F9D1FE80FF91F608171818091B4062E
:102EA0009091B5060E94007C0E94E1948091B40646
:102EB0009091B506DC01ED91FC910284F385E02D43
:102EC00019958091B4069091B5060E94ED7B0E9401
:102ED000E24366E07DE08091B4069091B5060E94E1
:102EE000007C0E94E243209111078091B4069091EA
:102EF000B5062223C9F16FEC7CE00E948F7A8091A5
:102F0000B4069091B5060E94ED7B60EB7CE0809169
:102F1000B4069091B5060E948F7A809171100E943C
:102F2000A9438091711081110E940D968091B40681
:102F30009091B5060E94ED7B61E97CE08091B4063A
:102F40009091B5060E948F7A809173100E94A943D8
:102F50008091731081110E94DF958091B406909149
:102F6000B5060E94ED7B04C061EF7CE00E94007C0E
:102F70000E94E1948091B4069091B506DC01ED9138
:102F8000FC910284F385E02D19958EE097E7A1E08E
:102F9000BB278BAB9CABADABBEAB8091B406909125
:102FA000B5060E94ED7B0E94E2436AE27FE08091D9
:102FB000B4069091B5060E94007C0E94E24361E154
:102FC0007FE08091B4069091B5060E948F7A20919F
:102FD000FC0A8091B4069091B506222319F06DE0A9
:102FE0007FE002C068E07FE00E94007C8091FC0AE4
:102FF000882349F16FEE7EE08091B4069091B5068A
:103000000E948F7A6091751070917610072E000CD7
:10301000880B990B0E9498B920E030E04AE754E40D
:103020000E94F1B5AB01BC0122E08091B406909101
:10303000B5060E94107B6AEE7EE08091B406909106
:10304000B5060E94007C9AEAE92E9FE0F92E29E25B
:10305000622E38E1232E3CEF332E4AE0A42EB12C11
:1030600054E6C52ED12CD7012C91222309F400C29D
:10307000F7013297008111810115110509F4F8C19A
:1030800080E796E7A1E0BB27820F911DA11DB11D2E
:10309000ABBFFC01879177247394811101C0712C1F
:1030A0002091B4063091B506C8010197849790F538
:1030B0006AEC7EE0C9010E948F7A09500C3148F415
:1030C000E02FF0E0EE0FFF1FE25EFD4F60817181A7
:1030D00002C060E27DE08091B4069091B5060E9446
:1030E0008F7A0C3130F4E02FF0E0EA5AFD4F808106
:1030F00001C080E090E08054914F092E000CAA0B93
:10310000BB0BABBFFC0187919EE0981B892F09F098
:1031100051C152C1C801845691098438934008F0C6
:103120003FC060EB7EE0C9010E948F7AC801B60102
:103130000E9451B56130710531F06230710559F46A
:103140006CEA7EE002C06EEA7EE08091B406909167
:10315000B5060E948F7A0E94DA438090B406909060
:10316000B5067720B1F0C8010E94514F811107C008
:1031700068EA7EE0C4010E948F7A87E01BC181303B
:1031800009F01AC165EA7EE0C4010E948F7A88E0E6
:1031900011C16CE97EE0C4010E948F7A82E00AC10D
:1031A000C801885E93408035964408F05AC0C80133
:1031B00068EE73E00E9451B54B016FE87EE0C901F3
:1031C0000E948F7AFAE08F16910410F40E94D24385
:1031D000B4018091B4069091B5060E94D7750E9403
:1031E000DA434090B4065090B5067720A1F1C801AB
:1031F0000E94514F782E6AE87EE0C2010E948F7AC9
:10320000672D8091B4069091B5060E94AD7464E874
:103210007EE08091B4069091B5060E948F7A829CE0
:10322000C001839C900D929C900D1124800F911FE2
:10323000B5010E9465B577278091B4069091B506D7
:103240000E94D77562E87EE08091B4069091B50641
:103250000E948F7AB1C069E77EE0C2010E948F7A36
:1032600061C0F801E853FA44E83E43E0F40708F08F
:1032700046C0EC30F10508F09FC08827EE58FF4F9C
:103280008F4F0C9478B56AE67EE019C06FE57EE05A
:10329000C9010E948F7A83E18DC06DE47EE027C072
:1032A0006DE37EE016C060E37EE055C064E27EE040
:1032B000C9010E948F7A82E17DC065E17EE0C9018B
:1032C0000E948F7A8FE076C066E07EE0F8CF66EFEE
:1032D0007DE0C9010E948F7A8EE06CC063EE7DE0D4
:1032E000C9010E948F7A8BE065C061ED7DE0C90164
:1032F0000E948F7A8CE05EC064EC7DE02CC0C80137
:1033000080529E44883E934078F400526DEA7DE0FE
:10331000C9010E948F7A0A3010F40E94D243802F94
:103320000E942D4384E046C0C80188509245883EE3
:10333000934020F4085066E97DE0EACF013FE5E5DF
:103340001E0719F465E87DE01CC0023FF5E51F0784
:1033500039F468E77DE0C9010E948F7A81E12AC0D3
:10336000033F45E5140739F46AE67DE0C9010E9490
:103370008F7A80E11FC0043F85E5180739F469E5BD
:103380007DE0C9010E948F7A8DE014C0053F95E56C
:10339000190739F461E47DE0C9010E948F7A86E063
:1033A00009C0063F154541F468E27DE0C9010E946D
:1033B0008F7A85E00E94899565EE7EE08091B40663
:1033C0009091B5060E948F7A6AED7EE08091B406F6
:1033D0009091B5060E948F7AF701608170E080912C
:1033E000B4069091B5060E94D775D7018C918A30AA
:1033F00020F482E00E94899504C0843610F40E9473
:10340000D2430E94DA43F7014081649EA001112457
:10341000052E000C660B770B8BA99CA9ADA9BEA944
:10342000480F591F6A1F7B1FDE0111968A019B01FD
:103430000F5F1F4F2F4F3F4F6BBFFA0187918D9347
:10344000B901A8018111F2CFBE016F5F7F4F80915A
:10345000B4069091B5060E94F07B8091B4069091DD
:10346000B506DC01ED91FC910284F385E02D199500
:10347000B3E0EB0EF11CE2E2EE16E0E1FE0609F02D
:10348000F2CD0E94E1948091B4069091B506DC01E2
:10349000ED91FC910284F385E02D19958091B4069D
:1034A0009091B5060E94ED7B0E94E2436BE87FE0BD
:1034B0008091B4069091B5060E94007C0E94E24380
:1034C00068E77FE08091B4069091B5060E948F7AFC
:1034D0000E949F5D20E030E040E050E40E9492B9FD
:1034E0002091B4063091B50687FF3FC065E77FE0C5
:1034F000C90159C0F0904B1000914E1011E00C948E
:10350000991166EA79E08091B4069091B5060E941F
:103510008F7A609151138091B4069091B5060E9404
:10352000AD7464EA79E08091B4069091B5060E948A
:103530008F7A0C941E126BE579E08091B40690911D
:10354000B5060E948F7A609153138091B4069091D2
:10355000B5060E94AD7469E579E08091B40690915A
:10356000B5060E948F7A0C947D1261E77FE0C90155
:103570000E94007C6EE57FE08091B4069091B506D4
:103580000E948F7A0E949F5DAB01BC0122E0809176
:10359000B4069091B5060E94107B6CE57FE08091A7
:1035A000B4069091B5060E94007C69E47FE08091AA
:1035B000B4069091B5060E948F7A8091C1100E9446
:1035C000A9432091C1108091B4069091B5062223A1
:1035D00079F066E47FE00E948F7A0E94C8956CE3E0
:1035E0007FE08091B4069091B5060E94007C02C0F5
:1035F0000E94ED7B0E94E1948091B4069091B50603
:10360000DC01ED91FC910284F385E02D1995809108
:10361000B4069091B5060E94ED7B0E94E24363EEF2
:103620007FE08091B4069091B5060E94007C0E94D4
:10363000E2436FEC7FE08091B4069091B5060E9462
:103640008F7A4091B1105091B2106091B310709187
:10365000B4108091B4069091B5060E94C6756BEBCC
:103660007FE08091B4069091B5060E948F7A4091D8
:10367000B9105091BA106091BB107091BC1080913C
:10368000B4069091B5060E94C67567EA7FE0809106
:10369000B4069091B5060E948F7A4091B510509172
:1036A000B6106091B7107091B8108091B4069091E7
:1036B000B5060E94C67563E97FE08091B4069091DB
:1036C000B5060E948F7A4091BD105091BE10609156
:1036D000BF107091C0108091B4069091B5060E9401
:1036E000C6750E94E1948091B4069091B506DC0104
:1036F000ED91FC910284F385E02D19958091B4063B
:103700009091B5060E94ED7B0E94E243E6960FB6CB
:10371000F894DEBF0FBECDBFDF91CF911F910F9107
:10372000FF90EF90DF90CF90BF90AF909F908F90E1
:103730007F906F905F904F903F902F9008952F92C1
:103740003F924F925F926F927F928F929F92AF9231
:10375000BF92CF92DF92EF92FF920F931F93CF937E
:10376000DF93CDB7DEB7AB970FB6F894DEBF0FBED1
:10377000CDBF83ED91E00E94C3BA6338714F8105DC
:10378000910519F00E947A8408C047ED51E060E08D
:1037900070E083E09FE00E94ABBA40E052EC61E051
:1037A00070E08EEE98E00E94F46C4091B51050915C
:1037B000B6106091B7107091B81081E598E00E9442
:1037C000F46C4091B9105091BA106091BB10709197
:1037D000BC1084EB97E00E94F46C4091BD105091B6
:1037E000BE106091BF107091C01087E197E00E94F9
:1037F000F46C82EA9DE0909315078093140783E6AA
:103800009BE090931307809312078EEE98E09093BD
:103810009513809394131092210E1092A70D10927D
:10382000A40D1092A60D1092A50D11E01093A80EF4
:103830000E94D8928091D5108093B7061092B60658
:103840001092800082E0809381008FE286BB10920C
:103850006F0010928500109284009BE29093A0006C
:1038600099E09093A10089BB109272001092A5007C
:103870001092A4001092A9001092A8001092AB0020
:103880001092AA001092AD001092AC0099EA9093A9
:103890002001109321018ABB109273001092250120
:1038A00010922401109229011092280110922B01EC
:1038B00010922A0110922D0110922C018091A00FDC
:1038C0009091A10F80934806909349068130F1F4BE
:1038D0008FE380931F0B1092200B61E00E943C4607
:1038E00085E19BE00E94AD881092210B1092220B83
:1038F00080914906882329F085E19BE00E94799513
:1039000011C085E19BE00E9463950CC0809149063F
:10391000882311F062E001C060E08FE30E943C4622
:103920000E943A5E8091A20F9091A30F80934E0661
:1039300090934F068130F1F48EE38093460B109202
:10394000470B61E00E943C468CE39BE00E94AD88FF
:103950001092480B1092490B80914F06882329F052
:103960008CE39BE00E94799511C08CE39BE00E9460
:1039700063950CC080914F06882311F062E001C06E
:1039800060E08EE30E943C460E94075E60E085E4B2
:103990000E943C4662E08CE30E943C4662E08BE37E
:1039A0000E943C4662E080E40E943C4662E081E482
:1039B0000E943C4662E082E40E943C4662E081E272
:1039C0000E943C4662E084E40E943C4661E089E358
:1039D0000E943C4661E08AE30E943C460E949A8B2A
:1039E0000E94D18B61E085E30E943C4661E085E066
:1039F0000E943C4661E070E085E00E94784661E00C
:103A000084E00E943C4661E087E00E943C4661E021
:103A100089E20E94D64461E089E20E943C466A9AAB
:103A200060E085E30E94D64460E085E00E94D644D1
:103A300060E084E00E94D64460E087E00E94D644C3
:103A4000729861E088E00E943C4680E090E09C0132
:103A50002D5F304FF901E955FF4F40814F3629F472
:103A6000329720813181232B31F4039688379105D9
:103A700071F760E001C061E088E00E94D64461E037
:103A80008BE20E943C4660E08BE20E94D6440E949A
:103A9000D18B0E9457758091050B813009F06CC065
:103AA0008091080B9091090BA0910A0BB0910B0B20
:103AB00040910C0B50910D0B60910E0B70910F0B00
:103AC000841B950BA60BB70B84379E40A105B1054F
:103AD00000F30E947A848091B4069091B5060E940A
:103AE000ED7B8091B4069091B5060E94ED7B0E941B
:103AF000E24361EF7FE08091B4069091B5060E94A9
:103B00008F7A01E010E00E949E8B0E94D18B6EEEB6
:103B100072E080E090E00E94C8486EEE7FE0809105
:103B2000B4069091B5060E948F7A0E949A8B0E94EB
:103B3000CD8B0530110531F064EF71E080E090E04D
:103B40000E94C8480F5F1F4F06301105E1F68091B3
:103B5000B4069091B5060E94ED7B0E94E2438091ED
:103B6000B4069091B5060E94ED7B8091B4069091C9
:103B7000B5060E94ED7B02C081118BCF80916F0052
:103B8000826080936F0080918400909185008056C0
:103B9000904F90938900809388000E941F2A84E6AA
:103BA0009BE09093BE128093BD12109170102091F3
:103BB0006F1080915E109091601030916110309381
:103BC0001607909312068093130630E0AFEFB0E033
:103BD0000E9429BB24E630E040E050E00E94DBBABE
:103BE00020935A13612F70E080E090E00E9496B914
:103BF00023EC34E64AEA5AE30E94F7B92AE939E9A4
:103C000049E55FE30E948DB560935413709355139B
:103C1000809356139093571310929500109294002E
:103C2000109290008CE08093910084EF90E090934C
:103C300099008093980011E018BB82E08093710096
:103C4000809100020E9473928091B4069091B50613
:103C50002091B70640915A1050915B105093131366
:103C6000409312132093730E9093720E8093710EF3
:103C7000109214061093141380917710853040F041
:103C80001092771060E070E084E791E00E94E874A1
:103C900010917710123009F444C008F5112309F48B
:103CA00066C0113009F05BC08CE090E00E9492B6D3
:103CB00022E433E0DC0111963C932E9324EB37E0B1
:103CC0001B963C932E931A979093B1068093B0065F
:103CD0001093DD0D1093E00D1093E30D67C01330CA
:103CE00009F45EC01430D9F586E090E00E9492B6E7
:103CF0008C0128EA33E0DC012D933D93CD0141E0B6
:103D000064E67BE00E94473C86E792E0F8019183FD
:103D100080831093B1060093B00681E08093DD0D9F
:103D200041C086E090E00E9492B62CED32E0FC01AA
:103D3000318320839093B1068093B0068FB7F894B7
:103D40002CED35E03093FD112093FC1110920212FE
:103D50008FBF81E08093DD0D8093E00D25C0109230
:103D6000771060E070E084E791E00E94E87486E0FC
:103D700090E00E9492B68C0128EA33E0DC012D939A
:103D80003D93CD0140E064E67BE00E94473C86E73E
:103D900092E0F801918380831093B1060093B006FE
:103DA0001092DD0D1092E00D1092E30D8091B0069F
:103DB0009091B106DC01ED91FC910190F081E02D34
:103DC00019958091D10D81111FC08091D40D811161
:103DD0001BC08091D70D811117C08091DA0D811120
:103DE00013C08091DD0D81110FC08091E00D811114
:103DF0000BC08091E30D811107C081E00E94D49235
:103E0000882309F418C310C3A12CB12C612C912C68
:103E10001DA2712C812C412C512C0AEE15E0EE24B0
:103E2000EA94A3E0FA2ECC24CA94DD24D3948EED38
:103E3000282E85E0382EC5018D5F904FFC01E95595
:103E4000FF4FE081EE2309F4E6C2DC01AB55BF4F22
:103E50008D919C91892B09F4DEC28E2F90E0FC019C
:103E6000F797EB32F10508F0D6C28827E258FF4FEA
:103E70008F4F0C9478B58091D10D882309F4CBC273
:103E80005110C9C289E190E00E9492B69C01FC01E8
:103E90001183008387E090E09383828315821482EC
:103EA000F782E682D186C086108EC9012AA73BA779
:103EB0000E9409802AA53BA5E2E3F4E0D901ED9335
:103EC000FC933093C20D2093C10DC9010E94F66D81
:103ED0007DC18091D40D882309F49DC241109BC2FD
:103EE00089E190E00E9492B69C01DC0111961C933E
:103EF0000E93E6E0F0E01396FC93EE93129715967E
:103F00001C921E9214971796FC92EE921697199691
:103F1000DC92CE92189758961C922AA73BA70E9433
:103F200009802AA53BA5E2E3F4E0D901ED93FC93D7
:103F30003093C40D2093C30DC9010E94F66D74C166
:103F40008091D70D882309F466C2811064C289E18B
:103F500090E00E9492B69C01DC0111961C930E9396
:103F6000E5E0F0E01396FC93EE93129715961C9201
:103F70001E9214971796FC92EE9216971996DC9261
:103F8000CE92189758961C922AA73BA70E940980A8
:103F90002AA53BA5E2E3F4E0D901ED93FC9330932D
:103FA000C60D2093C50DC9010E94F66D6BC18091AD
:103FB000DA0D882309F42FC271102DC289E190E037
:103FC0000E9492B69C01DC0111961C930E93E4E0D2
:103FD000F0E01396FC93EE93129715961C921E92A6
:103FE00014971796FC92EE9216971996DC92CE9241
:103FF000189758961C922AA73BA70E9409802AA5C9
:104000003BA5E2E3F4E0D901ED93FC933093C80DB6
:104010002093C70DC9010E94F66D62C18091DD0D2C
:10402000882309F4F8C12DA12111F5C189E190E09F
:104030000E9492B69C01DC0111961C930E93E2E063
:10404000F0E01396FC93EE93129715961C921E9235
:1040500014971796FC92EE9216971996DC92CE92D0
:10406000189758961C922AA73BA70E9409802AA558
:104070003BA5E2E3F4E0D901ED93FC933093CA0D44
:104080002093C90DC9010E94F66D62C18091E00DB7
:10409000882309F4C0C19110BEC189E190E00E945B
:1040A00092B69C01DC0111961C930E93E1E0F0E0C6
:1040B0001396FC93EE93129715961C921E921497EA
:1040C0001796FC92EE9216971996DC92CE9218975C
:1040D00058961C922AA73BA70E9409802AA53BA5B7
:1040E000E2E3F4E0D901ED93FC933093CC0D2093FF
:1040F000CB0DC9010E94F66D62C18091E30D88234A
:1041000009F489C1611087C189E190E00E9492B6EB
:104110009C01DC0111961C930E9313961C921E9227
:10412000129715961C921E9214971796FC92EE9277
:1041300016971996DC92CE92189758961C922AA739
:104140003BA70E9409802AA53BA582E394E0F901E0
:10415000918380833093CE0D2093CD0DC9010E94B1
:10416000F66D57C18091D10D882309F454C15110C7
:1041700052C18CE190E00E9492B69C01DC01119644
:104180001C930E93E7E0F0E01396FC93EE931297E6
:1041900015961C921E9214971796FC92EE92169703
:1041A0001996DC92CE92189758961C922AA73BA794
:1041B0000E9409802AA53BA5D9012D923C923093FB
:1041C000D00D2093CF0DC9010E94B86E5524539491
:1041D00022C18091D40D882309F41DC141101BC157
:1041E0008CE190E00E9492B69C01FC011183008357
:1041F00086E090E09383828315821482F782E682C0
:10420000D186C086108EC9012AA73BA70E940980CB
:104210002AA53BA5D9012D923C923093D30D209332
:10422000D20DC9010E94B86E44244394F4C0809119
:10423000D70D882309F4EFC08110EDC08CE190E028
:104240000E9492B69C01FC011183008385E090E0FE
:104250009383828315821482F782E682D186C08698
:10426000108EC9012AA73BA70E9409802AA53BA559
:10427000D9012D923C923093D60D2093D50DC901D2
:104280000E94B86E88248394C6C08091DA0D88237A
:1042900009F4C1C07110BFC08CE190E00E9492B6D9
:1042A0009C01FC011183008384E090E0938382836E
:1042B00015821482F782E682D186C086108EC901EB
:1042C0002AA73BA70E9409802AA53BA5D9012D92C8
:1042D0003C923093D90D2093D80DC9010E94B86E3D
:1042E0007724739498C08091DD0D882309F493C0DE
:1042F0002DA1211190C08CE190E00E9492B69C010A
:10430000DC0111961C930E93E2E0F0E01396FC930F
:10431000EE93129715961C921E9214971796FC9284
:10432000EE9216971996DC92CE92189758961C9298
:104330002AA73BA70E9409802AA53BA5D9012D9257
:104340003C923093DC0D2093DB0DC9010E94B86EC6
:1043500021E02DA360C08091E00D882309F45BC0AB
:10436000911059C08CE190E00E9492B69C01DC0152
:1043700011961C930E93E1E0F0E01396FC93EE93FC
:10438000129715961C921E9214971796FC92EE9215
:1043900016971996DC92CE92189758961C922AA7D7
:1043A0003BA70E9409802AA53BA5D9012D923C92EA
:1043B0003093DF0D2093DE0DC9010E94B86E992461
:1043C000939429C08091E30D882329F1611023C0C3
:1043D0008CE190E00E9492B69C01FC011183008365
:1043E0001382128215821482F782E682D186C086F9
:1043F000108E2AA73BA70E9409802AA53BA5D901B8
:104400002D923C923093E20D2093E10DC9010E9460
:10441000B86E66246394B3E0AB0EB11CE8E7AE1649
:10442000B10409F008CDE9CC82E00E94D49288233F
:1044300011F01FA216C081E00E94D492882329F0B7
:1044400082E00E94B8928111B5C78CE30E94AE440D
:10445000892B09F0A0C78CE30E94AE44892B09F098
:10446000A0C786E0E7EAF0E1DE01549601900D92E4
:104470008A95E1F7B090A0100091B0101091A110B2
:104480007091A2106091A3105091A4104091A510BA
:104490003091A6102091AD108091AE109091AF1088
:1044A000A091B006B091B106BEA3ADA3E091150EE8
:1044B000F091160EF9A7E8A79090D3106090CE1057
:1044C000E090C710F090C8108090D1107090D0107C
:1044D000C0903610D0903710509039104090341062
:1044E00030903510FFA1FB8BBA8E0B8F1C8F7D8F08
:1044F0006E8F5F8F48A339A32AA39CA38BA3F2E1FD
:10450000AF2EFE017396DE01119601900D92AA94D2
:10451000E1F7E4E6FBE0F0931D06E0931C06AFA193
:10452000A983B88609871A877B876C875D874E8742
:104530003F87288B9A8B898B82E1FE013196ADE211
:10454000B6E001900D928A95E1F73092F20D40921B
:10455000F30D5092A40ED0929D0EC0929C0E6092CC
:10456000170E7092A10E8092A00EF0929F0EE09214
:104570009E0E9092A50E88A599A59093A30E809368
:10458000A20E8DA19EA190931F0680931E0687E028
:1045900080930F0A1092100A61E00E943C4685E069
:1045A0009AE00E94AD881092110A1092120A80912E
:1045B0003806811102C0109239069091340691118B
:1045C00005C0811103C01092EC0AA3C081E0809362
:1045D000EC0A0091E70A1091E80A8091770A60E0FE
:1045E0000E943C46D801ED91FC910190F081E02DB4
:1045F000C801199580912D06882359F1813071F0F9
:104600008330C1F488E293E290932F0680932E06C4
:1046100089E08093320680E197E217C088EB9BE047
:1046200090932F0680932E0683E08093320688E9CC
:104630009AE30BC088E893E190932F0680932E06AF
:1046400086E08093320680EE9EE29093310680935E
:104650003006809134068823E9F180913806609114
:10466000320670E08823C9F080913A068823A9F0C9
:1046700080E090E00E9496B99B01AC0160E070E0A0
:1046800088EC92E40E94F1B56093200670932106B5
:10469000809322069093230625C080E090E00E943C
:1046A00096B99B01AC0160E070E088EC92E40E9456
:1046B000F1B56093200670932106809322069093B3
:1046C00023061092170610921806109219061092DF
:1046D0001A061FC010922006109221061092220680
:1046E000109223066091330670E080E090E00E9413
:1046F00096B99B01AC0160E070E088EC92E40E9406
:10470000F1B560931706709318068093190690937D
:104710001A0610922A061092240610921B06109276
:1047200025061092260610922706109228060E944F
:1047300074446E98769AEE9880916A008F7C80938C
:104740006A008091F30D882321F080916A008062D5
:1047500003C080916A00806380936A00EE980E9493
:104760001A4680E090E040E09C012D5F304FF90157
:10477000E955FF4F5081552331F032972081318127
:10478000232B09F04F5F03968837910569F7409313
:104790004106A0E5B6E020E030E089EC282E82E476
:1047A000382E92E9492E9CE5592E47E6642E4CE5B9
:1047B000742E5AE7852E5CE5952E6CECA62E62E4ED
:1047C000B62E4AE351E400E211E47DE2E72E71E403
:1047D000F72EE3E4CE2EE3E4DE2EC9018D5F904F89
:1047E000FC01E955FF4F6081662309F4B0C38B5586
:1047F0009F4FFC0180819181892B09F4A8C370E04F
:10480000FB013197ED39F10508F0A1C38827E75581
:10481000FF4F8F4F0C9478B588E29EE411969C93DD
:104820008E9395C386E29EE411969C938E938FC3DC
:1048300084E29EE411969C938E9389C38DE19EE45D
:1048400011969C938E9383C38BE19EE411969C9367
:104850008E937DC382EA9DE411969C938E9377C3D9
:1048600084EA9DE411969C938E9371C385E89DE440
:1048700011969C938E936BC381E79DE411969C9354
:104880008E9365C383E69DE411969C938E935FC3DC
:1048900087E09DE411969C938E9359C383EE9BE42D
:1048A00011969C938E9353C38AEF9CE411969C932C
:1048B0008E934DC38CEB9CE411969C938E9347C3CF
:1048C0008FEE9CE411969C938E9341C388EF9CE4F9
:1048D00011969C938E933BC381EF9CE411969C931D
:1048E0008E9335C38FED9CE411969C938E932FC3CA
:1048F0008DED9CE411969C938E9329C38BED9CE4E3
:1049000011969C938E9323C38BEC9CE411969C93FD
:104910008E931DC389EC9CE411969C938E9317C3D0
:104920008AEB9CE411969C938E9311C38AEA9CE4D3
:1049300011969C938E930BC388EA9CE411969C93EA
:104940008E9305C386EA9CE411969C938E93FFC2D6
:1049500089E49BE411969C938E93F9C287E49BE4CF
:1049600011969C938E93F3C285E49BE411969C93DD
:104970008E93EDC28AE59AE811969C938E93E7C2D6
:1049800084EA9CE411969C938E93E1C284E99CE4B2
:1049900011969C938E93DBC281E99BE411969C93C4
:1049A0008E93D5C282E79BE411969C938E93CFC2DF
:1049B00082E99CE411969C938E93C9C283E69CE4A1
:1049C00011969C938E93C3C28CE59CE411969C93A4
:1049D0008E93BDC28CE29CE411969C938E93B7C2D9
:1049E00083EC93E911969C938E93B1C281EE9BE484
:1049F00011969C938E93ABC28FED9BE411969C9382
:104A00008E93A5C28FE49FE411969C938E939FC2D0
:104A10008AE19FE411969C938E9399C28BED9EE45C
:104A200011969C938E9393C28DE49FE411969C9370
:104A30008E938DC288E19FE411969C938E9387C2DA
:104A400089ED9EE411969C938E9381C28BE49FE442
:104A500011969C938E937BC286E19FE411969C9362
:104A60008E9375C287ED9EE411969C938E936FC2D0
:104A700089E49FE411969C938E9369C284E19FE43C
:104A800011969C938E9363C285ED9EE411969C9340
:104A90008E935DC287E49FE411969C938E9357C2D8
:104AA00082E19FE411969C938E9351C283ED9EE424
:104AB00011969C938E934BC285E49FE411969C9330
:104AC0008E9345C280E19FE411969C938E933FC2E2
:104AD00081ED9EE411969C938E9339C283E49FE40A
:104AE00011969C938E9333C28EE09FE411969C9313
:104AF0008E932DC28FEC9EE411969C938E9327C2C9
:104B000081E49FE411969C938E9321C28CE09FE4F4
:104B100011969C938E931BC28DEC9EE411969C93F0
:104B20008E9315C28FE39FE411969C938E930FC2D0
:104B30008AE09FE411969C938E9309C28BEC9EE4CD
:104B400011969C938E9303C28DE39FE411969C93E0
:104B50008E93FDC188E09FE411969C938E93F7C1DC
:104B600089EC9EE411969C938E93F1C18BE39FE4B4
:104B700011969C938E93EBC186E09FE411969C93D3
:104B80008E93E5C187EC9EE411969C938E93DFC1D2
:104B900089E39FE411969C938E93D9C184E09FE4AE
:104BA00011969C938E93D3C185EC9EE411969C93B1
:104BB0008E93CDC183E99EE411969C938E93C7C1D9
:104BC00080E99EE411969C938E93C1C18DE89EE48A
:104BD00011969C938E93BBC18AE89EE411969C9398
:104BE0008E93B5C187E89EE411969C938E93AFC1D6
:104BF00084E89EE411969C938E93A9C181E89EE47B
:104C000011969C938E93A3C18EE79EE411969C937C
:104C10008E939DC186ED9BE411969C938E9397C1D4
:104C200083E49BE411969C938E9391C181E49BE471
:104C300011969C938E938BC180EB9BE411969C9371
:104C40008E9385C189E59BE411969C938E937FC1D9
:104C500084E293E411969C938E9379C18DE091E464
:104C600011969C938E9373C18BE091E411969C9363
:104C70008E936DC18FEF92E411969C938E9367C1D2
:104C800086EE92E411969C938E9361C185E292E444
:104C900011969C938E935BC18AED91E411969C933F
:104CA0008E9355C184EC9CE511969C938E934FC1D5
:104CB00080EB9CE511969C938E9349C18CE99CE511
:104CC00011969C938E9343C18BE993E911969C9323
:104CD0008E933DC189EF90E411969C938E9337C1DA
:104CE00087EE90E411969C938E9331C180E390E41B
:104CF00011969C938E932BC186EE9FE311969C9305
:104D00008E9325C188E090E411969C938E931FC1E9
:104D100088EF9FE311969C938E9319C18AE190E4EA
:104D200011969C938E9313C18EEB9FE311969C93E7
:104D30008E930DC18EEA9FE311969C938E9307C1CB
:104D400080ED9FE311969C938E9301C18EEC91E4CC
:104D500011969C938E93FBC082EC91E411969C93E8
:104D60008E93F5C086EB91E411969C938E93EFC0E1
:104D70008AEA91E411969C938E93E9C08EE991E4BE
:104D800011969C938E93E3C082E991E411969C93D3
:104D90008E93DDC086E891E411969C938E93D7C0E4
:104DA0008EEA90E411969C938E93D1C08CE990E4A6
:104DB00011969C938E93CBC08AE890E411969C93B5
:104DC0008E93C5C088E790E411969C938E93BFC0E4
:104DD00086E690E411969C938E93B9C084E590E4A6
:104DE00011969C938E93B3C082E490E411969C93A9
:104DF0008E93ADC083EE92E411969C938E93A7C0E0
:104E000080EE92E411969C938E93A1C08AED92E479
:104E100011969C938E939BC086E793E411969C9386
:104E20008E9395C087ED92E411969C938E938FC0DC
:104E300084ED92E411969C938E9389C08EEC92E45B
:104E400011969C938E9383C01196DC92CE927FC074
:104E50001196FC92EE927BC011961C930E9377C034
:104E600080E691E411969C938E9371C011965C93A9
:104E70004E936DC01196BC92AE9269C011969C92F1
:104E80008E9265C011967C926E9261C011965C9272
:104E90004E925DC011963C922E9259C0E6ECF2E41F
:104EA0001196FC93EE9353C08DEB92E411969C9374
:104EB0008E934DC0EAEBF2E41196FC93EE9347C05B
:104EC00087EB92E411969C938E9341C0E4EBF2E45D
:104ED0001196FC93EE933BC081EB92E411969C9368
:104EE0008E9335C0E6EAF2E41196FC93EE932FC060
:104EF0008FEA92E411969C938E9329C0E8EAF2E43B
:104F00001196FC93EE9323C08AED90E411969C9346
:104F10008E931DC0EDECF0E41196FC93EE9317C058
:104F200080EC90E411969C938E9311C0E4E9F2E436
:104F30001196FC93EE930BC082E892E411969C9339
:104F40008E9305C0E0E7F2E41196FC93EE932D5F9B
:104F50003F4F12962837310509F03FCC1092440696
:104F600080914806811114C080E090E0FC01E85572
:104F7000F04F20813181245631092436310528F043
:104F800003968837910591F703C081E0809344062A
:104F900010924A0680914E06811114C080E090E084
:104FA000FC01E855F04F20813181285C310924361D
:104FB000310528F003968837910591F703C081E009
:104FC00080934A068091B0069091B106DC01ED9184
:104FD000FC91E25BFF4F20917A1030917B10409161
:104FE0007810509179100190F081E02D61E01995D1
:104FF0008091B0069091B106DC01ED91FC91E25BED
:10500000FF4F20917E1030917F1040917C10509185
:105010007D100190F081E02D62E019958091B0063D
:105020009091B106DC01ED91FC91E25BFF4F209184
:105030008210309183104091801050918110019026
:10504000F081E02D63E019958091B0069091B10652
:10505000DC01ED91FC91E25BFF4F20918D103091CE
:105060008E1040918B1050918C100190F081E02DAA
:1050700064E019958091B0069091B106DC01ED9144
:10508000FC91E25BFF4F2091911030919210409182
:105090008F10509190100190F081E02D65E01995EE
:1050A0008091B0069091B106DC01ED91FC91E25B3C
:1050B000FF4F209195103091961040919310509190
:1050C00094100190F081E02D66E019958091B00672
:1050D0009091B106DC01ED91FC91E05BFF4F0190F6
:1050E000F081E02D4091841061E019958091B00627
:1050F0009091B106DC01ED91FC91E05BFF4F0190D6
:10510000F081E02D4091851062E019958091B00604
:105110009091B106DC01ED91FC91E05BFF4F0190B5
:10512000F081E02D4091861063E019958091B006E2
:105130009091B106DC01ED91FC91E05BFF4F019095
:10514000F081E02D4091971064E019958091B006B0
:105150009091B106DC01ED91FC91E05BFF4F019075
:10516000F081E02D4091981065E019958091B0068E
:105170009091B106DC01ED91FC91E05BFF4F019055
:10518000F081E02D4091991066E019958091B0066C
:105190009091B106DC01ED91FC9100ACF1ADE02DF8
:1051A0006091881019958091B0069091B106DC014C
:1051B000ED91FC9104ACF5ADE02D60919D10199539
:1051C0008091B0069091B106DC01ED91FC9106A4AE
:1051D000F7A5E02D6091891019958091B006909106
:1051E000B106DC01ED91FC9104A8F5A9E02D6091D8
:1051F0008A1019958091B0069091B106DC01ED916D
:10520000FC91EA5BFF4F0190F081E02D40919E10F0
:1052100060E019958091B0069091B106DC01ED91A6
:10522000FC91EA5BFF4F0190F081E02D40919F10CF
:1052300061E0199580E090E09C012D5F304FF9010D
:10524000E955FF4F4081423731F432972081318157
:10525000232B09F0B5C003968837910569F70E94A2
:1052600012948091B0069091B106DC01ED91FC9111
:10527000E05AFF4F0190F081E02D40E060919A10DC
:1052800019958091B0069091B106DC01ED91FC91E9
:10529000E05AFF4F0190F081E02D41E060919C10B9
:1052A00019958091B0069091B106DC01ED91FC91C9
:1052B000E05AFF4F0190F081E02D42E060919B1099
:1052C000199580917110882331F0809122108D30D2
:1052D00011F010927110109211071092740E8091BB
:1052E00072108093110680917410809310062091A3
:1052F000C51030E0AFEFB0E00E9429BB24E630E0FB
:1053000040E050E00E94DBBA20933B138091C41030
:1053100081110E942A8C0E9493970E9400496B0180
:105320007C0110E011110FC08091B706882359F05D
:105330002FE031E440ED57E060E070E084E69BE070
:105340000E94453E11E00E946071882351F00E9446
:10535000458B0E9417600E94D18B0E94ED700E94C5
:10536000618B0E944A82029711F00E94924F0E9424
:10537000E1940E944A820297A9F60E940049DC014A
:10538000CB018C199D09AE09BF098C3B9240A10548
:10539000B10540F218C082E00E94D49281110DC084
:1053A0005AC882E00E94B892882309F45AC883E060
:1053B0008FA357C8F1E0FFA354C822E02FA351C820
:1053C0000E9406944ECF0E9440970E94D18B8091FC
:1053D000000B811102C00E9455760E941F8286E355
:1053E0000E948448BC01990F880B990B61157105C7
:1053F0008105910511F00E941DB929EA3FE348EEAD
:1054000053E060E070E084E69BE0AB960FB6F89462
:10541000DEBF0FBECDBFDF91CF911F910F91FF90E7
:10542000EF90DF90CF90BF90AF909F908F907F9044
:105430006F905F904F903F902F900C94453E7F92DD
:105440008F929F92AF92BF92CF92DF92EF92FF9294
:105450000F931F93CF93DF9381E08093D10D8093BF
:10546000D40D8093D70D8093DA0D8093E60D809351
:10547000E90D909161109150953040F0809361104A
:1054800061E070E08EE591E00E94E8749091611017
:105490002DEF290F80912010233008F006C28A30AA
:1054A00079F03CF4883009F461C0893009F4B7C15F
:1054B000ADC18B3009F4A0C08C3009F4E1C0A6C1A5
:1054C00084E290E00E9492B6FC018091D41028E022
:1054D00030E0338322838824839499249A9495829C
:1054E0008482AA24AA94B12CB782A682118610863F
:1054F000108E33E8D32ED18E44EBE42E47E0F42E09
:10550000F38EE28E02E614E011830083C9EBD0E152
:10551000D1A3C0A312A283A3F093A606E093A5068D
:10552000CF010E94055784E290E00E9492B6FC01F0
:105530008091D41029E030E03383228395828482E5
:10554000B782A68211861086108ED18EF38EE28EDF
:1055500011830083D1A3C0A312A283A3F093A40656
:10556000E093A306CF010E940557FEC280E290E0BF
:105570000E9492B6FC0188E090E093838283AA2483
:10558000A394BB24BA94B582A482CC24CA94D12C0F
:10559000D782C68211861086108E0AE0F02EF18E18
:1055A00004EB17E0138F028FCAE4D4E0D183C083E9
:1055B000F093A606E093A506CF010E946E5680E206
:1055C00090E00E9492B6FC0189E090E09383828390
:1055D000B582A482D782C68211861086108EF18E83
:1055E000138F028FD183C083F093A406E093A306A8
:1055F000CF010E946E56B8C289E190E00E9492B637
:10560000FC0188E090E093838283EE24E394FF24FE
:10561000FA94F582E4820FEF10E017830683118677
:105620001086108ECEE3D4E0D183C083F093A6061B
:10563000E093A506CF010E945E6F1092E60D809167
:105640006110843009F090C289E190E00E9492B626
:10565000FC0189E090E093838283F582E4821783E2
:10566000068311861086108ED183C083F093A40622
:10567000E093A306CF010E945E6F1092E90D74C201
:10568000943009F049C089E190E00E9492B6EC01A3
:10569000FAEEAF2EF5E0BF2EB982A88287E090E047
:1056A0009B838A83CC24C394DD24DA94DD82CC826C
:1056B000EE24EA94F12CFF82EE8219861886188E69
:1056C000CE010E94098002E314E019830883D0937D
:1056D000A606C093A506CE010E94F66D1092D10DCC
:1056E00089E190E00E9492B6EC01B982A88286E03E
:1056F00090E09B838A83DD82CC82FF82EE821986D2
:105700001886188ECE010E94098019830883D093D1
:10571000A406C093A3064BC0953009F04EC089E1A2
:1057200090E00E9492B6EC016AEEA62E65E0B62EDD
:10573000B982A88287E090E09B838A83CC24C394BB
:10574000DD24DA94DD82CC82EE24EA94F12CFF820F
:10575000EE8219861886188ECE010E94098002E317
:1057600014E019830883D093A406C093A306CE0146
:105770000E94F66D1092D10D89E190E00E9492B6E0
:10578000EC01B982A88286E090E09B838A83DD8267
:10579000CC82FF82EE8219861886188ECE010E9476
:1057A000098019830883D093A606C093A506CE016D
:1057B0000E94F66D1092D40DD7C189E190E00E944D
:1057C00092B6EC018AEE95E09983888387E090E0B9
:1057D0009B838A8381E09FEF9D838C838FEF90E092
:1057E0009F838E8319861886188ECE010E940980A9
:1057F00082E394E099838883D093A606C093A5069C
:10580000CE010E94F66D1092D10DAEC189E0809359
:10581000201069E070E08DE191E00E94E87480E280
:1058200090E00E9492B6FC0188E090E0938382832E
:10583000AA24A394BB24BA94B582A482CC24CA948B
:10584000D12CD782C68211861086108E50E8F52E94
:10585000F18E04EB17E0138F028FC6E5D4E0D183FD
:10586000C083F093A606E093A506CF010E94B05630
:1058700080E290E00E9492B6FC0189E090E0938380
:105880008283B582A482D782C68211861086108E4A
:10589000F18E138F028FD183C083F093A406E0931F
:1058A000A306CF010E94B0565FC18A3009F456C0EA
:1058B0003CF4883009F4A0C0893009F400C1F6C076
:1058C0008B3009F4BAC08C3009F0F0C089E190E067
:1058D0000E9492B6EC017AEEA72E75E0B72EB9823F
:1058E000A88287E090E09B838A83CC24C394DD2444
:1058F000DA94DD82CC82EE24EA94F12CFF82EE82EF
:1059000019861886188ECE010E94098002E314E0E1
:1059100019830883D093A806C093A70689E190E075
:105920000E9492B6EC01B982A88286E090E09B8347
:105930008A83DD82CC82FF82EE8219861886188ED9
:10594000CE010E94098019830883D093AA06C093D0
:10595000A9061092D10D1092D40DF0C084E290E00F
:105960000E9492B6FC01C091D410D0916D1088E0D5
:1059700090E0938382838824839499249A949582D7
:105980008482AA24AA94B12CB782A682118610869A
:10599000108E83E8782E718E94EBC92E97E0D92E65
:1059A000D38EC28E22E6E22E24E0F22EF182E08235
:1059B00009EB10E111A300A3D2A3C3A3F093A8069F
:1059C000E093A70684E290E00E9492B6FC0189E091
:1059D00090E09383828395828482B782A682118627
:1059E0001086108E718ED38EC28EF182E08211A34A
:1059F00000A3D2A3C3A39EC080E290E00E9492B60F
:105A0000FC0188E090E093838283AA24A394BB24C2
:105A1000BA94B582A482CC24CA94D12CD782C682EF
:105A200011861086108EDAE0FD2EF18E04EB17E061
:105A3000138F028FCAE4D4E062C089E190E00E9433
:105A400092B6FC0188E090E093838283EE24E39495
:105A5000FF24FA94F582E4820FEF10E017830683A7
:105A600011861086108ECEE3D4E0D183C083F093EC
:105A7000A806E093A70689E190E00E9492B6FC0197
:105A800089E090E093838283F582E4821783068322
:105A900011861086108ED183C083F093AA06E093FE
:105AA000A9061092E60D1092E90D48C089E0809396
:105AB000201069E070E08DE191E00E94E87480E2DE
:105AC00090E00E9492B6FC0188E090E0938382838C
:105AD000AA24A394BB24BA94B582A482CC24CA94E9
:105AE000D12CD782C68211861086108E60E8F62EE1
:105AF000F18E04EB17E0138F028FC6E5D4E0D1835B
:105B0000C083F093A806E093A70680E290E00E948D
:105B100092B6FC0189E090E093838283B582A482EF
:105B2000D782C68211861086108EF18E138F028F57
:105B3000D183C083F093AA06E093A9068091A906B9
:105B40009091AA06DC01ED91FC910280F381E02D99
:105B500019958091A7069091A806DC01ED91FC9122
:105B60000280F381E02D199580916110833039F026
:105B7000823009F06CC0809120108C3051F189E1A5
:105B800090E00E9492B6EC018AEE95E099838883BA
:105B900086E090E09B838A8381E09FEF9D838C83E6
:105BA0008FEF90E09F838E8319861886188ECE0122
:105BB0000E94098082E394E099838883D093A106B0
:105BC000C093A006CE010E94F66D1092D40DC6E0DF
:105BD00029C089E190E00E9492B6EC018AEE95E03E
:105BE0009983888384E090E09B838A8381E09FEFA0
:105BF0009D838C838FEF90E09F838E831986188618
:105C0000188ECE010E94098082E394E099838883F4
:105C1000D093A106C093A006CE010E94F66D10920B
:105C2000DA0DC4E060912F10709130108C2F0E941B
:105C3000207F60913110709132108C2F0E941B7F59
:105C400080913310E091A006F091A106808FE09141
:105C500021108E2FEE0F990BAA0BBB0BFC0138976E
:105C6000E830F10508F0BBC08827EA5BFE4F8F4F94
:105C70000C9478B584E290E00E9492B6FC01809189
:105C8000D41028E030E03383228321E03FEF3583D6
:105C900024832FEF30E03783268311861086108E01
:105CA00094E8918F24EB37E0338F228F22E634E0A3
:105CB0003183208329EB30E131A320A312A283A3F7
:105CC0001EC080E290E00E9492B6FC0188E090E065
:105CD0009383828381E09FEF958384838FEF90E0AD
:105CE0009783868311861086108E87E8818F84EBD8
:105CF00097E0938F828F86E594E091838083F09381
:105D0000AF06E093AE0699C080E290E00E9492B6A2
:105D1000FC0188E090E09383828381E09FEF95838C
:105D200084838FEF90E09783868311861086108E90
:105D30008DE0818F84EB97E0938F828F8AE494E0EB
:105D4000DCCF89E190E00E9492B6FC0188E090E00F
:105D50009383828381E09FEF958384838FEF90E02C
:105D60009783868311861086108E8EE394E091834C
:105D70008083F093AF06E093AE061092E60D5DC00F
:105D80008CE190E00E9492B6EC018AEE95E0998356
:105D9000888385E090E09B838A8381E09FEF9D83E9
:105DA0008C838FEF90E09F838E8319861886188EE0
:105DB000CE010E9409808EED95E037C089E190E028
:105DC0000E9492B6FC0113821282158214821782FD
:105DD000168211861086108E8EE094E08ECF8CE0B5
:105DE000809321106CE070E08EE191E00E94E874F5
:105DF00089E190E00E9492B6EC018AEE95E09983E9
:105E0000888385E090E09B838A8381E09FEF9D8378
:105E10008C838FEF90E09F838E8319861886188E6F
:105E2000CE010E94098082E394E099838883D09315
:105E3000AF06C093AE061092D70D8091AE0690913A
:105E4000AF06DC01ED91FC910280F381E02D199504
:105E500080912910843658F4853608F084E664E68B
:105E6000681B8091AE069091AF060E949B5780916F
:105E700021108C508230A8F460912A1070912B1060
:105E800085E00E945D3F60912C1070912D1085E09F
:105E90000E94423F80912E10E091AE06F091AF0635
:105EA000808F20912210822F022E000C990BAA0BBA
:105EB000BB0BFC013897E830F10508F089C0882752
:105EC000E25BFE4F8F4F0C9478B584E290E00E9425
:105ED00092B6FC018091D41029E030E03383228314
:105EE00021E03FEF358324832FEF30E03783268393
:105EF00011861086108E94E8918F24EB37E0338F53
:105F0000228F22E634E03183208329EB30E131A374
:105F100020A312A283A357C080E290E00E9492B611
:105F2000FC0189E090E09383828381E09FEF958379
:105F300084838FEF90E09783868311861086108E7E
:105F400087E8818F84EB97E0938F828F86E594E0DA
:105F500038C080E290E00E9492B6FC0189E090E0B7
:105F60009383828381E09FEF958384838FEF90E01A
:105F70009783868311861086108E8DE0818F84EB47
:105F800097E0938F828F8AE494E01BC08091611028
:105F9000823009F0BBC1809120108C3009F0B6C16D
:105FA0001FC089E190E00E9492B6FC011382128228
:105FB000158214821782168211861086108E8EE04A
:105FC00094E091838083F093B306E093B2065EC0C1
:105FD00080916110823061F5809120108C3041F504
:105FE0008BE0809322106BE070E08FE191E00E94E3
:105FF000E87489E190E00E9492B6FC0189E090E0AB
:106000009383828381E09FEF958384838FEF90E079
:106010009783868311861086108E8EE394E0918399
:106020008083F093B306E093B2061092E90D2EC080
:106030008CE0809322106CE070E08FE191E00E9490
:10604000E87489E190E00E9492B6EC018AEE95E056
:106050009983888384E090E09B838A8381E09FEF2B
:106060009D838C838FEF90E09F838E8319861886A3
:10607000188ECE010E94098082E394E09983888380
:10608000D093B306C093B2061092DA0D8091B20697
:106090009091B306DC01ED91FC910280F381E02D3B
:1060A000199580912810843658F4853608F084E6D6
:1060B00064E6681B8091B2069091B3060E949B57DC
:1060C000809122108C50823000F5609123107091E5
:1060D000241084E00E945D3F60912510709126108D
:1060E00084E00E94423F80912710E091B206F09137
:1060F000B306808F809122108D3039F48091271063
:10610000E091A60EF091A70E808F8EE190E00E94A4
:1061100092B6EC01F0903810C0903C10D0903D1039
:10612000A0903A10B0903B108AEE95E09983888356
:1061300083E090E09B838A8381E09FEF9D838C8343
:106140000FEF10E01F830E8319861886188ECE017C
:106150000E94098086E294E099838883BA8EA98E92
:10616000DC8ECB8EFD8ED093160EC093150E6091F3
:106170003E1070913F1083E00E945D3F609140109F
:106180007091411083E00E94423F80913810E0916D
:10619000150EF091160E808F809138100E94B37406
:1061A0008091150E9091160EDC01ED91FC9102800C
:1061B000F381E02D199580914210882339F185E211
:1061C00090E00E9492B6FC01809147109091481097
:1061D0002091451030914610409143105091441049
:1061E00068E070E0738362831582148217830683EC
:1061F00011861086108E6AE174E071836083528F7D
:10620000418F348F238F968F858F22C085E290E057
:106210000E9492B6FC018091451090914610209109
:1062200043103091441048E050E05383428315827C
:1062300014821783068311861086108E4AE154E07B
:1062400051834083328F218F948F838F168F058FD8
:10625000F0932C06E0932B0680912B0690912C0650
:106260000E943C6F8091E60D8823F9F089E190E06F
:106270000E9492B6FC0188E090E0938382831582AD
:1062800014828FEF93E0978386838FEF91E091875D
:106290008087108E8EE394E091838083F093E50DE8
:1062A000E093E40DCF010E945E6F8091E90D882399
:1062B00009F474C089E190E00E9492B6FC0189E083
:1062C00090E093838283158214828FEF93E097830B
:1062D00086838FEF91E091878087108E8EE394E024
:1062E00091838083F093E80DE093E70DCF01DF9178
:1062F000CF911F910F91FF90EF90DF90CF90BF90C3
:10630000AF909F908F907F900C945E6F2C3009F42B
:1063100098CE8CE190E00E9492B6EC018AEE882E35
:1063200085E0982E9982888294E0A92EB12CBB82B8
:10633000AA82CC24C394DD24DA94DD82CC82EE24BC
:10634000EA94F12CFF82EE8219861886188ECE010F
:106350000E9409800EED15E019830883D093B306DF
:10636000C093B2068CE190E00E9492B6EC01998253
:106370008882BB82AA82DD82CC82FF82EE8219866D
:106380001886188E0E94098019830883D093A70E5F
:10639000C093A60ECE010E94B86E76CEDF91CF914B
:1063A0001F910F91FF90EF90DF90CF90BF90AF9033
:1063B0009F908F907F9008952F923F924F925F927F
:1063C0006F927F928F929F92AF92BF92CF92DF9205
:1063D000EF92FF920F931F93CF93DF93CDB7DEB76A
:1063E000C65AD1090FB6F894DEBF0FBECDBFCDB6E9
:1063F000DEB6CC55DF4F1882C45AD040CD55DF4FA2
:106400001882C35AD0408091A80D8A3709F447C03A
:10641000C0F4873709F4D9C238F48F3109F430C594
:10642000863709F4E2C1F2C5883709F4DDC289373D
:1064300009F0ECC50E9408820E9400492B013C0132
:1064400029C08E3709F42EC338F48B3709F4CAC13A
:106450008C3709F4D8C2DAC5813809F402C582380C
:1064600009F4EDC4803809F0D1C565C40E94004923
:10647000DC01CB0184199509A609B7098032934044
:10648000A105B10508F007C50E94924F0E9408823D
:106490000E942D560E944A82029741F7FCC40E9436
:1064A0004A82029729F060E084E80E94C1968BC17D
:1064B0008091010B823031F0833039F482E0809397
:1064C000260E03C081E08093EF1281E08093B20D2D
:1064D0008E010C551F4F2BE0AE0144575F4F68E80B
:1064E00071E90E943B960E941F82893058F001504A
:1064F00011092BE0AE014F575F4F68E872E981E068
:106500000E943B961092B10D772473940E943582BD
:10651000882309F43DC1198222961FAE22978091EB
:10652000B10D81110EC0BE0164577F4FCE018F5B4C
:106530009F4F0E94B0B8CC55DF4F0881C45AD0405D
:106540000FC07092B10DBE016F577F4FCE018F5BB0
:106550009F4F0E94B0B8CD55DF4F0881C35AD0403D
:106560001091B10DADB6BEB68091FD0AEDB7FEB784
:1065700022E0829FE019F10911240FB6F894FEBFC2
:106580000FBEEDBF8DB79EB701967C016EE076E041
:10659000CE0183569F4F0E94507A8091010B82302A
:1065A00089F0833061F1813009F0A1C04091FD0A8A
:1065B00050E0B7018091C8129091C9120E946052B8
:1065C00010E039C02091FD0A30E05FB7F89440E058
:1065D000842F90E08217930774F4880F991FF701B6
:1065E000E80FF91FDC01A253BD4E8D919C91918360
:1065F00080834F5FEDCF5FBF1092EE121CC02091E1
:10660000FD0A30E05FB7F89440E0842F90E08217F5
:10661000930774F4880F991FF701E80FF91FDC0145
:10662000A45DB14F8D919C91918380834F5FEDCF9D
:106630005FBF1092C5126DE270E0CE0183569F4F8E
:106640000E947F792091FD0A293048F0112321F022
:10665000113021F418E004C028E001C020E010E06F
:10666000121758F5F701E10FF11DE10FF11D6081DF
:1066700071814AE0CE0189569F4FCB55DF4F288369
:10668000C55AD0400E94257ABE0169567F4FCE017F
:1066900083569F4F0E94A679CE0189569F4F0E9434
:1066A000207ACE0183569F4F0E94D28C1F5FCB551C
:1066B000DF4F2881C55AD040D3CF40E450E0BE011F
:1066C0006F5F7F4FCE0183569F4F0E94C98CCF557D
:1066D000DF4F1881C15AD040CE0183569F4F0E9490
:1066E000207A0FB6F894BEBE0FBEADBE0BC0CE0171
:1066F00083569F4F0E94207A0FB6F894BEBE0FBEFD
:10670000ADBE10E0BE016F5F7F4FCE018F5B9F4F2C
:106710000E94B0B8010F10E0E1E4F0E0EC0FFD1FC3
:10672000E00FF11F1082BE016F5B7F4F80919413C9
:10673000909195130E94B37AB801CE018F5B9F4F61
:106740000E944A56BC0180919413909195130E9427
:10675000D7756AE080919413909195130E94887A7E
:106760008091941390919513DC01ED91FC9102843A
:10677000F385E02D19950E941F82893048F08091A1
:10678000B10D811103C07092B10D02C01092B10D14
:106790000E9408820E942D560E94EA6F81110CDE31
:1067A0008091A70D81110FC08091B20D882359F0FF
:1067B0008091210E811107C08091A50D9091A60DA9
:1067C0000A970CF4A3CE8091010B823039F083300C
:1067D00009F01CC481E08093260E18C481E08093E8
:1067E000EF1214C41092B20D48C31091AB0D8FEF8D
:1067F000810F853028F060E089E80E94C19606C4C8
:10680000133079F018F41230F9F004C0143079F034
:10681000153099F040E6442E49E0542E612C712C3D
:1068200019C0412C3BE4532E612C712C13C0412C18
:1068300026E9522E612C712C0DC0412C92EC592E60
:1068400066246394712C06C080E8482E85E2582E99
:10685000612C712C00E0E12EF12C5701BFE8AB0E4A
:10686000B11C1501E89427F83324E6E9EE0EF11C7B
:10687000E894E7F8FF24023091F018F4013051F069
:1068800004C0033089F00430A1F040E659E060E034
:1068900070E013C040E855E260E070E00EC040E0F8
:1068A0005BE460E070E009C040E056E960E070E061
:1068B00004C040E052EC61E070E084EB97E00E949D
:1068C000F46C84EB97E00E94FA780E9400494B0137
:1068D0005C01F2E38F0E911CA11CB11C0E94ED55CE
:1068E0000E940049681579058A059B05B8F360E8A0
:1068F00070E084EB97E00E94DE716FE070E084EB63
:1069000097E00E94DE71612F84EB97E00E94B478DB
:10691000B10184EB97E00E94DE710E9400494B01B7
:106920005C012AE0820E911CA11CB11C0E94ED5555
:106930000E940049681579058A059B05B8F367E848
:1069400070E084EB97E00E94DE716FE070E084EB12
:1069500097E00E94DE71612F84EB97E00E94B4788B
:10696000B70184EB97E00E94DE7184EB97E00E9410
:10697000FA780E9400494B015C013EE5830E31E04C
:10698000931EA11CB11C0E94ED550E940049681580
:1069900079058A059B05B8F30F5F053009F06BCFC9
:1069A000B301A20184EB97E00E94F46C4092B9100D
:1069B0005092BA106092BB107092BC10B301A20149
:1069C00086EB91E00E94058D58C283E090E00E9422
:1069D00092B62AE0DC012C9324EB37E012963C932C
:1069E0002E9311976AE00CC083E090E00E9492B66B
:1069F0002DE0FC01208324EB37E0328321836DE01E
:106A00000E94BC513AC24091AB0D5091AC0D009127
:106A1000AD0D1091AE0D6091A90D7091AA0DCE0132
:106A20000196CB55DF4F4883C55AD040CA55DF4F3A
:106A30005883C65AD0400E940A87CB55DF4F488101
:106A4000C55AD040CA55DF4F5881C65AD040892B0D
:106A5000E9F08D81873050F4853080F48130B0F0DA
:106A6000642F8B819C810E943B760DC0893070F42D
:106A7000B8018B819C810E94058D05C0BA018B8174
:106A80009C810E94E8740E943D9704C061E085E803
:106A90000E94C1968091A40D8111B8C281E08093BB
:106AA000A40DB4C2B090A90DE090AA0DC956DF4F55
:106AB0001882C759D0406EE076E0CE018F579F4FC5
:106AC0000E94507A6B2D7E2DCE0184579F4F0E94DD
:106AD0000A87892B09F4C9C0C057DF4FE881C05924
:106AE000D0404E2F50E0FA013197E830F10508F020
:106AF000BCC08827EA5AFE4F8F4F0C9478B5C25716
:106B0000DF4F88819981CE58D0400E94BBBA23962E
:106B10001FAE1EAE239725961FAE1EAE2597279655
:106B20001FAE1EAE27974AE0BE016F5F7F4F90E019
:106B30003EC0C257DF4F88819981CE58D0400E9415
:106B4000BBBA682F880F770B4AE00AC0C257DF4FE5
:106B500088819981CE58D0400E94C8BA4AE0BC01D1
:106B6000CE0101960E94257ABE016F5F7F4FCE0154
:106B70008F579F4F0E944679CE01019663C0C2573E
:106B8000DF4F88819981CE58D0400E94C8BA2396A1
:106B90001FAE1EAE239725961FAE1EAE25972796D5
:106BA0001FAE1EAE27974AE0BE016F5F7F4F0E9467
:106BB00069B935C0C257DF4F88819981CE58D0401E
:106BC0000E94C3BA23961FAE1EAE239725961FAE12
:106BD0001EAE259727961FAE1EAE27972AE0AE0160
:106BE0004F5F5F4F0E943AB91AC0C257DF4F88818A
:106BF0009981CE58D0400E94C3BA23961FAE1EAED4
:106C0000239725961FAE1EAE259727961FAE1EAE64
:106C100027972AE0AE014F5F5F4F0E9448B9BE013F
:106C20006F5F7F4FCE018F5B9F4F0E94007ABE0146
:106C30006F5B7F4FCE018F579F4F0E944679CE01E9
:106C40008F5B9F4F0E94207A4BE050E0BE016F5B4C
:106C50007F4FCE018F579F4F0E94C98CCB57DF4F7C
:106C6000F880C558D04011E002C0F12C10E0CE01F0
:106C70008F579F4F0E94207A112309F4BCCD8E01BB
:106C800009561F4F20E4AE014F5F5F4F68E87B2D30
:106C90008E2D0E943B96BE016F5B7F4FCE01019609
:106CA0000E94B0B8C956DF4F8881C759D040F80E4E
:106CB00081E08F0DC956DF4F8883C759D040E1E08E
:106CC000F0E0EC0FFD1FEF0DF11D9CE79083E1E07C
:106CD000F0E0EC0FFD1FE80FF11D1082BE016F5FA9
:106CE0007F4F80919413909195130E94B37AC95667
:106CF000DF4F6881C759D04070E0CE0101960E94F5
:106D00004A56BC0180919413909195130E94D775B7
:106D10006AE080919413909195130E94887A8091F3
:106D2000941390919513DC01ED91FC910284F3850D
:106D3000E02D19956BC18091A90D9091AA0D803815
:106D4000910509F063C18E0104571F4F20E4AE0185
:106D50004F5F5F4F68E870E880E00E943B9662EF0B
:106D600075E0CE018F579F4F0E94507ACE018F570A
:106D70009F4F0E94D28CC457DF4F2881CC58D040FF
:106D8000CB57DF4F88819981C558D040820F911D24
:106D9000C457DF4F8883CC58D04022961FAE22972D
:106DA0004BE050E0BE016F5B7F4FCE018F579F4F8E
:106DB0000E94D977BE016F5B7F4FCE0101960E9482
:106DC000B0B8C457DF4F8881CC58D040E1E0F0E044
:106DD000EC0FFD1FE80FF11D1082BE016F5F7F4FAA
:106DE00080919413909195130E94B37AC457DF4F0A
:106DF0006881CC58D04070E0CE0101960E944A567E
:106E0000BC0180919413909195130E94D7756AE00C
:106E100080919413909195130E94887A8091941395
:106E200090919513DC01ED91FC910284F385E02DA6
:106E30001995CE018F579F4F0E94207AE7C080910D
:106E4000A90D9091AA0D8238910509F0DFC08E013D
:106E500004571F4F20E4AE014F5F5F4F68E872E8B0
:106E60007BCF8091A90D9091AA0D8138910509F0F1
:106E7000CDC08091B20D8111C9C00E943D97C6C09E
:106E80008091A90D9091AA0D4F9709F0BFC081E0A4
:106E90008093A70DBBC00E944A82029719F060E060
:106EA00084E8ABCC8091000B811102C00E94557622
:106EB0000E941F82F82E6EE076E0CE0184579F4F2D
:106EC0000E94507AC956DF4F1882C759D0408E01B0
:106ED00009561F4F20E4AE014F5F5F4F68E879E726
:106EE00080E00E943B96CF57DF4F19821882C1582D
:106EF000D040CD57DF4F19821882C358D040CB57AE
:106F0000DF4F19821882C558D0406F2D70E080E0A5
:106F100090E02AE0AE014F5B5F4F0E943AB9BE019C
:106F20006F5B7F4FCE018F579F4F0E94007ABE014B
:106F30006F577F4FCE0184579F4F0E944679CE01F5
:106F40008F579F4F0E94207A4BE050E0BE016F5B4D
:106F50007F4FCE0184579F4F0E94D977C057DF4F94
:106F60001881C059D040BE016F5B7F4FCE010196A2
:106F70000E94B0B8C956DF4F8881C759D040810FF1
:106F800091E0980FC956DF4F9883C759D040E1E090
:106F9000F0E0EC0FFD1FE80FF11D8CE78083E1E0CE
:106FA000F0E0EC0FFD1FE90FF11D1082BE016F5FD5
:106FB0007F4F80919413909195130E94B37AC95694
:106FC000DF4F6881C759D04070E0CE0101960E9422
:106FD0004A56BC0180919413909195130E94D775E5
:106FE0006AE080919413909195130E94887A809121
:106FF000941390919513DC01ED91FC910284F3853B
:10700000E02D1995CE0184579F4F16CF0FB6F894F7
:10701000DEBE0FBECDBECA55DF4F0FB6F894DEBF41
:107020000FBECDBFDF91CF911F910F91FF90EF90D9
:10703000DF90CF90BF90AF909F908F907F906F9098
:107040005F904F903F902F9008951092E50A089519
:10705000FC01128213821482158216821782128614
:10706000089580E00895CF93DF93C7E7DAE081E0E9
:1070700090E09A8389831092E50A0E94A3486C836A
:107080007D838E839F83E49AEC9ADF91CF9108955C
:107090000F931F93CF938C0169E070E18EEE98E01F
:1070A0000E948F7AD8011896ED91FC911997608112
:1070B00071818EEE98E00E94F271C1E0D8011A96BB
:1070C0008C91C81710F564E070E18EEE98E00E9494
:1070D0008F7A6C2F8EEE98E00E94AD7461E070E1C3
:1070E0008EEE98E00E948F7AF80190858185E92FD5
:1070F000F82FEC0FF11DEC0FF11D608171818EEE08
:1071000098E00E94F271CF5FD9CFCF911F910F917C
:1071100008951F920F920FB60F9211240BB60F9283
:107120001F932F933F934F935F936F937F938F930F
:107130009F93AF93BF93EF93FF93CF93DF9300D0D1
:107140001F92CDB7DEB78091770A0E94AE4411E05E
:10715000892B09F010E00E94A34869837A838B830E
:107160009C8389819A81AB81BC8140917B0A50913B
:107170007C0A60917D0A70917E0A841B950BA60B98
:10718000B70B2091780A3091790A2430310509F43F
:107190004CC02530310521F021303105E9F414C00F
:1071A00020917A0A222339F02091E50A20FF02C0BB
:1071B000289A01C02898112379F0813E2EE2920787
:1071C000A105B10548F02BC0112379F125E030E08D
:1071D0003093790A2093780A2091780A3091790ABD
:1071E0002530310511F5E091E50AF0E0EE0FFF1FC3
:1071F000E158F54F9183808389819A81AB81BC816D
:1072000080937B0A90937C0AA0937D0AB0937E0AB8
:107210008091E50A8F5F8093E50A833330F084E044
:1072200090E09093790A8093780A0F900F900F90D6
:107230000F90DF91CF91FF91EF91BF91AF919F910F
:107240008F917F916F915F914F913F912F911F91FE
:107250000F900BBE0F900FBE0F901F90189580914E
:10726000BD0D9091BE0D91609093BE0D8093BD0DAC
:1072700008958091BD0D9091BE0D80689093BE0DD4
:107280008093BD0D08958091BD0D9091BE0D8061DC
:107290009093BE0D8093BD0D0895FC0182818823DB
:1072A00071F08381882359F013828091BD0D9091F4
:1072B000BE0D24E082279093BE0D8093BD0D0895EE
:1072C000FC018281882371F0838181110BC081E0F0
:1072D00083838091BD0D9091BE0D84609093BE0D0F
:1072E0008093BD0D0895FC018481882371F0858110
:1072F000882359F015828091BD0D9091BE0D28E034
:1073000082279093BE0D8093BD0D0895FC0184816A
:10731000882371F0858181110BC081E08583809184
:10732000BD0D9091BE0D88609093BE0D8093BD0DF4
:1073300008958091BD0D9091BE0D20E2822790931B
:10734000BE0D8093BD0D08958091BD0D9091BE0D31
:1073500080629093BE0D8093BD0D0895DC01ED9188
:10736000FC910680F781E02D60E070E0199477FFD2
:1073700003C07195619571096F3F710519F014F0A3
:107380006FEF70E08091BD0D9091BE0D8C7B917080
:107390009093BE0D8093BD0D8091BD0D9091BE0D5B
:1073A0006F30710514F480641FC06733710514F4E5
:1073B00081641AC06F3571051CF48164906114C03A
:1073C000673871051CF4816490630EC06F3A7105D3
:1073D0001CF48164906408C0673D71051CF48164ED
:1073E000906502C0816490669093BE0D8093BD0D40
:1073F000089580E094E09093BE0D8093BD0D0895B4
:107400008091BD0D9091BE0D92609093BE0D8093C2
:10741000BD0D8091BD0D9091BE0D80649093BE0D09
:107420008093BD0D089508950895089508950895D1
:107430000895089508950895089580E008950895A1
:107440000895089508950895089508950895089554
:107450000895089508950895089508950895089544
:107460000895089580E0089508950895FC016483C7
:107470000895FC0162830895FC0113821482158231
:10748000168217821086118608950895089508952A
:10749000FC0183810895FC0165830895FC016483E8
:1074A0000895FC0160870895FC0166830895FC013E
:1074B00082810895FC01128213821482158261E098
:1074C00086E10E943C4661E086E10E94D644E2E704
:1074D000F0E08081816080831092BE0D1092BD0D1E
:1074E0000895FF920F931F93CF93DF938C01C62FC4
:1074F000F42ED22F6AED70E0DC011A968D919C91EA
:107500001B970E94DE71F80182859385DC01ED9165
:10751000FC910190F081E02D6C2F1995F801828586
:107520009385DC01ED91FC910190F081E02D6F2DB0
:107530001995F80182859385DC01ED91FC9101900C
:10754000F081E02D6D2F1995EC2FF0E0BF01665210
:107550007F4F6F0D711D6D0F711D6F777727F801CC
:1075600082859385DF91CF911F910F91FF900C94AD
:10757000DE7120E040E0B5CF65E4FBCF68E4F9CFF1
:10758000CF93DF93FC012381222321F0EC0161E4FE
:10759000F0DF1B82DF91CF910895CF93DF93FC0141
:1075A0002381211105C0EC0160E4E3DF81E08B83DE
:1075B000DF91CF910895FC012581222311F060E530
:1075C000D8CF0895FC012481222311F06CE3D1CFA0
:1075D0000895FC012085222331F02185222319F012
:1075E00011866BE3C6CF0895FC012085222339F074
:1075F0002185211104C021E021876AE3BACF0895D3
:10760000FC012681222331F02781222319F01782E1
:1076100069E3AFCF0895FC012681222339F0278149
:10762000211104C021E0278368E3A3CF089567E315
:10763000A0CF6AE49ECF69E49CCF66E39ACF65E36E
:1076400098CF6EE496CF64E394CF63E392CF62E386
:1076500090CF61E38ECF60E38CCF6FE28ACF6DE293
:1076600088CF6CE286CF242F462F6CE43ACF77FF89
:1076700003C071956195710920E0462F6EE231CF0C
:10768000462F20E067E42DCF462F20E066E429CF87
:10769000262F64E426CFCF92DF92FF920F931F93A1
:1076A000CF93DF938C01F62E443F81E0580738F0EA
:1076B000413187E2580728F040E157E202C044EF29
:1076C00051E0243F81E0380738F0E90121313742A9
:1076D00028F0C0E1D7E202C0C4EFD1E0CA01845F64
:1076E000914022E3C22ED12CB6010E9451B5462F03
:1076F0002F2D62E4C801F5DECE01845F9140B60112
:107700000E9451B5462F2F2D63E4C801DF91CF9120
:107710001F910F91FF90DF90CF90E3CE242F462F43
:1077200062E5DFCE242F462F61E5DBCE262F40E039
:107730006FE3D7CE262F40E06EE3D3CE262F40E076
:107740006DE3CFCE462F20E06FE4CBCE462F20E076
:107750006DE4C7CEFC016283611104C020E040E00B
:107760006BE4BFCE089577FF03C0719561957109F1
:1077700020E0462F6BE4B5CE4F925F926F927F92DE
:107780008F929F92AF92BF92CF92DF92EF92FF9231
:107790000F931F93CF93DF936C01A4ECCA1AADEF44
:1077A000DA0AD601ED91FC917E970CF05DC0FC01E8
:1077B000E858FF4F812C912CA191B191AB2B21F472
:1077C0002115310549F450C0BFEF8B1A9B0AAEE179
:1077D0008A16910489F748C0EC015401AA0CBB1C1D
:1077E000AA0CBB1CAC0EBD1EF501EC54FF4F408330
:1077F0005183628373837401EE0CFF1CEC0EFD1E3B
:10780000F701E858FF4F31832083EC54FF4F118379
:107810000083BE01680D791DFB01EC55FE4F81E030
:1078200080830E940049F501608371838283938382
:10783000C65CDD4F88819981F701E250FE4F91834C
:107840008083D6012D913C9111972F5F3F4F2D934F
:107850003C939C012F5F3F4F1216130614F021E05A
:1078600030E03983288302C08FEF9FEFDF91CF9103
:107870001F910F91FF90EF90DF90CF90BF90AF904E
:107880009F908F907F906F905F904F9008950F938F
:107890001F93CF93DF93EC017093950E6093940E3A
:1078A00040939B0E81E090E00E9492B68C010E9472
:1078B00009801093C00D0093BF0D91E090937B0E53
:1078C00090937C0E1092B50D1092B40D10927F0E15
:1078D00010927E0E1092800E10927D0E24EF31E0F9
:1078E0003093870E2093860E28EB3BE03093890E71
:1078F0002093880E20E233E030938E0E20938D0E7D
:107900002CEA3DE03093900E20938F0E28E037E074
:107910003093970E2093960E24E931E13093990E1F
:107920002093980E1092830E1092820E1092810E68
:1079300010928A0E1092910E10929A0E1092B30D20
:107940001092850E1092840E10928C0E10928B0E57
:107950001092930E1092920E988399839A83DF91DE
:10796000CF911F910F9108951F920F920FB60F9212
:1079700011240BB60F922F933F934F935F936F9306
:107980007F938F939F93AF93BF93EF93FF938091D8
:10799000BC0D8F5F8093BC0D9091BB0D891708F4CF
:1079A000FAC01092BC0D8091BA0D90E0873091051D
:1079B00008F0F1C0FC018827E25AFE4F8F4F0C946B
:1079C00078B560E086E1F2D780E48093BB0D81E07A
:1079D00043C061E086E1EAD788E08093BB0D33C005
:1079E00060E086E1E3D78091B80D9091B90D97FFE3
:1079F00005C088E18093BB0D84E02EC088E08093B1
:107A0000BB0D83E029C061E086E1D0D788E1809397
:107A1000BB0D8091B70D8F5F8093B70D803148F01B
:107A20001092B70D85E018C061E086E1BFD788E00D
:107A3000EECF8091B80D9091B90D880F991F90935A
:107A4000B90D8093B80D82E007C060E086E1AED743
:107A500088E08093BB0D86E08093BA0D9CC061E006
:107A600086E1A4D780EC8093BB0D8091BD0D9091F1
:107A7000BE0D9093B90D8093B80D8091BD0D90917E
:107A8000BE0D91FF1DC08091B60D8823B1F080918D
:107A9000BD0D9091BE0D22E092279093BE0D809374
:107AA000BD0D8091BD0D9091BE0D80649093BE0D73
:107AB0008093BD0D1092B60D03C081E08093B60D8A
:107AC0008091BD0D9091BE0D92FF0EC08091B60DBC
:107AD000882339F01092BE0D1092BD0D1092B60D94
:107AE00003C081E08093B60D8091BD0D9091BE0DD5
:107AF00084FF14C08091B60D882369F08091BD0D7C
:107B00009091BE0D20E182279093BE0D8093BD0D14
:107B10001092B60D03C081E08093B60D8091BD0D2B
:107B20009091BE0D87FF13C08091B60D882361F040
:107B30008091BD0D9091BE0D80589093BE0D8093A5
:107B4000BD0D1092B60D03C081E08093B60D8091FB
:107B5000BD0D9091BE0D90FF14C08091B60D88238D
:107B600069F08091BD0D9091BE0D21E09227909318
:107B7000BE0D8093BD0D1092B60D03C081E08093C1
:107B8000B60D8091BD0D9091BE0D9093B90D80936F
:107B9000B80D1092BA0DFF91EF91BF91AF919F91E7
:107BA0008F917F916F915F914F913F912F910F90A6
:107BB0000BBE0F900FBE0F901F901895DC01A250C6
:107BC000BE4F20E030E04D915D914617570739F4E4
:107BD000280F391FF901EC55FE4F808108952F5F62
:107BE0003F4F2E31310579F780E00895CF93DF9331
:107BF000EC01C45CDD4FA881B981109709F442C043
:107C0000FC01E250FE4F20E030E0419151914617D7
:107C1000570799F5A901440F551F480F591FFA013D
:107C2000E858FF4F60817181672B61F111821082EA
:107C3000FC01E20FF31FEC55FE4F1082FA01EE53E8
:107C4000FE4F11821082235D3F4F220F331F220F00
:107C5000331FFC01E20FF31F108211821282138284
:107C6000FA01E859FE4F11821082EA56FF4F118245
:107C700010821197B983A88305C02F5F3F4F2E3123
:107C8000310519F6DF91CF9108950F931F9301E00D
:107C900010E072DD1F910F91089510927B0E2FE975
:107CA0003FE344EF51E060E070E08091940E9091EA
:107CB000950EEBDF9093B50D8093B40D08950F935F
:107CC0001F9300E010E058DD1F910F9108952F924F
:107CD0003F924F925F926F927F928F929F92AF925C
:107CE000BF92CF92DF92EF92FF920F931F93CF93A9
:107CF000DF9300D000D0CDB7DEB78C010E940049E1
:107D000098012E533E4F3C832B831E830D83D80155
:107D1000AC55BE4FBA83A9831801B2E02B1ABEEF4F
:107D20003B0AF901AA24A394B12C32E0832E912CB2
:107D3000118210829F012A543140D9012D913C912A
:107D4000232B09F44DC0AD81BE812D913D914D9104
:107D50005C9113977D01B4EBEB0EF11CD701CD9034
:107D6000DD90ED90FC902B013C01421A530A640A0D
:107D7000750A4C145D046E047F0490F1C20ED31E8C
:107D8000E41EF51EAD81BE81CD92DD92ED92FC9296
:107D90001397A981BA812C91222311F19F012659B1
:107DA0003109D9012D913C912115310519F4B18288
:107DB000A08216C07F01BAE5EB1AF108D7014D91F8
:107DC0005C911197421753075CF4B182A0824F5F18
:107DD0005F4F4D935C934217530714F0918280825A
:107DE00032962D813E812C5F3F4F3E832D83A981AA
:107DF000BA811196BA83A983E215F30509F098CFE9
:107E0000EB81FC8181919191FC83EB838130910521
:107E100099F00297C9F4EB81FC81EC54F140019098
:107E2000F081E02D1995AB81BC81DA966D917C9142
:107E3000DB97C801DBDE08C0EB81FC81EC54F1402C
:107E40000190F081E02D19952B813C81221533059D
:107E5000B9F626960FB6F894DEBF0FBECDBFDF9100
:107E6000CF911F910F91FF90EF90DF90CF90BF9037
:107E7000AF909F908F907F906F905F904F903F90CA
:107E80002F9008956E3E22E0720738F06B3C98E028
:107E9000790728F06AEC78E002C06EEE72E0660FB7
:107EA000771F9FB7F89425E1829FF0011124E550D8
:107EB000FE4E748363839FBF08956E3E22E0720777
:107EC00038F06B3C98E0790728F06AEC78E002C063
:107ED0006EEE72E0660F771F9FB7F89425E1829FE0
:107EE000F0011124E550FE4E768365839FBF08950F
:107EF000660F771F282F30E095E1899FF00111244C
:107F0000E550FE4E858196816817790718F46581E2
:107F1000768107C0838194818617970710F4638167
:107F200074818FB7F89495E1929FF001939FF00DC3
:107F30001124E550FE4E728361838FBF089581E066
:107F400080937B0E6CED75E0D3CF6CED75E080E037
:107F5000CFCF8091B7068093B60608958091E90D42
:107F6000882359F08091E70D9091E80DDC01ED91A7
:107F7000FC910480F581E02D199408958091E90D1C
:107F8000882369F08091E70D9091E80DDC01ED9177
:107F9000FC910190F081E02D6FEF73E0199408954A
:107FA0008091E90D882389F08091EB0D882321F0E1
:107FB00080E090E0D3DF03C080E090E0DFDF9091CD
:107FC000EB0D81E089278093EB0D08952091E90D59
:107FD000222369F0A091E70DB091E80DED91FC919D
:107FE00011970190F081E02DBC01CD011994089505
:107FF0008091E60D882359F08091E40D9091E50D74
:10800000DC01ED91FC910480F581E02D1994089537
:108010008091E60D882369F08091E40D9091E50D43
:10802000DC01ED91FC910190F081E02D6FEF73E0A8
:10803000199408958091E60D882389F08091EA0DC6
:10804000882321F080E090E0D3DF03C080E090E05F
:10805000DFDF9091EA0D81E089278093EA0D089592
:108060002091E60D222369F0A091E40DB091E50D79
:10807000ED91FC9111970190F081E02DBC01CD01B3
:10808000199408952091E30D222369F0A091E10D48
:10809000B091E20DED91FC9111970190F081E02DEE
:1080A000BC01CD01199408952091E00D222369F0BF
:1080B000A091DE0DB091DF0DED91FC911197019033
:1080C000F081E02DBC01CD01199408952091DD0DC2
:1080D000222369F0A091DB0DB091DC0DED91FC91B4
:1080E00011970190F081E02DBC01CD011994089504
:1080F0002091DA0D222369F0A091D80DB091D90D0D
:10810000ED91FC9111970190F081E02DBC01CD0122
:10811000199408952091D70D222369F0A091D50DCF
:10812000B091D60DED91FC9111970190F081E02D69
:10813000BC01CD01199408952091D40D222369F03A
:10814000A091D20DB091D30DED91FC9111970190BA
:10815000F081E02DBC01CD01199408952091D10D3D
:10816000222369F0A091CF0DB091D00DED91FC913B
:1081700011970190F081E02DBC01CD011994089573
:108180008091B0069091B106DC01ED91FC91E25A2C
:10819000FF4F0190F081E02D19948091B0069091ED
:1081A000B106DC01ED91FC91E45AFF4F0190F081A2
:1081B000E02D19948091B0069091B106DC01ED910B
:1081C000FC91E65AFF4F0190F081E02D19948091C7
:1081D000421081110DC080912B0690912C06DC017C
:1081E000ED91FC910190F081E02D60E070E0199438
:1081F00008958091421081110DC080912B069091BD
:108200002C06DC01ED91FC910190F081E02D6FEFE7
:1082100070E0199408950C94D85C0C94185D8091CA
:10822000B706882361F00E944A82029741F06BE210
:1082300071E18091B4069091B5060C94007C08958C
:108240008091B606882341F06DE470E18091B40618
:108250009091B5060C94007C08958091B606882311
:1082600041F06DE370E18091B4069091B5060C94F5
:10827000007C0895CF93DF932091EE0D3091EF0DA8
:1082800028173907D1F09093EF0D8093EE0D2091D0
:10829000B606222391F0EC016CEF70E18091B406F8
:1082A0009091B5060E948F7ABE018091B40690919C
:1082B000B506DF91CF910C94F271DF91CF910895C3
:1082C000CF93DF932091EC0D3091ED0D28173907F6
:1082D000D1F09093ED0D8093EC0D2091B606222302
:1082E00091F0EC0162EE70E18091B4069091B506D8
:1082F0000E948F7ABE018091B4069091B506DF91FD
:10830000CF910C94F271DF91CF9108952091E30DFC
:10831000222339F0BC018091CD0D9091CE0D0C94AB
:10832000E57108952091E00D222339F0BC01809180
:10833000CB0D9091CC0D0C94E57108952091DD0D3D
:10834000222339F0BC018091C90D9091CA0D0C9483
:10835000E57108952091DA0D222339F0BC01809156
:10836000C70D9091C80D0C94E57108952091D70D1B
:10837000222339F0BC018091C50D9091C60D0C945B
:10838000E57108952091D40D222339F0BC0180912C
:10839000C30D9091C40D0C94E57108952091D10DF9
:1083A000222339F0BC018091C10D9091C20D0C9433
:1083B000E5710895CF92DF92EF92FF922091000233
:1083C000213019F420914E1004C02230C9F52091BB
:1083D00054102223A9F19C01211584E0380710F0E4
:1083E0002FEF33E0ADE0B0E00E9429BB2FEF33E088
:1083F00040E050E00E94DBBA69017A018FEFC81AB1
:10840000D80AE80AF80A809153138C15C9F0C09273
:1084100053138091B606882399F06BE970E180913F
:10842000B4069091B5060E948F7A6C2D8091B406A7
:108430009091B506FF90EF90DF90CF900C949874D8
:10844000FF90EF90DF90CF900895CF92DF92EF9260
:10845000FF9220910002213019F420914B1004C0AA
:108460002230C9F5209151102223A9F19C01211538
:1084700084E0380710F02FEF33E0ADE0B0E00E9469
:1084800029BB2FEF33E040E050E00E94DBBA6901E6
:108490007A018FEFC81AD80AE80AF80A80915113B6
:1084A0008C15C9F0C09251138091B606882399F0BB
:1084B00064E870E18091B4069091B5060E948F7ACD
:1084C0006C2D8091B4069091B506FF90EF90DF90EF
:1084D000CF900C949874FF90EF90DF90CF90089518
:1084E00081E08093AD060E94265F8091B6068823C6
:1084F00041F06AE670E18091B4069091B5060C9463
:10850000007C089583E08093AD060E94505D8091C9
:10851000B606882341F067E770E18091B406909138
:10852000B5060C94007C089582E08093AD060E940D
:10853000505D8091B606882341F06DE570E1809131
:10854000B4069091B5060C94007C08950C94C294E6
:108550008091010281110C94A6940C94C2940C9405
:10856000A69484E60C94D09189E10C94D09182E396
:108570000C94D0918BE40C94D091809100028130C6
:1085800011F482E001C081E00C94739282E00C94BB
:10859000739281E00C9473920C94180E9091731066
:1085A00081E089270C946D5E80E00C946D5E81E023
:1085B0000C946D5E9091711081E089270C949F5E00
:1085C00080E00C949F5E81E00C949F5E4091A60F2A
:1085D0005091A70F6091A40F7091A50F8CE39BE0C1
:1085E0000E9468888091B606882341F062E270E1BB
:1085F0008091B4069091B5060C94007C089580910A
:108600004F06882339F08CE39BE00E94639528E1B4
:108610003DE506C08CE39BE00E94799528ED3CE5A2
:108620004CE251E060E070E084E69BE02EDB80915C
:10863000B606882341F06FE070E18091B406909116
:10864000B5060C94007C08958CE39BE00E94749521
:1086500081110C94D85C0C94185D682F8091B4063D
:108660009091B5060E94AD7469E271E18091B40603
:108670009091B5060C948F7AF0DF8091B4069091BA
:10868000B5060C94ED7BCF92DF92EF92FF929C01A6
:10869000A3E6B0E00E9429BB2FEF33E040E050E0BA
:1086A0000E94DBBA69017A018FEFC81AD80AE80A7A
:1086B000F80A809110068C15A1F0C09210068091E6
:1086C000B606882371F06BEC70E18091B40690914E
:1086D000B5060E948F7A8C2DFF90EF90DF90CF909F
:1086E000CBCFFF90EF90DF90CF900895CF92DF92A5
:1086F000EF92FF929C01A3E6B0E00E9429BB2FEF0E
:1087000033E040E050E00E94DBBA69017A018FEF6C
:10871000C81AD80AE80AF80A809111068C15A1F047
:10872000C09211068091B606882371F062EB70E169
:108730008091B4069091B5060E948F7A8C2DFF909F
:10874000EF90DF90CF9098CFFF90EF90DF90CF9099
:1087500008952091B4063091B506882319F06EE88B
:1087600077E002C062E977E0C9010C948F7AF1DF0B
:108770008091B4069091B5060C94ED7B2091B406DF
:108780003091B506882319F06EE171E102C063E211
:1087900071E1C9010E948F7A8091B4069091B5066B
:1087A0000C94ED7B6CE171E18091B4069091B5067B
:1087B0000C948F7A68E171E18091B4069091B506CE
:1087C0000C948F7ACF93CDE266E171E18091B4068B
:1087D0009091B5060E948F7AC150B1F78091B4068E
:1087E0009091B5060E94ED7B8091B4069091B506FC
:1087F000DC01ED91FC910284F385E02DCF91199479
:1088000090E0FC013197E231F10508F04EC0882775
:10881000EB59FE4F8F4F0C9478B5809180008F7785
:1088200003C0809180008F7D8093800008958091A7
:108830008000877FF9CF84B58F7702C084B58F7DA4
:1088400084BD08958091B0008F7703C08091B000FF
:108850008F7D8093B0000895809190008F7707C03E
:10886000809190008F7D03C080919000877F8093DE
:10887000900008958091A0008F7707C08091A0009C
:108880008F7D03C08091A000877F8093A000089512
:10889000809120018F7707C0809120018F7D03C0D8
:1088A00080912001877F80932001089510922A06ED
:1088B0001092240610921B0610922506109226068E
:1088C000109227061092280681E08093E90A4091D1
:1088D00030065091310660E070E024E734E4809186
:1088E0001C0690911D06D1C98091F80981111CC008
:1088F0001092300A1092310A1092320A1092330A02
:108900001092340A1092350A1092380A8091E70AC0
:108910009091E80ADC01ED91FC910190F081E02D4D
:1089200019951092E90A089524E734E445E050E0EF
:1089300060E070E080911C0690911D06A6C96091D0
:10894000FC0D7091FD0D80911C0690911D0636D98D
:10895000882319F081E08093FB0D0895CF93DF9376
:10896000282F30E0F901E55EFD4E8491F901EB52CC
:10897000FE4ED491F901E157FE4EC491CC2389F00B
:1089800081113EDFEC2FF0E0EE0FFF1FEB58FE4EA3
:10899000A591B491EC91ED2381E090E021F480E089
:1089A00002C080E090E0DF91CF9108951F93CF93B4
:1089B000DF93282F30E0F901E55EFD4E8491F90147
:1089C000EB52FE4ED491F901E157FE4EC491CC23F7
:1089D000C1F0162F811114DFEC2FF0E0EE0FFF1F16
:1089E000E55AFE4EA591B4918FB7F894111105C0C8
:1089F0009C91ED2FE095E92302C0EC91ED2BEC93D7
:108A00008FBFDF91CF911F91089560E087E0CEDFA7
:108A10001092EA0A089561E087E0C8DF81E0809360
:108A2000EA0A0895CF93DF938091090E811110C057
:108A300084EF91E09093080E8093070E8BE290E014
:108A40009093060E8093050E81E08093090E20C05E
:108A50008091050E9091060E8532910514F00497D1
:108A600009C08331910514F0029704C0823091054A
:108A70002CF001979093060E8093050E8091050EC1
:108A80009091060E97FF04C01092060E1092050EEC
:108A9000C091040ECC2311F0B8DF01C0BCDF81E02F
:108AA0008C278093040EC091070ED091080E1C16DF
:108AB0001D0654F01092090EA8DF21E835E44AEFB4
:108AC00050E060E070E007C022E135E4AE010D2E19
:108AD000000C660B770B80911C0690911D06D5D873
:108AE0009093030E8093020E8091050E9091060ED6
:108AF000C81BD90BD093080EC093070EDF91CF91FE
:108B000008950F931F93CF93DF938091EB0A8823EF
:108B100029F0DF91CF911F910F9184CF0091020E28
:108B20001091030EC0911C06D0911D06B801CE0114
:108B300045D8882319F0B801CE0158D8DF91CF91DC
:108B40001F910F9162CFCF92DF92EF92FF9210921E
:108B5000EB0A209120063091210640912206509187
:108B60002306609125067091260680912706909134
:108B700028060E948CB56B017C0120E030E0A90141
:108B80000E9492B987FD09C0C0922506D0922606A0
:108B9000E0922706F092280608C01092250610924F
:108BA00026061092270610922806FF90EF90DF907D
:108BB000CF90A7CFEF92FF921F93CF93DF9300D078
:108BC000CDB7DEB784E689838CE38A8388E28B8322
:108BD0001091FE0D1330E0F4E12EF12C10FF02C0D5
:108BE00014DF01C018DFE1E0F0E0EC0FFD1FEE0D37
:108BF000FF1D408150E060E070E02AED35E4809197
:108C00001C0690911D0641D81F5F1093FE0D03C0F6
:108C1000FCDE1092FE0D0F900F900F90DF91CF9120
:108C20001F91FF90EF90089560E088E0BFCE61E073
:108C300089E2BCCE0F931F93CF93DF9360E08BE26A
:108C4000B5DE0091F00D1091F10DC0911C06D09190
:108C50001D06B801CE010E94DE3D882341F0B80117
:108C6000CE01DF91CF911F910F910C94F63DDF91D2
:108C7000CF911F910F910895CF93DF9390E0FC0166
:108C8000EB52FE4E2491FC01E157FE4E8491882365
:108C900061F190E0880F991FFC01EF5BFE4EC591DA
:108CA000D491FC01E55AFE4EA591B491611109C021
:108CB0009FB7F8948881209582238883EC912E2396
:108CC0000BC0623061F49FB7F8943881822F809591
:108CD00083238883EC912E2B2C939FBF06C08FB7E4
:108CE000F894E8812E2B28838FBFDF91CF910895D0
:108CF0001F93CF93DF93182FEB0161E0BDDF209727
:108D000011F460E004C0CF3FD10531F461E0812F60
:108D1000DF91CF911F914ACEE12FF0E0E55EFD4E4D
:108D2000E4914E2F50E0FA013197E231F10508F05D
:108D30009DC08827E958FE4F8F4F0C9478B584B5B5
:108D4000806884BDC7BD97C084B5806284BDC8BD3E
:108D500092C080918000806880938000D0938900C9
:108D6000C093880088C080918000806280938000DA
:108D7000D0938B00C0938A007EC080918000886071
:108D800080938000D0938D00C0938C0074C080913C
:108D9000B00080688093B000C093B3006CC0809135
:108DA000B00080628093B000C093B40064C0809132
:108DB0009000806880939000D0939900C0939800B1
:108DC0005AC080919000806280939000D0939B0065
:108DD000C0939A0050C0809190008860809390006A
:108DE000D0939D00C0939C0046C08091A0008068F5
:108DF0008093A0008091A0008F7B8093A000D093EF
:108E0000A900C093A80037C08091A0008062809321
:108E1000A000D093AB00C093AA002DC08091A00009
:108E200088608093A000D093AD00C093AC0023C0B5
:108E300080912001806880932001D0932901C09304
:108E4000280119C080912001806280932001D09375
:108E50002B01C0932A010FC080912001886080936C
:108E60002001D0932D01C0932C0105C0C038D1053D
:108E70000CF04CCF46CFDF91CF911F9108950F9307
:108E80001F93CF93DF938091010E90912A06811159
:108E90002AC0992309F456C00091FF0D1091000ECD
:108EA000C0911C06D0911D06B801CE010E94DE3D86
:108EB000882321F0B801CE010E94F63DACDD2FE3FE
:108EC00037E442EC51E060E070E080911C06909144
:108ED0001D060E945F3E9093000E8093FF0D81E07F
:108EE0008093010E59C08091EA0A992361F088238A
:108EF00029F0DF91CF911F910F9187CDDF91CF9115
:108F00001F910F9188CD8823C9F36091FF0D709157
:108F1000000E80911C0690911D060E94F63D2FE3E5
:108F200037E444E150E060E070E080911C069091ED
:108F30001D060E945F3E9093000E8093FF0D1092DD
:108F4000010E2AC0C0910A02D0910B022297D09341
:108F50000B02C0930A021C161D066CF4BE01772793
:108F600087E0C6DECC2321F081E08093EA0A14C0BA
:108F70001092EA0A11C06091FF0D7091000E80916D
:108F80001C0690911D060E94F63D3FDD8FEF90E09C
:108F900090930B0280930A02DF91CF911F910F9162
:108FA00008950F931F93CF93DF930091F70D1091C6
:108FB000F80DC091F90DD091FA0DC00FD11FD093CB
:108FC000FA0DC093F90DBE01772787E091DECC231F
:108FD00021F081E08093EA0A02C01092EA0A10169A
:108FE0001106ECF58091F50D9091F60DC817D90793
:108FF0000CF485C08091FB0D882371F01092F60D62
:109000001092F50D8CEF9FEF9093F80D8093F70D74
:1090100081E08093F40D73C068E770E080E090E039
:109020000E94647ADC01CB010A96A11DB11D9093C8
:10903000F60D8093F50D68E270E080E090E00E940C
:10904000647ADC01CB010A96A11DB11D6627772742
:10905000681B790B7093F80D6093F70D50C0012BCE
:1090600009F44DC08091F50D9091F60D8C179D0778
:109070000CF445C08091F40D882311F10091FC0D92
:109080001091FD0DC0911C06D0911D06B801CE01B6
:109090000E94DE3D882399F1B801CE010E94F63D81
:1090A000B4DC1092FA0D1092F90D1092F40D80912B
:1090B0002A06882321F1DF91CF911F910F91DFCEF6
:1090C00069E670E080E090E00E94647ADC01CB0108
:1090D0008A569F4FAF4FBF4F9093F60D8093F50D7B
:1090E00068E270E080E090E00E94647ADC01CB01ED
:1090F0000A96A11DB11D9093F80D8093F70DDF9195
:10910000CF911F910F910895863308F08653909167
:109110007B00282F2870977F922B90937B0087707D
:10912000806480937C0080917A00806480937A00D0
:1091300080917A0086FDFCCF8091780020917900A3
:1091400090E0922B08953FB7F89480910F0E909184
:10915000100EA091110EB091120E26B5A89B05C05D
:109160002F3F19F00196A11DB11D3FBFBA2FA92FA6
:10917000982F8827820F911DA11DB11DBC01CD0123
:1091800042E0660F771F881F991F4A95D1F708950F
:109190008F929F92AF92BF92CF92DF92EF92FF9207
:1091A0006B017C01D0DF4B015C01C114D104E104EF
:1091B000F104E9F0C8DFDC01CB0188199909AA099B
:1091C000BB09883E9340A105B10578F321E0C21A9E
:1091D000D108E108F10888EE880E83E0981EA11CF2
:1091E000B11CC114D104E104F10421F7DECFFF90DA
:1091F000EF90DF90CF90BF90AF909F908F900895A9
:109200002FB7F89460910B0E70910C0E80910D0E9B
:1092100090910E0E2FBF08951F920F920FB60F92CE
:1092200011242F933F938F939F93AF93BF9380917C
:109230000B0E90910C0EA0910D0EB0910E0E309170
:109240000A0E23E0230F2D3720F40196A11DB11D36
:1092500005C026E8230F0296A11DB11D20930A0E1A
:1092600080930B0E90930C0EA0930D0EB0930E0EE8
:1092700080910F0E9091100EA091110EB091120ED0
:109280000196A11DB11D80930F0E9093100EA09317
:10929000110EB093120EBF91AF919F918F913F919C
:1092A0002F910F900FBE0F901F9018950F931F9343
:1092B000CF93DF930091020E1091030EC0911C0614
:1092C000D0911D06B801CE010E94DE3D8823A1F099
:1092D000B801CE010E94F63D2FE934E448EB5BE093
:1092E00060E070E080911C0690911D060E94453E52
:1092F0009093030E8093020E6091FC0D7091FD0D12
:1093000080911C0690911D060E94DE3D81114BC08C
:109310001092FB0D8FEF90E09093FA0D8093F90D72
:109320007ADB68E770E080E090E00E94647ADC011C
:10933000CB010A96A11DB11D9093F60D8093F50DFA
:1093400068E270E080E090E00E94647ADC01CB018A
:109350000A96A11DB11D66277727681B790B7093AC
:10936000F80D6093F70D21ED37E444E150E060E043
:1093700070E080911C0690911D060E945F3E9093C4
:10938000FD0D8093FC0D2FE934E448EB5BE060E0D9
:1093900070E080911C0690911D060E94453E9093BE
:1093A000030E8093020EDF91CF911F910F910895CC
:1093B0008F929F92AF92BF92CF92EF92FF920F93B4
:1093C0001F93CF93DF9320913B06223008F07AC0A1
:1093D0007B018C018090250690902606A0902706A0
:1093E000B090280620E030E0A901C501B4010E9438
:1093F00092B9181654F520E030E0A901C501B40176
:109400000E948AB6181654F420E030E048E452E492
:10941000C501B4010E9492B91816D4F420E030E0DE
:1094200048E452E4C501B4010E948AB618169CF4BF
:1094300020E030E048EC52E4C501B4010E9492B94A
:1094400087FF09C0CBE4D0E008C0C0E0D0E005C091
:10945000C2E3D0E002C0C4E6D0E08FEF8C0D8230D2
:1094600070F4209739F06C2FC8010E949B576C2F25
:10947000C7010DC0C8010E94E66CC70116C08DEF80
:109480008C0D8330F8F4209779F06C2FC801DF91B0
:10949000CF911F910F91FF90EF90CF90BF90AF9021
:1094A0009F908F900C949B57C801DF91CF911F9193
:1094B0000F91FF90EF90CF90BF90AF909F908F90C3
:1094C0000C94E66CDF91CF911F910F91FF90EF907C
:1094D000CF90BF90AF909F908F9008958F929F9262
:1094E000AF92BF92CF92DF92EF92FF92C09025068B
:1094F000D0902606E0902706F090280620E030E085
:10950000A901C701B6010E948AB620E030E040E020
:109510005FE387FD0BC0C701B6010E948DB54B010B
:109520005C010E9459B697FD27C010C0C701B60163
:109530000E948CB50E9459B697FD1EC06536710514
:1095400081059105DCF424E6822F14C0C501B40125
:109550000E9459B665367105810591057CF420E0BD
:1095600030E040E05FE3C701B6010E948DB50E9484
:1095700059B684E6861B03C084E601C080E0FF90F4
:10958000EF90DF90CF90BF90AF909F908F90089515
:109590000F931F93CF93DF9300911506109116063A
:1095A000C0911C06D0911D06B801CE010E94DE3D7F
:1095B000882321F0B801CE010E94F63D8091EB0A8C
:1095C000882339F01092EB0ADF91CF911F910F9110
:1095D00098CADF91CF911F910F91089560E089E2C1
:1095E000E5D927E136E442E350E060E070E08091A5
:1095F0001C0690911D060C94453E1F920F920FB6CB
:109600000F9211240BB60F922F933F934F935F93BA
:109610006F937F938F939F93AF93BF93EF93FF933A
:109620008091F30D8823B1F0669918C0EE982AE175
:1096300036E44CE251E060E070E080911C069091CD
:109640001D060E94453E8091F20D882339F00E944C
:109650003A6204C0669B02C0EE98ECDAFF91EF918B
:10966000BF91AF919F918F917F916F915F914F913A
:109670003F912F910F900BBE0F900FBE0F901F9038
:1096800018950C94F85C0C94345D0C94898A0C94B5
:10969000C48A80911F0E882319F00E94898A02C013
:1096A0000E94C48A90911F0E81E0892780931F0E2B
:1096B00008954091A60F5091A70F6091A40F70914B
:1096C000A50F85E19BE00E9468888091B6068823FB
:1096D00041F064EF73E18091B4069091B5060C946B
:1096E000007C08950E94898A4091C7105091C8104B
:1096F00060E070E024EC3AE884E69BE00E94453E9E
:1097000090939213809391138091B606882341F031
:1097100064E973E18091B4069091B5060C94007CE5
:1097200008950E94C48A4091C7105091C81060E00B
:1097300070E029E83AE884E69BE00E94453E909379
:109740009213809391138091B606882341F061E8CB
:1097500073E18091B4069091B5060C94007C089555
:1097600080914906882339F085E19BE00E9463954A
:1097700024E33DE506C085E19BE00E94799528EF52
:109780003CE54CE251E060E070E084E69BE00E9442
:10979000453E8091B606882341F061EE73E18091E9
:1097A000B4069091B5060C94007C089585E19BE089
:1097B0000E94749581110C94F85C0C94345D0C94A7
:1097C00006940C9412940F931F93CF93DF93009100
:1097D0001A0E10911B0EC0911C06D0911D06B801E7
:1097E000CE010E94DE3D882379F0B801CE010E94AF
:1097F000F63D80911E0690911F06DC01ED91FC91D3
:1098000000A0F1A1E02D19950091180E1091190EEC
:10981000C0911C06D0911D06B801CE010E94DE3D0C
:10982000882321F0B801CE010E94F63D7298809104
:10983000B606882361F069E773E18091B4069091E0
:10984000B506DF91CF911F910F910C94007CDF91B1
:10985000CF911F910F910895CF93DF938091901333
:10986000882319F11092901360E088E09FD8C0918E
:109870009113D0919213BE0184E69BE00E94DE3DDD
:10988000882329F0BE0184E69BE00E94F63D80918A
:10989000B606882371F068EC73E18091B40690916C
:1098A000B506DF91CF910C94007CDF91CF910C94A1
:1098B0009D95DF91CF91089580919013811102C001
:1098C0000C949D950895CF93DF93809193138823F3
:1098D00011F10E94898A10929313C0919113D09133
:1098E0009213BE0184E69BE00E94DE3D882329F0AE
:1098F000BE0184E69BE00E94F63D8091B606882377
:1099000071F06FEA73E18091B4069091B506DF9132
:10991000CF910C94007CDF91CF910C94D98ADF9188
:10992000CF9108950C94D98A8091200E882319F044
:109930000E94898A02C00E94008C9091200E81E0D2
:1099400089278093200E08950C94008C0C94138C1E
:109950000C942A8C80911E0E882319F00E94138C7F
:1099600002C00E942A8C90911E0E81E0892780936C
:109970001E0E08950C94548C0E94548C8091B00655
:109980009091B106DC01ED91FC9104A0F5A1E02DD0
:1099900019940C94918C80911D0E882319F00E94CB
:1099A000548C02C00E94918C90911D0E81E08927F9
:1099B00080931D0E08950C94AD8C0C94835D809162
:1099C0001C0E882319F00E94AD8C02C00E94835D9A
:1099D00090911C0E81E0892780931C0E08950C94B1
:1099E00084938091F20D81110C946E930C94849366
:1099F0000C946E930E94158B8091B0069091B106E5
:109A0000DC01ED91FC9102A0F3A1E02D1994CF931C
:109A1000DF93C0911C06D0911D0660911A0E7091C3
:109A20001B0ECE010E94DE3D811129C04091170E10
:109A300050E060E070E028E231E6CE010E945F3E37
:109A400090931B0E80931A0E80911E0690911F0614
:109A5000DC01ED91FC91068CF78DE02D199580913C
:109A60003906882361F06091180E7091190E80916B
:109A70001C0690911D060E94DE3D882371F08091A6
:109A8000B6068823E9F060E773E18091B40690910F
:109A9000B506DF91CF910C94007C0E94466126E4CC
:109AA00031E644E650E060E070E080911C06909161
:109AB0001D060E945F3E9093190E8093180EDFCF13
:109AC000DF91CF9108958ADD8091B606882341F019
:109AD00065E473E18091B4069091B5060C94007C26
:109AE0000895E091150EF091160E82810E94BA7EC3
:109AF0008091B606882341F067E273E18091B40655
:109B00009091B5060C94007C08958091F30D882304
:109B100019F00E94CF6102C00E94B9618091B6061F
:109B2000882379F0209134108091B4069091B50685
:109B3000222319F06BEE72E102C064E073E10C9431
:109B4000007C08950C94265FCF938091ED0A8823C2
:109B500009F46FC00E94E5619091EB0A882339F007
:109B6000911167C080914006882339F162C091113C
:109B700060C08091B606882341F06CEC72E1809160
:109B8000B4069091B5060E94007C0E94886281E034
:109B90008093290680910702813009F04AC08091A4
:109BA0006E10882309F445C0809134108823F1F0A9
:109BB0008091F20D81112FC019C082E08093400680
:109BC0008091B606882341F068ED72E18091B40679
:109BD0009091B5060E94007CC1E0C0933F060E94B0
:109BE000265F0E948862C093290623C040913610E8
:109BF00050913710141615065CF4052E000C660BF8
:109C0000770B21E931E984E69BE0CF910C94453E46
:109C1000CF910C9491912CE931E942E350E060E05E
:109C200070E084E69BE00E945F3E9093140E809368
:109C3000130ECF9108950C94505D8091AC06811164
:109C40000C94265F0C94505D0C94CA5F0C94C56014
:109C50000E94BA878091140681110C94CA5F0C94FB
:109C6000C560CF93DF93D82FC62F8091B006909117
:109C7000B106DC01ED91FC91EC5BFF4F0190F081AE
:109C8000E02D462F6D2F19958091B606882399F106
:109C900062E972E18091B4069091B5060E948F7AD4
:109CA000DD2329F0D13059F46DE872E102C068E893
:109CB00072E18091B4069091B5060E948F7AC73008
:109CC00069F028F4C130B9F46EE972E10CC0C83013
:109CD00041F0C93081F468EA72E105C062EC72E1DA
:109CE00002C064EB72E18091B4069091B506DF91F9
:109CF000CF910C94007CDF91CF91089569E081E0D1
:109D0000B0CF68E081E0ADCF67E081E0AACF61E04D
:109D100081E0A7CF69E080E0A4CF68E080E0A1CF38
:109D200067E080E09ECF61E080E09BCF6CE772E16E
:109D30008091B4069091B5060C948F7ACF93C82F7A
:109D40008091B0069091B106DC01ED91FC91EE5B43
:109D5000FF4F0190F081E02D6C2F19958091B60690
:109D6000882389F0E3DF6C2F8091B4069091B506CB
:109D70000E94AD7464E772E18091B4069091B506DB
:109D8000CF910C94007CCF9108958CE0D7CF8BE0DD
:109D9000D5CF8AE0D3CF89E0D1CF88E0CFCF87E09D
:109DA000CDCF86E0CBCF85E0C9CF84E0C7CF83E0BD
:109DB000C5CF82E0C3CF81E0C1CFCF93C82F8091C0
:109DC000B0069091B106DC01ED91FC91E05CFF4F93
:109DD0000190F081E02D6C2F19958091B6068823B3
:109DE00089F0A4DF6C2F8091B4069091B5060E9493
:109DF000AD7461E672E18091B4069091B506CF91A1
:109E00000C94007CCF9108958CE0D7CF8BE0D5CF18
:109E10008AE0D3CF89E0D1CF88E0CFCF87E0CDCF24
:109E200086E0CBCF85E0C9CF84E0C7CF83E0C5CF44
:109E300082E0C3CF81E0C1CFCF93C82F8091B0061D
:109E40009091B106DC01ED91FC9106ACF7ADE02DEF
:109E50006C2F19958091B606882349F067DF6C2F27
:109E60008091B4069091B506CF910C949874CF91DF
:109E700008958CE0E1CF8BE0DFCF8AE0DDCF89E091
:109E8000DBCF88E0D9CF87E0D7CF86E0D5CF85E09C
:109E9000D3CF84E0D1CF83E0CFCF82E0CDCF81E0BC
:109EA000CBCF9C010197849710F4822F0895C901AC
:109EB000845691098438934040F4C90164E670E007
:109EC0000E9451B5822F94E61BC0283E43E0340720
:109ED000D8F0C90168EE73E00E9451B548E15CEF2B
:109EE000649FC001659F900D749F900D1124280FF1
:109EF000391FC9016AE070E00E9465B5822F9AE0BF
:109F0000699F80191124089580E0089581E080936D
:109F1000F80A089581E08093F90A089581E080931A
:109F2000FA0A0895CF9380916A0EC0910C028111B4
:109F300001C1C23009F450C0C33009F49DC0C13022
:109F400009F028C18091FA0A811124C181E090E0D2
:109F50000E9492B69093C9128093C81262E083E087
:109F60000E943C461092690E1092C2121092C112C9
:109F70001092C61280E090E0FC01EE0FFF1FE95A3C
:109F8000F14F11821082019688309105A9F7109245
:109F9000680E1092670E80916A008C6080936A0050
:109FA000ED9A8FB7F894209184003091850030931A
:109FB000560E2093550E8FBF2EE83FE44AEF50E037
:109FC00060E070E08091BD129091BE120E94453E0B
:109FD00081E080936A0EDEC08091F90A8111DAC0B7
:109FE00081E090E00E9492B69093CB128093CA12C7
:109FF000809104018E7F809304018091050181602E
:10A000008093050187E197E09093F5128093F41215
:10A010002EE240EA56E861E070E00E947A7D80918D
:10A0200065008B7F809365001092350189E08093F5
:10A0300034018EE2809332018CEF8093300180E90D
:10A04000809331011092F3121092F2121092F112D9
:10A050001092F0121092EE12EEECF2E18CED95E01F
:10A060008193919322E1EE3EF207D1F7C1E0C093D4
:10A07000EF122AE83FE451C08091F80A81118AC0AA
:10A0800081E090E00E9492B69093CD128093CC1222
:10A09000809104018E7F809304018091050181608D
:10A0A0008093050187E197E090932B0E80932A0E11
:10A0B00026E040E052EC61E070E00E947A7D809101
:10A0C00065008B7F809365001092350180E180935D
:10A0D000340186E0809332018EEF8093300180E975
:10A0E000809331011092C4121092C3121092290E63
:10A0F0001092280E1092C512ECE2FEE08CED95E075
:10A10000819391932EE0E834F207D1F71092270E55
:10A11000C1E0C093260E26E83FE44AEF50E060E03D
:10A1200070E08091BD129091BE120E94453EC09396
:10A130006A0E30C0C23069F0C330D1F0C13051F581
:10A140008091FA0A811126C08091C1129091C212A9
:10A150001DC08091F90A81111DC08091CA12909191
:10A16000CB120E9401818091F2129091F3120EC0E5
:10A170008091F80A81110EC08091CC129091CD127D
:10A180000E949A838091C3129091C412029711F495
:10A19000C093010B80910C028230A1F1833009F44D
:10A1A00054C0813009F074C08091FA0A882309F400
:10A1B0006FC0ED98E59A1092690E1092C712109236
:10A1C000C2121092C1121092C61280E090E0FC01FF
:10A1D000EE0FFF1FE95AF14F11821082019688306D
:10A1E0009105A9F71092680E1092670E8091C8121F
:10A1F0009091C9120E9427B710926A0E1092F90A24
:10A2000082E044C08091F90A882309F441C080911A
:10A21000F4129091F5120E94587D809131018F7750
:10A2200080933101809131018F7E809331011092B2
:10A2300030018091CA129091CB120E9427B71092E0
:10A240006A0E1092F80A83E021C08091F80A8823F0
:10A25000F9F080912A0E90912B0E0E94587D8091EA
:10A2600031018F7780933101809131018F7E80930E
:10A270003101109230018091CC129091CD120E9448
:10A2800027B710926A0E1092FA0A81E080930C02AE
:10A290008091BD129091BE12CF910C94673EAF9207
:10A2A000BF92CF92DF92EF92FF920F931F93CF93C3
:10A2B000DF937C016B015A01D0E0C0E08D2F90E06C
:10A2C000F701A181B2818A159B05D0F4F601E80F50
:10A2D000F91F60810CE510E921E03327C6270C0F38
:10A2E000111D211D311D2BBFF801C791ED91FC916E
:10A2F00011970190F081E02DCD011995DF5FDECF40
:10A30000ED91FC9111970190F081E02D6C2FCD0122
:10A31000DF91CF911F910F91FF90EF90DF90CF9041
:10A32000BF90AF901994CF93DF9300D01F921F92EC
:10A33000CDB7DEB7FE01319625E0DF011D922A95EB
:10A34000E9F724E8298325E52C832AE22D836A8313
:10A350004B8345E050E0BF01A2DF65E070E080E0A4
:10A3600090E00E94C84880E00F900F900F900F90EF
:10A370000F90DF91CF910895EF92FF921F93CF93AB
:10A38000DF931F92CDB7DEB77C01162FFC016181F0
:10A3900072810E94267565E070E080E090E00E9486
:10A3A000C84842E462E4C701BEDF412F60E0C70154
:10A3B000BADF811163C040E061E0C701B4DF811101
:10A3C0005DC040E062E0C701AEDF811157C046E0EA
:10A3D00062E0C701A8DF811151C040E063E0C7011E
:10A3E000A2DF81114BC040E064E0C7019CDF11E0B7
:10A3F000811110E040E065E0C70195DF811101C0E7
:10A400001F5F40E066E0C7018EDF811101C01F5F62
:10A4100040E067E0C70187DF811101C01F5F40E0B6
:10A4200068E0C70180DF811101C01F5F40E069E083
:10A43000C70179DF811101C01F5F44E06AE0C701F5
:10A4400072DF811101C01F5F44E06AE0C7016BDF6A
:10A45000811101C01F5F62E370E080E090E00E9424
:10A46000C84882E8898341E050E0BE016F5F7F4FBA
:10A47000C70115DF81E0183011F0111180E00F9055
:10A48000DF91CF911F91FF90EF900895CF93DF93CD
:10A4900000D01F92CDB7DEB72AEA2983FC012081C4
:10A4A0002A836B834C8344E050E0BE016F5F7F4F93
:10A4B000F6DE0F900F900F900F90DF91CF910895DF
:10A4C0003FB7F89420E0822F90E0841795079CF422
:10A4D000FC01EE0FFF1FE75AF14FA081B181880FF9
:10A4E000991FFB01E80FF91FCD0196958795918380
:10A4F00080832F5FE8CF3FBF1092C61208952F923E
:10A500003F925F926F927F928F929F92AF92CF9283
:10A51000DF92EF92FF920F931F93CF93DF931F92DF
:10A520001F92CDB7DEB76DB67EB60E94FE810E9447
:10A53000F4810E944A82029709F025C20E94358266
:10A54000882309F41AC2C090BF12D090C012E090C4
:10A55000BD12F090BE12B601C7010E94DE3D8823F5
:10A56000F1F0F701E250FE4F00E010E0819191918F
:10A570008C159D0571F40E940049000F111F000FFA
:10A58000111FF701E00FF11F6083718382839383B2
:10A5900008C00F5F1F4F0E31110541F702C00E9426
:10A5A0001E831092FB0AEDB6FEB64091FE0A509152
:10A5B000FF0ACA01880F991F2DB73EB7281B390B18
:10A5C0000FB6F8943EBF0FBE2DBF0DB71EB70F5F7D
:10A5D0001F4F8091010B823061F0833021F1813077
:10A5E00009F070C0B8018091C8129091C91268DF5B
:10A5F00033C03FB7F89420E0822F90E0841795078E
:10A6000074F4880F991FF801E80FF91FDC01A253B9
:10A61000BD4E8D919C91918380832F5FEDCF3FBF85
:10A620001092EE1219C03FB7F89420E0822F90E00C
:10A630008417950774F4880F991FF801E80FF91F24
:10A64000DC01A45DB14F8D919C91918380832F5F3C
:10A65000EDCF3FBF1092C51220E06AE071E0822F7B
:10A6600090E04091FE0A5091FF0A8417950754F537
:10A67000689FF001699FF00D1124E652FF4EA085FE
:10A68000B1858C918823E1F0A081B1813C91C80112
:10A69000830F911D830F911DDC0112978D919C9169
:10A6A000A281B3814D915C9111970480F581E02DD9
:10A6B0004817590711F4108203C070838D939C933F
:10A6C0002F5FCDCF0FB6F894FEBE0FBEEDBE8091CA
:10A6D000D411882321F083ED91E10E94668280915C
:10A6E000DE11882321F08DED91E10E946682809138
:10A6F000E811882321F087EE91E10E946682809123
:10A70000F211882321F081EF91E10E94668280910D
:10A71000FC0A882309F465C08091E811811105C005
:10A720008091F211882309F450C08091EB1190912F
:10A73000EC11E091EF11F091F01123813481281791
:10A74000390724F48085811109C00EC0218132812E
:10A750008217930734F48085811106C088E090E069
:10A7600005C080E190E002C080E290E02091F51108
:10A770003091F611E091F911F091FA114381548171
:10A780004217530724F42085222349F00AC041814F
:10A790005281241735073CF42085222311F0816073
:10A7A00003C0846001C082602091CE113091CF112E
:10A7B0002817390719F41092D01107C09093CF11C0
:10A7C0008093CE1181E08093D0118091CE11909131
:10A7D000CF11429709F4DBC081E08093F41180939C
:10A7E000EA11EBE7F1E18EE791E19A83898398EE34
:10A7F000892E93E0992E55245394CF010197DC01C3
:10A800008C91882309F4ACC0E480F580D7011796B9
:10A810008C911797882309F4A3C08081882309F4B9
:10A820009FC04181528118966C918401041B150BC5
:10A83000101611061CF08A01085E134020E030E07B
:10A8400022242394312C8FE097E2A12CC62ED12C08
:10A850002C143D04ACF56430A9F040F4623071F082
:10A86000633019F5C90180539A4F13C0653071F0F8
:10A870006630D9F4C9018E549A4F0BC0C9018A526F
:10A880009A4F07C0C90188539A4F03C0C901825427
:10A890009A4FDC0112968D919C911397841B950B16
:10A8A00097FF03C09195819591098017910714F442
:10A8B000A22C8C01BFEF2B1A3B0A2E5F3F4FC8CF53
:10A8C00081E08A0DD70119969C919923F1F16430AA
:10A8D00099F028F4623041F0633049F036C06530B9
:10A8E000A1F06630D9F031C0813021F52DC0813022
:10A8F00049F1833051F51EC0813011F1823011F1E0
:10A90000833011F1843009F515C08130B9F08230FF
:10A91000B9F08430C9F08530C1F40CC0813061F0E9
:10A92000823061F0833061F0843061F0853061F015
:10A93000863059F481E009C086E007C085E005C093
:10A9400084E003C083E001C082E0A981BA819C91C8
:10A95000981302C0108204C05082A981BA818C93DE
:10A96000379629813A81295F3F4F3A83298331E124
:10A97000EF3CF30709F041CF04C00E940A820E9415
:10A980001E8381E066C00E940A8280E062C0E0907F
:10A99000D111F090D2111E141F040CF055C08091FB
:10A9A000E9110091BD121091BE1260916D0E70916F
:10A9B0006E0E8823B1F081E08093EA11C8010E94F5
:10A9C000DE3D811115C0A701FF0C660B770B20E956
:10A9D0003EE7C8010E94453E90936E0E80936D0E37
:10A9E00007C0C8010E94DE3D811102C01092EA1129
:10A9F0008091F3110091BD121091BE1260916B0E07
:10AA000070916C0E8823D1F081E08093F411C8011D
:10AA10000E94DE3D8111E5CE4091D1115091D211BD
:10AA2000052E000C660B770B2DE83EE7C8010E944F
:10AA3000453E90936C0E80936B0ED3CEC8010E945E
:10AA4000DE3D8111CECE02C01092EA111092F411B7
:10AA5000C8CE0FB6F8947EBE0FBE6DBE0F900F909D
:10AA6000DF91CF911F910F91FF90EF90DF90CF90EA
:10AA7000AF909F908F907F906F905F903F902F90BE
:10AA800008951F920F920FB60F9211240BB60F92DA
:10AA90002F933F934F938F939F93EF93FF938091C7
:10AAA0008400909185002091550E3091560E821BA6
:10AAB000930B20918400309185003093560E2093A3
:10AAC000550E803727E1920770F19093580E8093CE
:10AAD000570E8091C1129091C212029751F4909139
:10AAE000690E8091C71298133CC081E08093C61212
:10AAF0003EC08091C1129091C212892B49F481E02D
:10AB000090E09093C2128093C1121092540E2FC005
:10AB10008091C1129091C212019761F58091690EE6
:10AB20008430D8F527C02091690E283008F047C03E
:10AB30009C012C5D3540293B3B4068F4E091690E57
:10AB4000EF5FE093690EF0E0EE0FFF1FE95AF14F5F
:10AB50009183808334C08091C1129091C212029778
:10AB600071F583E090E09093C2128093C11210922D
:10AB7000690E25C08091C1129091C2120397B9F756
:10AB80009091690E8091C7129813F1CF8091C712EE
:10AB9000843068F382E090E0E6CF8091540E8F5FBE
:10ABA0008093540E863018F382E090E09093C212A6
:10ABB0008093C1128091690E8093C712D8CFFF9104
:10ABC000EF919F918F914F913F912F910F900BBEDD
:10ABD0000F900FBE0F901F9018950F931F938091A9
:10ABE0004C0E81110DC00E9400496093480E709375
:10ABF000490E80934A0E90934B0E81E080934C0E49
:10AC00000E9400490091480E1091490E20914A0E71
:10AC100030914B0EDC01CB01801B910BA20BB30BCF
:10AC2000893E9340A105B105A8F08AE30E94AE4495
:10AC3000892B11F060E001C061E08AE30E94D644F4
:10AC40000E9400496093480E7093490E80934A0E0B
:10AC500090934B0E1F910F9108950F931F930E9495
:10AC600000490091220E1091230E2091240E309164
:10AC7000250EDC01CB01801B910BA20BB30B85339E
:10AC80009142A105B10518F081E08093210E1F913A
:10AC90000F91A3CFFC0180E090E06150710977FD36
:10ACA00018C02191022E000C330B322F222782274D
:10ACB000932728E0AC01440F551F97FF06C0CA0137
:10ACC00031E2832730E1932701C0CA01215091F777
:10ACD000E4CF08950895089508950895CF93DF93DC
:10ACE000EC018091700E811109C06A8D7B8DCE01BF
:10ACF00049960E94267581E08093700E21E83FEF0F
:10AD00003B872A878FE790E09D878C871F861E866A
:10AD1000398B288B9B8B8A8B1D8A1C8ADF91CF9164
:10AD200008950F931F93CF93DF93EC011F8A1E8A20
:10AD30008C01075E1F4F40E060E0C8010E94C480A4
:10AD400040E064E0C8010E94C4800E9400496C8F0A
:10AD50007D8F8E8F9F8FDF91CF911F910F910895DF
:10AD60000F931F93CF93DF93EC0180916F0E8111AE
:10AD700012C00A8D1B8D6AEA70E0C8010E94DE7164
:10AD8000D801ED91FC910284F385E02DC80119955D
:10AD900081E080936F0E4AE06EE0CE0149960E94FA
:10ADA000C48021E83FEF3B872A878FE790E09D87AB
:10ADB0008C871F861E86398B288B9B8B8A8B1D8ADE
:10ADC0001C8ADF91CF911F910F9108950F931F93CC
:10ADD000CF93DF93EC011F8A1E8A8C01075E1F4F01
:10ADE00040E060E0C8010E94878040E064E0C80164
:10ADF0000E9487800E9400496C8F7D8F8E8F9F8F6D
:10AE0000DF91CF911F910F9108950F931F93CF93CF
:10AE1000DF93EC01E8A1F9A180819181A281B38146
:10AE20008E01075E1F4F81159649A105B10509F4F2
:10AE300052C040E056E960E070E084EB97E00E9489
:10AE4000F46C64E170E080E090E00E94C848E8A102
:10AE5000F9A180819181A281B38181152BE49207B0
:10AE6000A105B105E9F068F4803629E09207A10553
:10AE7000B105A1F080389542A105B105C1F442E0C9
:10AE800012C0811521EE9207A105B10559F0811577
:10AE9000924CA140B10559F445E005C041E003C022
:10AEA00043E001C046E06FE0C8010E94878084EB68
:10AEB00097E00E94FA78E8A1F9A14081518162816E
:10AEC000738184EB97E00E94F46C64E170E080E0B1
:10AED00090E00E94C8484AE06EE0C8010E94878066
:10AEE00041E067E1C8010E9487804AA168E1C8018A
:10AEF0000E9487804BA18FEF840F8E3108F04CE0C9
:10AF000066E1C8010E94878021E83FEF3B872A87DE
:10AF10008FE790E09D878C871F861E86398B288B54
:10AF20009B8B8A8B1D8A1C8ADF91CF911F910F9179
:10AF300008950C94E571EF92FF920F931F93CF93B6
:10AF4000DF93EC016623E1F0262F653608F024E656
:10AF50000A891B89E888F988D801AE19BF0930E051
:10AF60000E9486B528EC30E040E050E00E9407BB2C
:10AF7000E20EF31EFB86EA86021B130B1D870C876D
:10AF8000DF91CF911F910F91FF90EF900895CF9394
:10AF9000DF93CDB7DEB7A2970FB6F894DEBF0FBE32
:10AFA000CDBF80310CF080E12EEC34E13A8329836F
:10AFB00026EC34E13C832B832EEB34E13E832D835E
:10AFC00026EB34E138872F832EEA34E13A8729874C
:10AFD00026EA34E13C872B872EE934E13E872D8732
:10AFE00026E934E1388B2F8728E834E13A8B298B26
:10AFF00026E734E13C8B2B8B29E534E13E8B2D8B0E
:10B0000024E434E1388F2F8B2AE334E13A8F298FFF
:10B0100020E334E13C8F2B8F23E234E13E8F2D8FF0
:10B0200027E134E138A32F8F2FE034E13AA329A39D
:10B03000E82FEE0FFF0BEC0FFD1F81819281A2968E
:10B040000FB6F894DEBF0FBECDBFDF91CF9108954C
:10B050008F929F92AF92BF92CF92DF92EF92FF9228
:10B060000F931F93DC0118968D919C9119971E9652
:10B07000CD90DC901F976817790709F456C0589651
:10B08000FC9058974C01092E000CAA08BB088B01B4
:10B09000072E000C220B330B861797073CF41696ED
:10B0A000ED91FC911797FF2039F015C01496ED91A2
:10B0B000FC911597FF2079F00D2C000CEE08FF088D
:10B0C000A9019801281939094A095B091C966D9153
:10B0D0007C911D970EC00D2C000CEE08FF08A901F5
:10B0E0009801281939094A095B091A966D917C91D2
:10B0F0001B97CB01770FAA0BBB0BBC01CD016C19C1
:10B100007D098E099F090E9442B58F01FF0F220B16
:10B11000330BA9019801281939094A095B090E94D2
:10B12000DBBAC20ED31EE41EF51EC6011F910F919D
:10B13000FF90EF90DF90CF90BF90AF909F908F9057
:10B140000895EF92FF920F931F93CF93DF938C019B
:10B15000FC01778B668B7CDFEC01F80182819381A7
:10B160008830910529F57801F9E1EF0EF11CD7FF40
:10B1700006C06AE0C1388FEFD80754F001C068E01C
:10B180002C2F9D2FC038D1052CF02FE790E002C066
:10B1900021E89FEF422F592F57FF03C0519541954A
:10B1A0005109C70173D9CD2B59F54FE766E026C089
:10B1B000099731F57801E9E1EE0EF11CD7FF06C0E1
:10B1C0006EE0C138FFEFDF0754F001C06CE02C2FB8
:10B1D0009D2FC038D1052CF02FE790E002C021E868
:10B1E0009FEF422F592F57FF03C0519541955109A9
:10B1F000C7014CD9CD2B21F44FE767E0C70146D9F1
:10B200000E940049F801648F758F868F978FDF91B8
:10B21000CF911F910F91FF90EF900895CF93DF93FF
:10B22000EC017F8B6E8B14DF9C018A819B818830BF
:10B230009105C1F437FF06C061E021388FEF380770
:10B240004CF001C060E0A901203831052CF04FE737
:10B2500050E002C041E85FEF57FF1FC05195419594
:10B2600051091BC00997E9F4922F832F203831052B
:10B2700014F09FE780E0492F582F41388FEF58078F
:10B2800014F441E85FEF57FF03C051954195510910
:10B29000632F661F6627661F6C5FCE0149960E946A
:10B2A000C4800E9400496C8F7D8F8E8F9F8FDF91AD
:10B2B000CF9108950F931F93CF93DF93EC010E94DA
:10B2C00000490C8D1D8D2E8D3F8DDC01CB01801B27
:10B2D000910BA20BB30B853F9140A105B10540F046
:10B2E0006E897F89CE01DF91CF911F910F9196CF0B
:10B2F000DF91CF911F910F910895CF93DF93EC01D0
:10B300007F8B6E8BA5DE9C018A819B8188309105A5
:10B31000C1F437FF06C061E021388FEF38074CF0E9
:10B3200001C060E0A901203831052CF04FE750E062
:10B3300002C041E85FEF57FF1FC051954195510989
:10B340001BC00997E9F4922F832F2038310514F0A0
:10B350009FE780E0492F582F41388FEF580714F4AA
:10B3600041E85FEF57FF03C0519541955109632FA5
:10B37000661F6627661F6C5FCE0149960E94878014
:10B380000E9400496C8F7D8F8E8F9F8FDF91CF91B0
:10B3900008950F931F93CF93DF93EC010E94004910
:10B3A0000C8D1D8D2E8D3F8DDC01CB01801B910BF3
:10B3B000A20BB30B853F9140A105B10540F06E890A
:10B3C0007F89CE01DF91CF911F910F9196CFDF91B1
:10B3D000CF911F910F910895CF93DF93EC0161E01E
:10B3E00089E00E943C4660E089E00E94D6441092C9
:10B3F000F8098CE295E099838883DF91CF910895D5
:10B40000CF92DF92EF92FF928091F909833009F099
:10B4100061C08091FA098130D1F488EE93E0A0E018
:10B42000B0E080938B0990938C09A0938D09B09321
:10B430008E0980E797E1A0E0B0E080938F099093B8
:10B440009009A0939109B093920932E001C030E0D5
:10B45000E091FA09F0E0E550F64F2081A0E1A30F5A
:10B4600048EE53E060E070E088EBC82E8BE0D82E09
:10B47000E12CF12C832F90E0FC01EE0FFF1FEE0F6B
:10B48000FF1FE557F64F27FF10C0C082D182E2822E
:10B49000F382880F991F880F991FFC01E157F64F1F
:10B4A00040835183628373830FC0408351836283DF
:10B4B0007383880F991F880F991FFC01E157F64F7E
:10B4C000C082D182E282F3823E5F220F3A13D2CF52
:10B4D0003093F409FF90EF90DF90CF900895CF93D1
:10B4E000DF938091F809811153C01092F6091092F0
:10B4F000F309C1E0C093F809D091F70961E089E050
:10B500000E943C4660E089E00E94D6442D2F30E046
:10B5100040E050E060E47FE180E090E00E94DBBA30
:10B52000C093B00089E08093B1002093B3008BEA10
:10B53000289F212D112426952093B40080916F001F
:10B540008B7F80936F008091B00080628093B00009
:10B550002091840030918500E091F30981E08E0F05
:10B560008093F30984E0E89FF0011124E557F64F3A
:10B5700080819181A281B381820F931F90938B0070
:10B5800080938A00B29A80916F00846080936F00EC
:10B59000DF91CF9108954F925F926F927F928F9239
:10B5A0009F92AF92BF92CF92DF92EF92FF928AE189
:10B5B0008093F4092093F50988E28093F70981E0EC
:10B5C0008093FA098093FB098EE08093F90980EC5F
:10B5D00092E1A0E0B0E080938B0990938C09A09356
:10B5E0008D09B0938E0980EB94E0A0E0B0E08093E9
:10B5F0008F0990939009A0939109B0939209A4E1C7
:10B60000440F551F661F771FAA95D1F722E030E03F
:10B61000B0EBCB2EB4E0DB2EE12CF12C80E6482EF3
:10B6200089E0582E612C712C90E4892E9CE9992E8A
:10B63000A12CB12CC901880F991F880F991FFC01FB
:10B64000E557F64F77FF05C04082518262827382D0
:10B6500004C0C082D182E282F382C9010196880FC0
:10B66000991F880F991FFC01E557F64F283129F0E3
:10B67000C082D182E282F38204C080829182A2825F
:10B68000B382440F551F661F771F2E5F3F4F2A312D
:10B69000310581F6FF90EF90DF90CF90BF90AF9093
:10B6A0009F908F907F906F905F904F9018CF8F9268
:10B6B0009F92AF92BF92CF92DF92EF92FF9282E180
:10B6C0008093F40986E08093F50996E29093F70958
:10B6D00091E09093FA099093FB098093F90988ED22
:10B6E00090E4A0E0B0E080938B0990938C09A09344
:10B6F0008D09B0938E098CE19CE0A0E0B0E08093CE
:10B700008F0990939009A0939109B0939209742F97
:10B7100066275527442722E030E0ACE1CA2EACE092
:10B72000DA2EE12CF12CB8E38B2EB8E19B2EA12C64
:10B73000B12CC901880F991F880F991FFC01E5578B
:10B74000F64F77FF05C080829182A282B38204C047
:10B75000C082D182E282F382F901EE0FFF1FEE0F69
:10B76000FF1FE157F64FC082D182E282F382440F7D
:10B77000551F661F771F2E5F3F4F22313105C9F6D7
:10B780008CE199E8A0E0B0E08093CF099093D009D4
:10B79000A093D109B093D209FF90EF90DF90CF90A2
:10B7A000BF90AF909F908F909ACE1F920F920FB63E
:10B7B0000F9211240BB60F922F933F934F935F93E9
:10B7C0006F937F938F939F93AF93BF93EF93FF9369
:10B7D0009091F3098091F409981316C01092F3091F
:10B7E0008091FA098F5F8093FA099091FA0980910C
:10B7F000FB09891740F481E08093FA098091F609EA
:10B800008F5F8093F609FCDD9091F6098091F50930
:10B8100098130DC08091B0008F7D8093B00080910F
:10B820006F008B7F80936F001092F80927C0809182
:10B83000B00085FF04C08091B0008F7D03C080916F
:10B84000B00080628093B000209184003091850028
:10B85000E091F30981E08E0F8093F30984E0E89F83
:10B86000F0011124E557F64F80819181A281B381C7
:10B87000820F931F90938B0080938A00FF91EF912A
:10B88000BF91AF919F918F917F916F915F914F91F8
:10B890003F912F910F900BBE0F900FBE0F901F90F6
:10B8A00018958091B0069091B106DC01ED91FC9164
:10B8B0000084F185E02D19958091B0069091B10634
:10B8C000DC01ED91FC910480F581E02D19948091CB
:10B8D0001306882371F0109213068091B606882310
:10B8E00041F06FEB75E18091B4069091B5060C9430
:10B8F000007C089580916110833099F08091130647
:10B9000081110FC081E0809313068091B6068823D1
:10B9100041F06AEA75E18091B4069091B5060C9405
:10B92000007C089580911306882319F080E090E050
:10B93000CECF80E090E0DECF80911206833079F0A8
:10B9400083E0809312068091B606882341F069E96E
:10B9500075E18091B4069091B5060C94007C089531
:10B9600080911206823079F082E0809312068091F5
:10B97000B606882341F068E875E18091B40690919D
:10B98000B5060C94007C089580911206813079F000
:10B9900081E0809312068091B606882341F067E724
:10B9A00075E18091B4069091B5060C94007C0895E1
:10B9B0008091070180FF1BC08091B606882351F05B
:10B9C0008CE39BE00E947495811108C08091480B24
:10B9D000811104C08CE39BE00C9463956AE876E1E6
:10B9E0008091B4069091B5060E94007CF3CF089533
:10B9F0008091070181FF1BC08091B606882351F01A
:10BA000085E19BE00E947495811108C08091210B13
:10BA1000811104C085E19BE00C9463956DE576E1AE
:10BA20008091B4069091B5060E94007CF3CF0895F2
:10BA30008091070180FF17C08091B606882331F0FE
:10BA40008CE39BE00E947495882321F08CE39BE0BB
:10BA50000C94799564E776E18091B4069091B506EF
:10BA60000E94007CF3CF08958091070181FF17C0E9
:10BA70008091B606882331F085E19BE00E947495A1
:10BA8000882321F085E19BE00C94799567E476E1C9
:10BA90008091B4069091B5060E94007CF3CF089582
:10BAA0000E94BA8780911406882361F18091EB0A85
:10BAB000811128C08091AC06811124C081E080935F
:10BAC000AC060E94509480913F06882319F0109292
:10BAD0003F060CC08091B0069091B106DC01ED915B
:10BAE000FC910088F189E02D61E019958091B606FE
:10BAF000882341F06CE475E18091B4069091B5061D
:10BB00000C94007C089561E085E30E94D644809106
:10BB1000B0069091B106DC01ED91FC9106A8F7A961
:10BB2000E02D19958091B606882341F069ED76E104
:10BB30008091B4069091B5060C94007C08958F9284
:10BB40009F92AF92BF92CF92DF92EF92FF9285E4E5
:10BB50000E948448BC01990F880B990B0E9498B9E8
:10BB600020E030E040E85AE30E94F7B920E030E0FE
:10BB700040EA50E40E94F7B96B017C0180910E020B
:10BB8000882351F0C092770ED092780EE092790E11
:10BB9000F0927A0E10920E0226E636E646E65FE353
:10BBA0006091770E7091780E8091790E90917A0E57
:10BBB0000E94F7B94B015C0120ED3CEC4CEC5DE3DD
:10BBC000C701B6010E94F7B99B01AC01C501B401E0
:10BBD0000E948DB56093770E7093780E8093790EE6
:10BBE00090937A0E2DE33CE248E450E40E94F7B9CA
:10BBF0002AE939E949E95EE30E948DB5FF90EF90AB
:10BC0000DF90CF90BF90AF909F908F900895CF938B
:10BC1000DF938091070180FD2AC0C0914B06D0912F
:10BC20004C0680914F06882371F08EE30E94844871
:10BC3000813092402CF010924C0610924B060AC0B4
:10BC400081E090E003C08EE30E94844890934C060C
:10BC500080934B0680914B0690914C068C179D0764
:10BC600019F410924D0603C081E080934D06DF91D8
:10BC7000CF910895CF93DF938091070181FD2AC072
:10BC8000C0914506D091460680914906882371F0FF
:10BC90008FE30E948448813092402CF01092460637
:10BCA000109245060AC081E090E003C08FE30E9435
:10BCB000844890934606809345068091450690916E
:10BCC00046068C179D0719F41092470603C081E0C1
:10BCD00080934706DF91CF9108959091B60688230F
:10BCE000D9F0809111078823B9F081E08093731017
:10BCF0008093740E992311F166E176E18091B40688
:10BD00009091B5060E948F7A0E94DF958091B406CB
:10BD10009091B5060C94ED7B10927310992341F02D
:10BD20006EE276E18091B4069091B5060E94007CA7
:10BD300080917110811102C01092740E089590913B
:10BD4000B6068823F9F0809111078823D9F08091F5
:10BD500022108D30B9F481E0809371108093740EBD
:10BD6000992311F165ED75E18091B4069091B506C6
:10BD70000E948F7A0E940D968091B4069091B5062C
:10BD80000C94ED7B10927110992341F065EF75E1F1
:10BD90008091B4069091B5060E94007C809173104A
:10BDA000811102C01092740E089580916110833049
:10BDB00041F12CF48130A9F0823099F02DC0863009
:10BDC0005CF58091A5069091A606DC01ED91FC91B1
:10BDD0000480F581E02D19958091A3069091A40629
:10BDE00014C08091A9069091AA06DC01ED91FC9106
:10BDF0000480F581E02D19958091A7069091A80601
:10BE000004C08091A5069091A606DC01ED91FC91FD
:10BE10000480F581E02D19958091B0069091B106CE
:10BE2000DC01ED91FC91E65BFF4F0190F081E02D8C
:10BE300019958091B0069091B106DC01ED91FC91CD
:10BE40000284F385E02D60E070E019940E94BA87C7
:10BE5000809114068823D1F08091AC068823B1F03C
:10BE60001092AC060E941E9480913F06882389F0B0
:10BE700010923F068091B606882341F060E675E196
:10BE80008091B4069091B5060E94007C1092AC0699
:10BE900008958091B0069091B106DC01ED91FC917E
:10BEA0000088F189E02D60E01995E4CFCF93DF930E
:10BEB000C091750ED091760EBE0184E69BE00E9483
:10BEC000DE3D882329F0BE0184E69BE00E94F63D1A
:10BED0001092760E1092750EDF91CF9108950F9308
:10BEE0001F93CF93DF938091661090916710A0917C
:10BEF0006810B0916910181619061A061B060CF086
:10BF000044C00E94BA87809114068823C9F1009129
:10BF1000750E1091760EB80184E69BE00E94DE3D1E
:10BF20008823D9F0E2E6FDE0C0E0D0E08191919174
:10BF30008017910769F40E940049CC0FDD1FCC0FD8
:10BF4000DD1FCC59D44F688379838A839B831DC0BE
:10BF50002196CE31D10551F718C04091661050910D
:10BF60006710609168107091691021EB30E684E6EB
:10BF70009BE00E94453E9093760E8093750E05C01F
:10BF8000DF91CF911F910F9191CFDF91CF911F91B1
:10BF90000F9108958091EB0A811148C00E94BA87E1
:10BFA000809114138823B1F080911406882391F0B6
:10BFB00010921406109214130E94E1878091730E60
:10BFC000882341F067E275E18091710E9091720EC5
:10BFD0000E94007C8091420690914306806290937B
:10BFE0004306809342068091AC06882311F081E0DD
:10BFF00001C080E00E94829481E080933F0626DFAA
:10C000008091771081110FC080912A06882359F002
:10C0100021E53CE544E650E060E070E084E69BE02A
:10C020000E94453E01C03DDCC0DE59CF0895BDDE13
:10C030000E94C84A0E94BA87809114068111AADF23
:10C040008091B2069091B306DC01ED91FC910480E1
:10C05000F581E02D19958091AE069091AF06DC0137
:10C06000ED91FC910480F581E02D199580914210AD
:10C07000882359F080912B0690912C06DC01ED91DC
:10C08000FC910480F581E02D1994089580910D02B2
:10C09000882351F054DD20E030E040E050E40E947D
:10C0A00092B987FF39C008954ADD20E030E04AE7C1
:10C0B00054E40E94F7B90E945EB62091C2103091FC
:10C0C000C3104091B9066217730710F4442351F16D
:10C0D000442309F445C033DD20E030E04AE754E46E
:10C0E0000E94F7B90E945EB62091C2103091C31031
:10C0F00062177307A8F11092B90681E08093B80621
:10C100008091B606882361F161EA76E18091B406F8
:10C110009091B5060C94007C10920D0281E0809302
:10C12000B806089581E08093B9061092B806809110
:10C13000B606882391F060EC76E18091B406909188
:10C14000B5060E948F7A0E94C8956DEB76E18091CA
:10C15000B4069091B5060E94007C69DF0C94FB89BF
:10C1600008950E94BA8780911406882369F012DF2F
:10C170008091B606882341F067E375E18091B406AB
:10C180009091B5060C94007C08958091EB0A811182
:10C190005EC08091AD06823068F08091B60688233B
:10C1A00009F455C065EE74E18091B4069091B5062E
:10C1B0000C94007C0E94BA8780911413882309F4A0
:10C1C00046C080911406811142C081E0809314061C
:10C1D000109214130E94E1878091730E882341F01E
:10C1E00066ED74E18091710E9091720E0E94007C58
:10C1F000809142069091430680619093430680931C
:10C2000042068091B0069091B106DC01ED91FC915F
:10C210000280F381E02D19958091AD06811116C041
:10C2200040915C1050915D1081E080933F06411574
:10C23000510559F060E070E020E53DE584E69BE0C3
:10C240000E94453E0E941E9401C02ADC48CE0895FB
:10C2500080910F02882311F0729801C0729A909118
:10C260000F0281E0892780930F0208951092ED0A52
:10C2700040912E0650912F0660E070E02FE431E6E9
:10C2800080911C0690911D060C94453E81E08093A0
:10C29000E90A809138060E9408720C9474441F9336
:10C2A000CF93DF93CDB7DEB765970FB6F894DEBFB7
:10C2B0000FBECDBF11E01093ED0A8091A50E88232B
:10C2C000B9F185E09AE00E9454881092160A82E340
:10C2D00090E09A83898328E230E03C832B832EE62A
:10C2E00030E03E832D8324EF31E038872F831D8A91
:10C2F00025E1FE013196A7E1BAE001900D922A9561
:10C30000E1F79093150A8093140A84E08093130A4E
:10C3100085E09AE00E9459950E9400496093050AC1
:10C320007093060A8093070A9093080A1093110AE3
:10C3300065960FB6F894DEBF0FBECDBFDF91CF91EB
:10C340001F91089580919B0E811112C08CE591E997
:10C35000A1E0BB27ABBFFC016791769182E00E9410
:10C36000783F81E080937C0E1092800E10927D0EBB
:10C37000089561E08BE20E94D644EE9A2AE136E409
:10C3800048E853E160E070E080911C0690911D0642
:10C390000E94453E9093F10D8093F00D089561E069
:10C3A0008BE20E94D644EE9A2AE136E448E853E153
:10C3B00060E070E080911C0690911D060E94453E51
:10C3C0009093F10D8093F00D089581E20E94AE44A8
:10C3D00021E0892B09F420E0822F08958091340612
:10C3E000882309F446C081E08093E90AEEDF8823C0
:10C3F00029F0809137068823D1F106C08091350657
:10C40000811105C0809134060E94087230C090915D
:10C410003406963061F5823081F08330D1F081307E
:10C4200031F5E091550AF091560A74978081918117
:10C4300045E550E060E070E017C0E091550AF091EA
:10C44000560A7497808191814AE550E060E070E07F
:10C450000BC0E091550AF091560A74978081918142
:10C460004FE550E060E070E08B5A954F20D90C9476
:10C47000744408958091F30D882339F08091F20D72
:10C48000882319F081E08093E60A80911E0690913E
:10C490001F06DC01ED91FC910688F789E02D1995C6
:10C4A0008091A10E81110E94EE4A8091A00E8823F6
:10C4B00091F061E088E00E94D64440919E0E509138
:10C4C0009F0E60E070E024E136E480911C069091BC
:10C4D0001D060E94453E8091F30D882321F0809136
:10C4E000F20D811101C07ADF8091F20D882379F07D
:10C4F0008091F30D882359F08091A40E882339F0A0
:10C50000E091A20EF091A30E82810E94BA7EAECE7F
:10C510008091EB0A811156C058DF8823F1F081E049
:10C520008093EB0A80911E0690911F06DC01ED912D
:10C53000FC910288F389E02D19950E94814523EA38
:10C5400035E448E95AE360E070E080911C06909180
:10C550001D060E94453E8ADE09C08091F20D8823A7
:10C5600029F18091F30D882311F019DF37CF01DF16
:10C570008091A40E882339F0E091A20EF091A30ED1
:10C5800082810E94BA7E40919C0E50919D0E14169D
:10C590001506BCF4052E000C660B770B2AE332E679
:10C5A00080911C0690911D060C94453E8091A40E2E
:10C5B000882339F0E091A20EF091A30E82810E94AF
:10C5C000BA7E58CF08950F931F9320919B0E21118F
:10C5D00035C04CE551E961E077279C01220F331FFC
:10C5E000820F931F092E000CAA0BBB0B0296A11DF4
:10C5F000B11D840F951FA61FB71FABBFFC0187910C
:10C600000CE511E921E033274091800E93E0499F2A
:10C61000A0011124052E000C660B770B4E5F5F4FB7
:10C620006F4F7F4F040F151F261F371F2BBFF801B9
:10C630000791801718F01F910F9184CE1F910F91D1
:10C6400008958F929F92AF92BF92CF92DF92EF9216
:10C65000FF920F931F93CF93DF93EC01A62E80914F
:10C660009B0E81116BC04CE551E961E077276E01AB
:10C67000CC0CDD1CCC0EDD1E0D2C000CEE08FF08D2
:10C68000D701C6010296A11DB11D480F591F6A1F8F
:10C690007B1F6BBFFA0187914CE551E961E0772779
:10C6A000B090800E93E0B99E80011124012E000C01
:10C6B000220B330B0E5F1F4F2F4F3F4F400F511F69
:10C6C000621F731F6BBFFA014791481708F036C00D
:10C6D00080907E0E90907F0E0091940E1091950E9A
:10C6E000B401C8010E94DE3D882321F0B401C801D5
:10C6F0000E94F63D8CE591E9A1E0BB278C0D9D1DC4
:10C70000AE1DBF1DABBFFC016791769182E00E9418
:10C71000783FB0927D0EC093800EAA2079F01092DF
:10C720007C0E22EA31E642E350E060E070E0C801AE
:10C730000E94453E90937F0E80937E0EDF91CF91B5
:10C740001F910F91FF90EF90DF90CF90BF90AF902F
:10C750009F908F900895CF92DF92EF92FF928091F9
:10C760009B0E811134C080919A0E882381F161E083
:10C770008EE090E066DF6091980E7091990ECB018B
:10C78000A0E0B0E0C090960ED090970EE12CF12C76
:10C79000C816D906EA06FB0664F4BC01CD016C1983
:10C7A0007D098E099F090E94647AC60ED71EE81E75
:10C7B000F91E2BEA33E6B701A6018091940E909101
:10C7C000950E0E94453E9093930E8093920EFF909B
:10C7D000EF90DF90CF900895CF92DF92EF92FF928B
:10C7E00080919B0E811134C08091910E882381F13C
:10C7F00061E08DE090E025DF60918F0E7091900EEA
:10C80000CB01A0E0B0E0C0908D0ED0908E0EE12C58
:10C81000F12CC816D906EA06FB0664F4BC01CD016A
:10C820006C197D098E099F090E94647AC60ED71E75
:10C83000E81EF91E2CEE33E6B701A6018091940E96
:10C840009091950E0E94453E90938C0E80938B0E96
:10C85000FF90EF90DF90CF900895CF92DF92EF920C
:10C86000FF9280919B0E811134C080918A0E8823A3
:10C8700081F161E08CE090E0E4DE6091880E7091DF
:10C88000890ECB01A0E0B0E0C090860ED090870E5C
:10C89000E12CF12CC816D906EA06FB0664F4BC01AB
:10C8A000CD016C197D098E099F090E94647AC60E1C
:10C8B000D71EE81EF91E2DE234E6B701A6018091CD
:10C8C000940E9091950E0E94453E9093850E809314
:10C8D000840EFF90EF90DF90CF90089580919B0E93
:10C8E00081112CC08091830E882341F080918A0EA3
:10C8F000811104C081E080938A0EAFDF8091820EA7
:10C90000882361F080919B0E811108C08091910E67
:10C91000811104C081E08093910E5EDF8091810ED1
:10C92000882361F080919B0E811108C080919A0E3E
:10C93000811104C081E080939A0E0DCF08958091FB
:10C940009B0E81110BC080917B0E882339F060ED26
:10C9500077E081E00E94783F0C944D3E08952F923D
:10C960003F924F925F926F927F928F929F92AF927F
:10C97000BF92CF92DF92EF92FF920F931F93CF93CC
:10C98000DF9300D01F92CDB7DEB75C0150DB0E9471
:10C990009A8B0E94D18B8091B4069091B5060E942B
:10C9A000ED7B0E94E24324E0A216B10409F49CC08E
:10C9B0000CF04FC0A3E0AA16B10409F03CC18CE111
:10C9C00090E00E9492B69C838B838AEE95E0AB81C7
:10C9D000BC8111969C938E931396BC92AE92129743
:10C9E00081E09FEF15969C938E9314978FEF90E0C4
:10C9F00017969C938E93169719961C921E921897D1
:10CA000058961C925897CD010E9409808EED95E0B2
:10CA1000EB81FC8191838083E091150EF091160EDD
:10CA2000D08C00913F121091401216950795E0901E
:10CA30003D12F0903E12F694E79468EC77E1809115
:10CA4000B4069091B5060E94007C812C99249394A1
:10CA500012C1B5E0AB16B10409F4A6C0E6E0AE160B
:10CA6000B10409F0E8C08CE190E00E9492B69C838A
:10CA70008B838AEE95E0AB81BC8111969C938E935B
:10CA80001396BC92AE92129781E09FEF15969C93FD
:10CA90008E9314978FEF90E017969C938E93169732
:10CAA00019961C921E92189758961C925897CD0171
:10CAB0000E9409808EED95E0EB81FC81918380835B
:10CAC000E091A006F091A106D08C00917E12109109
:10CAD0007F1216950795E0907C12F0907D12F694E7
:10CAE000E7946BEF77E1A0C08CE190E00E9492B6F2
:10CAF0009C838B838AEE95E0AB81BC8111969C93DD
:10CB00008E931396BC92AE92129781E09FEF15968A
:10CB10009C938E9314978FEF90E017969C938E932F
:10CB2000169719961C921E92189758961C92589711
:10CB3000CD010E9409808EED95E0EB81FC8191830F
:10CB40008083009154121091551216950795E0902C
:10CB50005212F0905312F694E794809122108C5068
:10CB6000823040F4E091B206F091B306D08C6BE3D2
:10CB700078E15AC080916110823009F07AC08091CA
:10CB800020108C3009F075C0E091A006F091A1064C
:10CB9000D08C6BE178E18091B4069091B5060E944B
:10CBA000007C8824839466C08CE190E00E9492B659
:10CBB0009C838B838AEE95E0AB81BC8111969C931C
:10CBC0008E931396BC92AE92129781E09FEF1596CA
:10CBD0009C938E9314978FEF90E017969C938E936F
:10CBE000169719961C921E92189758961C92589751
:10CBF000CD010E9409808EED95E0EB81FC8191834F
:10CC00008083E091AE06F091AF06D08C009169125E
:10CC100010916A1216950795E0906712F0906812CD
:10CC2000F694E7946BED77E18091B4069091B506A8
:10CC30000E94007C1EC06FEA77E18091B40690915B
:10CC4000B5060F900F900F900F90DF91CF911F912D
:10CC50000F91FF90EF90DF90CF90BF90AF909F909B
:10CC60008F907F906F905F904F903F902F900C949B
:10CC7000007C812C912C0E94E24362EA77E1809152
:10CC8000B4069091B5060E94007C66E977E1809138
:10CC9000B4069091B5060E948F7AB8018091B406CF
:10CCA0009091B5060E940A766AE877E18091B40611
:10CCB0009091B5060E948F7AB7018091B406909149
:10CCC000B5060E940A766EE777E18091B4069091EE
:10CCD000B5060E948F7A8D2D0E94BE438091B406C6
:10CCE0009091B5060E94ED7BAB81BC81ED91FC91EA
:10CCF00011970280F381E02DCD011995CA2C8A2D60
:10CD00000E94257F8D3D9540A8F464E378E08A2D4C
:10CD10000E941B7FEB81FC81F78AE68AB701828142
:10CD20000E94357F6CED75E08A2D0E94207FDD200A
:10CD3000C1F01AC064E873E08A2D0E94207FAB81A5
:10CD4000BC8157961C930E935697B80112968C91FE
:10CD50000E94357F6CED75E08A2D0E941B7FDD20DF
:10CD600019F03324339401C0312C21E02983212C84
:10CD70002A830E947F528091E811882359F1AB8168
:10CD8000BC81ED91FC9111976091ED117091EE11C4
:10CD90000190F081E02DCD0119958C2D0E94257F09
:10CDA0008D3DB5E09B075CF48438E3E09E0784F09A
:10CDB0008C018D3D954074F00CED15E00BC07C01AD
:10CDC000853398403CF064E3E62E68E0F62E02C01E
:10CDD00004E813E02A8121111FC08091DE1188230D
:10CDE000C9F1E091E511F091E611858196814091BC
:10CDF000E1115091E2119C0121533109421753076F
:10CE00004CF1C196841795072CF10E9400496415D6
:10CE1000750586059705F0F08091DE118823C1F035
:10CE20004091E1115091E211E091E511F091E6118C
:10CE3000858196819C01285C3109421753072CF0AB
:10CE400088539F4F841795071CF481E0382605C04E
:10CE500021E02A83222009F47CC0332009F445C054
:10CE6000DD20F9F064E873E08C2D0E94207F99208A
:10CE700009F458C060913C1070913D1041E08C2D38
:10CE80000E94DA7E0E94E194AB81BC8112968C9163
:10CE90000E94257F08171907ACF38C2D0E94AC7EE9
:10CEA00041C064E378E08C2D0E941B7F9920B1F093
:10CEB00060913C1070913D1040E08C2D0E94DA7E14
:10CEC0000E94E194AB81BC8112968C910E94257FD7
:10CED0008E159F05ACF38C2D0E94AC7EEB81FC81FE
:10CEE000F78AE68AB701828110C0DD20B1F064E3E1
:10CEF00078E08C2D0E941B7FAB81BC815796FC9201
:10CF0000EE925697B70112968C910E94357F6CED88
:10CF100075E08C2D0E94207F12C064E873E08C2D98
:10CF20000E94207FEB81FC81178B068BB8018281E8
:10CF30000E94357F6CED75E08C2D0E941B7F0E9456
:10CF400000492B013C01F8EC4F0E511C611C711C77
:10CF50001A8229812223D9F18091D4118823A9F141
:10CF60004091D7115091D811E091DB11F091DC1173
:10CF7000858196819C01285C3109421753072CF06A
:10CF800088539F4F8417950704F581E0D826809138
:10CF9000B4069091B506DD2039F06FE677E10E9486
:10CFA000007C82E090E006C06DE577E10E94007CA5
:10CFB00081E090E00E94A28B0E940049AB81BC817D
:10CFC0005896DC922224239403C0212C1EC0212CCD
:10CFD0008091D411882309F472C2E091DB11F091A1
:10CFE000DC11858196814091D7115091D8119C0117
:10CFF00021533109421753070CF461C2C19621E055
:10D000002983841795070CF45AC20E9408820E9453
:10D01000577584E69BE00E94673E8091050B88234C
:10D0200009F4A7CE8091070B882309F4A2CE0E94B1
:10D0300057750E94928D8823D1F384E0A816B1041D
:10D04000D9F134F4B3E0AB16B10409F438C1C4C16A
:10D05000E5E0AE16B10409F4CDC0F6E0AF16B104B8
:10D0600009F0BAC11093301000932F10F0923210D3
:10D07000E0923110D0923310B8018CE291E00E941E
:10D08000E874B7018EE291E00E94E8746D2D80E3B0
:10D0900091E00E943B76B80186E00E945D3FB701B7
:10D0A00086E00E94423FE091A006F091A106D08E5A
:10D0B0006CED75E086E091C08820C1F010933010CF
:10D0C00000932F10F0923210E0923110D092331072
:10D0D000B8018CE291E00E94E874B7018EE291E021
:10D0E0000E94E8746D2D80E391E017C01093241026
:10D0F00000932310F0922610E0922510D092271072
:10D10000B80180E291E00E94E874B70182E291E008
:10D110000E94E8746D2D84E291E00E943B76B80194
:10D1200084E00E945D3FB70184E00E94423F882076
:10D1300049F0E091A006F091A106D08E6CED75E06B
:10D1400084E04BC0E091B206F091B306D08E80919E
:10D1500022108D3029F4E091A60EF091A70ED08E0A
:10D160006CED75E084E00E94357F66E970E080E058
:10D1700090E00E94C848809122108D3011F584E023
:10D180000E94257FA091B206B091B3068D3D9540D7
:10D190004CF0ED91FC9111970190F081E02D6FEF33
:10D1A0007FEF08C0ED91FC9111970190F081E02D87
:10D1B00061E070E0CD0119958091B2069091B306BF
:10D1C0006FC08091B2069091B306DC01ED91FC91A5
:10D1D0000480F581E02D1995FFC00E94357F66E936
:10D1E00070E080E090E00E94C8488091A006909195
:10D1F000A106EBCF10932B1000932A10F0922D1064
:10D20000E0922C10D0922E10B80187E291E00E949B
:10D21000E874B70189E291E00E94E8746D2D8BE219
:10D2200091E00E943B76B80185E00E945D3FB70126
:10D2300085E00E94423FE091AE06F091AF06D08EAD
:10D240006CED75E085E00E94357F66E970E080E076
:10D2500090E00E94C848809121108D3059F585E0FA
:10D260000E94257FA091AE06B091AF068D3D9540FE
:10D270004CF0ED91FC9111970190F081E02D6FEF52
:10D280007FEF08C0ED91FC9111970190F081E02DA6
:10D2900061E070E0CD0119958091AE069091AF06E6
:10D2A000DC01ED91FC910190F081E02D60E070E0F7
:10D2B000199592C08091AE069091AF0686CF1093DB
:10D2C0003F1000933E10F0924110E0924010D09237
:10D2D0003810B8018BE391E00E94E874B7018DE348
:10D2E00091E00E94E8746D2D85E391E00E943B7609
:10D2F000B80183E00E945D3FB70183E00E94423F96
:10D3000080913810E091150EF091160E808F80916B
:10D3100038100E94B37483E00E94257F209138105A
:10D32000222369F1B9E0BC1538F020913F12309109
:10D3300040123695279502C02EEE32E082179307F1
:10D3400009F44AC060913C1070913D1041E083E0C7
:10D350000E94DA7E0E94E194EB81FC8182810E942E
:10D36000257F08171907B4F383E00E94AC7EAB81D8
:10D37000BC8157961C930E935697B80129C029E09B
:10D380002C1508F49EC020913D1230913E12369526
:10D3900027958217930701F160913C1070913D1021
:10D3A00040E083E00E94DA7E0E94E194EB81FC8100
:10D3B00082810E94257F8E159F05B4F383E00E9431
:10D3C000AC7EAB81BC815796FC92EE925697B7012A
:10D3D00012968C910E94357F8091B4069091B5068B
:10D3E0000E94ED7B0E94E243B4E0AB16B10459F019
:10D3F000E5E0AE16B10451F0F3E0AF16B10471F4FC
:10D4000063E177E105C063E477E102C06AE277E1B6
:10D410008091B4069091B5060E94007C0E94E24380
:10D4200068E077E18091B4069091B5060E94007C97
:10D430006CEF76E18091B4069091B5060E948F7AE8
:10D44000B8018091B4069091B5060E940A7660EF0B
:10D4500076E18091B4069091B5060E948F7AB7016B
:10D460008091B4069091B5060E940A7664EE76E14A
:10D470008091B4069091B5060E948F7A8D2D0E94FE
:10D48000BE438091B4069091B5060E94ED7B0F904B
:10D490000F900F900F90DF91CF911F910F91FF9000
:10D4A000EF90DF90CF90BF90AF909F908F907F9044
:10D4B0006F905F904F903F902F900C94CD8B19827E
:10D4C000A4CD2AEC38E065CF089508950895089515
:10D4D0000895623039F0633041F0613041F4409397
:10D4E000830E08954093820E08954093810E08950F
:10D4F000623069F06330A1F06130D1F45093870E4F
:10D500004093860E3093890E2093880E0895509391
:10D510008E0E40938D0E3093900E20938F0E0895B3
:10D520005093970E4093960E3093990E2093980E39
:10D530000895FC018581089508950895089508953A
:10D5400020919B0E211102C0FC016283089520915D
:10D550009B0E211102C0FC016483089520919B0E53
:10D56000211102C0FC0163830895089508958091FC
:10D570009B0E811102C00C949F3F0895089580E096
:10D58000089508950895089508950895089580913F
:10D590009B0E811103C08FE090E015C80895809123
:10D5A0009B0E811121C0633091F028F4613049F065
:10D5B000623051F00895653081F060F0663081F09E
:10D5C000089589E090E00EC08AE090E00BC08BE007
:10D5D00090E008C08CE090E005C08DE090E002C0D3
:10D5E0008EE090E00C94E362089520919B0E21114F
:10D5F00008C0FC018481882321F082E090E00C9433
:10D60000E362089520919B0E211108C0FC018381E3
:10D61000882321F081E090E00C94E36208958091EA
:10D620009B0E811104C08BE090E00C94E36208959E
:10D6300080919B0E811104C060E080E190E001C800
:10D64000089580919B0E811105C060E08FE090E00D
:10D650000C942163089580919B0E811127C0633043
:10D66000A1F028F4613049F0623059F00895653036
:10D67000A1F078F06630A9F0089560E089E090E0CC
:10D6800013C060E08AE090E00FC060E08BE090E0C3
:10D690000BC060E08CE090E007C060E08DE090E0BF
:10D6A00003C060E08EE090E00C94216308958091C7
:10D6B0009B0E811127C06330A1F028F4613049F03E
:10D6C000623059F008956530A1F078F06630A9F025
:10D6D000089561E089E090E013C061E08AE090E0A5
:10D6E0000FC061E08BE090E00BC061E08CE090E067
:10D6F00007C061E08DE090E003C061E08EE090E063
:10D700000C942163089520919B0E211109C0FC0106
:10D710008281882329F061E088E090E00C94216305
:10D72000089520919B0E211109C0FC01848188235A
:10D7300029F061E082E090E00C942163089520914B
:10D740009B0E211109C0FC018381882329F061E02F
:10D7500081E090E00C942163089580919B0E8111EB
:10D7600005C061E086E090E00C942163089580910B
:10D770009B0E811105C060E08BE090E00C9421636A
:10D78000089580919B0E811105C061E087E090E0D3
:10D790000C942163089580919B0E811105C061E076
:10D7A00085E090E00C9421630895CF93DF93FC0112
:10D7B00025812223A1F1EC0180919B0E81112EC0C5
:10D7C0006091840E7091850E8091940E9091950ECB
:10D7D0000E94F63D10928A0E80919B0E81110CC022
:10D7E00060918B0E70918C0E8091940E9091950E9D
:10D7F0000E94F63D1092910E80919B0E81110CC0FB
:10D800006091920E7091930E8091940E9091950E6E
:10D810000E94F63D10929A0E1092B30D1D82DF9178
:10D82000CF910895CF93DF93FC01258121111EC074
:10D83000EC0180919B0E811117C08091B30D811175
:10D8400013C02EE634E648EB5BE060E070E08091C8
:10D85000940E9091950E0E94453E9093850E809374
:10D86000840E81E08093B30D81E08D83DF91CF91B1
:10D87000089580919B0E882329F06CED75E081E07E
:10D880000C94783F84E090E00C94E36280919B0ECE
:10D89000882329F068EE73E081E00C94783F60E023
:10D8A00084E090E00C94216380919B0E81111BC059
:10D8B00080917B0E8823B9F068EE73E081E00E94CE
:10D8C000783F10927B0E2FE93FE348E95AE360E08E
:10D8D00070E08091940E9091950E0E94453E909339
:10D8E000B50D8093B40D08956CED75E080E00C9457
:10D8F000783F24EF31E0DB010E9486B52FEF30E066
:10D9000040E050E00E94DBBACA01B90164527A4F8C
:10D910008F4F9F4F80E00C94783F80919B0E88231F
:10D9200039F060ED77E081E00E94783F0C944D3E45
:10D9300061E083E090E00C94216320919B0E211123
:10D9400003C002960C949F64089520919B0E22239D
:10D9500089F06FE676E080E00E94783F25EA3FE3B9
:10D9600042E350E060E070E08091940E9091950E5B
:10D970000C94453E02960C949F6480E00E94937E36
:10D9800081E00E94937E80919B0E811103C082E012
:10D990000E94937E6CED75E080E00E94783F6CED14
:10D9A00075E081E00E94783F80919B0E81110DC04F
:10D9B0008CE591E9A1E0BB27ABBFFC0167917691B3
:10D9C00082E00E94783F0C94A2610895FC01808956
:10D9D00091899387828782899389958784878489AF
:10D9E000958997878687089526E00C947A7D089517
:10D9F0000895FC01828193818830910529F4109269
:10DA00002B0110922A010895099721F410922901FF
:10DA1000109228010895FC01178A168A6CED75E0B2
:10DA200082810C94357FCF93DF93EC011F8A1E8A8D
:10DA30008A810E94AC7E8B8D882331F08A810E947E
:10DA4000257F9A8F898F1B8EDF91CF910895DF926A
:10DA5000EF92FF920F931F93CF93DF93EC018A8194
:10DA6000893010F40E94937EDD8C6B8D7C8D098D46
:10DA70001A8DEA80FB8089E08E1508F466C00F30AD
:10DA8000110538F001369DE6190728F000E61DE67D
:10DA900002C00FE010E06F30710538F061368DE69E
:10DAA000780728F060E67DE602C06FE070E080E075
:10DAB00090E00E9496B920E030E04AE754E40E94EA
:10DAC000F1B520E030E04CE852E40E94F7B99B0148
:10DAD000AC0160E070E08AEF94E40E94F1B50E942E
:10DAE00059B6FF2425E12E9DF0012F9DF00D112444
:10DAF000E550FE4EDD2071F023813481AB0177FFCC
:10DB000004C044275527461B570B88279927841B99
:10DB1000950B0AC025813681AB0177FF04C04427ED
:10DB20005527461B570BCA014FB7F89455E15E9D28
:10DB3000F0015F9DF00D1124E550FE4E108B07871C
:10DB4000328B218B948B838B4FBF9D8D6B8D7C8D06
:10DB50008A819923F9F08A3058F495E1899FF00180
:10DB60001124E550FE4E058116811695079502C0D9
:10DB70000EEE12E041E00E94DA7E61E070E080E0AB
:10DB800090E00E94C8488A810E94257F08171907E3
:10DB9000A0F31EC08A3058F495E1899FF00111244A
:10DBA000E550FE4E038114811695079502C00AECDC
:10DBB00018E040E00E94DA7E61E070E080E090E0F2
:10DBC0000E94C8488A810E94257F80179107A0F390
:10DBD0008A810E94AC7EB8018A81DF91CF911F912A
:10DBE0000F91FF90EF90DF900C94357FCF93DF93F0
:10DBF000EC018A81893010F40E94937E48EE53E054
:10DC00005B874A8720ED37E03D872C878CED95E0D8
:10DC10009F878E87598B488B3B8B2A8B9D8B8C8B58
:10DC2000DF91CF910895CF93DF93EC017F8B6E8BC3
:10DC3000888599856817790769F48A810E94AC7E86
:10DC40008B8D882329F18A810E94257F9A8F898F65
:10DC50001B8E1EC0CE010E942858EA81EA30B0F423
:10DC60009C01C39714F022E330E02E3C8FEF38077D
:10DC700014F42EEC3FEF8FB7F89495E1E99FF00193
:10DC80001124E550FE4E318720878FBF81E08B8FB6
:10DC9000DF91CF910895CF93DF93EC018BA19CA1ED
:10DCA000892B11F01CA21BA29B0177FF03C03195A9
:10DCB00021953109B901CE010E94285890932D0178
:10DCC00080932C019F8B8E8B0E9400496F8F78A3CD
:10DCD00089A39AA3DF91CF9108950F931F93CF93B8
:10DCE000DF938C01FC01778B668B0E942858EC0136
:10DCF000F8018281938188309105D1F4D7FF06C065
:10DD000060E08AE00E94D64461E005C061E08AE0FC
:10DD10000E94D64460E086E00E94D644D7FF03C04C
:10DD2000D195C195D109D0932B01C0932A011BC075
:10DD30000997C9F4D7FF06C060E08DE00E94D64481
:10DD400061E005C061E08DE00E94D64460E08BE0B8
:10DD50000E94D644D7FF03C0D195C195D109D09375
:10DD60002901C0932801DF91CF911F910F91089550
:10DD7000CF93DF93EC018A81893010F40E94937E67
:10DD80002EEC3FEF3B872A8782E390E09D878C87CC
:10DD90001F861E86398B288B9B8B8A8B1D8A1C8A3B
:10DDA0006EEE72E08A810E94207F6AEC78E08A81C0
:10DDB0000E941B7F8CED95E09A8F898F1B8EDF91DF
:10DDC000CF910895CF93DF93EC018BA19CA1892B78
:10DDD00011F01CA21BA2CE01F9DD10922D011092B0
:10DDE0002C011F8A1E8A0E9400496F8F78A389A385
:10DDF0009AA3DF91CF9108950F931F93CF93DF9351
:10DE0000FC0123A134A1232B91F1EC010E940049D4
:10DE10000F8D18A129A13AA1DC01CB01801B910B28
:10DE2000A20BB30B4097A105B10508F18BA19CA1F2
:10DE30000197E9F46E897F89615071097F8B6E8B40
:10DE4000CE01161617062CF0DF91CF911F910F917E
:10DE5000B9CF0E94285890932D0180932C019F8B5D
:10DE60008E8B0E9400496F8F78A389A39AA3DF91BC
:10DE7000CF911F910F910895CF93DF93EC018D8D7A
:10DE80009E8D1B861A869D878C871F861E86198A03
:10DE9000188A9B8B8A8B1D8A1C8A61E08CE20E9407
:10DEA0003C468A819B81089721F410922D011092A3
:10DEB0002C011CA21BA2DF91CF910895CF93DF9379
:10DEC000EC0121E03FEF3B872A878FEF90E09D87B1
:10DED0008C871F861E86398B288B9B8B8A8B1D8A8D
:10DEE0001C8A61E08AE00E943C4661E086E00E9474
:10DEF0003C4661E08DE20E943C4661E08DE00E947C
:10DF00003C4661E08BE00E943C4661E08EE20E946C
:10DF10003C468A819B818830910529F410922B011F
:10DF200010922A0106C0099721F41092290110923B
:10DF30002801DF91CF9108950F931F93CF93DF9323
:10DF4000EC010E9400490C8D1D8D2E8D3F8DDC0152
:10DF5000CB01801B910BA20BB30B853F9140A10518
:10DF6000B10548F06E897F89CE01DF91CF911F9175
:10DF70000F910C94A158DF91CF911F910F910895AB
:10DF80000F931F93CF93DF938C01FC01178A168A9E
:10DF9000EC01699640E068E0CE010E9446524FE7EE
:10DFA00066E0CE010E94465240E06CE0CE010E9445
:10DFB00046524FE767E0CE010E9446520E94004958
:10DFC000F801648F758F868F978FDF91CF911F91A6
:10DFD0000F9108956F927F928F929F92AF92BF920E
:10DFE000CF92DF92EF92FF920F931F93CF93DF9325
:10DFF0008091941390919513DC01ED91FC91048034
:10E00000F581E02D1995B12C181619060CF0D5C024
:10E01000AA24A3948091941390919513DC01ED911F
:10E02000FC910480F581E02D1995892B09F4C5C078
:10E03000C091020F81E08C0F8093020F80919413A6
:10E0400090919513DC01ED91FC910680F781E02D14
:10E050001995EC2FF0E0EE53F14F80838A30D1F622
:10E06000E090020FF12C1092B00D1092AF0D1092B3
:10E07000AB0D1092AC0D1092AD0D1092AE0D109232
:10E08000AA0D1092A90D1092A80D82ECC82E8EE058
:10E09000D82E00E010E0D0E0C0E00E151F050CF017
:10E0A0006FC0F60191916F019D3009F466C09C37F5
:10E0B000A1F19A3009F055C0CC2359F16C2E712C86
:10E0C000C30101970E94478D7093B00D6093AF0D0F
:10E0D0000E9400496093220E7093230E8093240EB9
:10E0E0009093250E8091A80E882309F462C0809039
:10E0F000AF0D9090B00DB8016619770982EC9EE0E3
:10E100000E944A568816990609F453C01092C10E0F
:10E1100052C01092C10ED0E030C08C2F90E0FC01B4
:10E12000E25AFC4E1082D13099F068F0D230B1F44E
:10E130000E94478D6093AB0D7093AC0D8093AD0D35
:10E140009093AE0D0BC00E94478D6093A80D06C042
:10E150000E94478D7093AA0D6093A90DDF5FC0E008
:10E160000CC00F3311053CF4EC2FF0E0E25AFC4EEA
:10E170009083CF5F02C01092C10E0F5F1F4F8DCFF3
:10E180008091C10E81110EC08091A50D9091A60DB8
:10E1900001969093A60D8093A50D60E087E80E94FC
:10E1A000C19602C0BB24B3941092C20E1092020F0B
:10E1B00031CFA092C10ED1E0E0CF8B2DDF91CF9176
:10E1C0001F910F91FF90EF90DF90CF90BF90AF9095
:10E1D0009F908F907F906F900895CF931092A70D8E
:10E1E0001092A40D1092A60D1092A50D61E089E386
:10E1F0000E94D6440E94ED558091941390919513FE
:10E20000DC01ED91FC910480F581E02D1995892BBD
:10E2100061F08091941390919513DC01ED91FC9144
:10E220000680F781E02D1995E7CF0E943D978091F8
:10E23000941390919513DC01ED91FC910284F38588
:10E24000E02D19951092210E0E9400496093220E34
:10E250007093230E8093240E9093250EC1E0BADEB6
:10E2600081110E94DC310E942D560E94088280910B
:10E27000A50D9091A60D0A9724F48091210E882374
:10E2800031F060E08AE80E94C196C093A70D8091AA
:10E29000A70D882321F38091A40D882341F047ED39
:10E2A00051E060E070E083E09FE00E94ABBA60E084
:10E2B00089E30E94D64460E08AE3CF910C94D6446F
:10E2C000EF92FF920F931F93CF93DF9300D000D074
:10E2D000CDB7DEB76CEF75E0CE0101960E94507AA3
:10E2E0000D811E81F02EEE24E39480919413909181
:10E2F0009513DC01ED91FC910480F581E02D1995D9
:10E30000892B21F18091941390919513DC01ED916B
:10E31000FC910680F781E02D19958F3439F4E09255
:10E32000C00E8093B50EE092B40EDFCF9091C00E78
:10E330009923D9F2E091B40E91E09E0F9093B40E20
:10E34000F0E0EB54F14F80839F1578F28091B40E8A
:10E350008F1510F4F12C20C04BE050E069EA7EE00C
:10E36000CE01019626D6A5EBBEE0ECEFF5E0FF244A
:10E37000F3941127CF018C5F95408017910734F4F7
:10E380009D9181919817B1F3F12CF4CF1092B50EB5
:10E390001092C00E1092B40ECE0101960E94207A07
:10E3A0008F2D26960FB6F894DEBF0FBECDBFDF913E
:10E3B000CF911F910F91FF90EF900895DC01ED91A7
:10E3C000FC910190F081E02D1994CF93DF93EC0143
:10E3D0007F8B6E8B0E942858BC018A81DF91CF9180
:10E3E0000C94357F0F931F93CF93DF93EC01AB0118
:10E3F00060E070E02AE00E94C87A8C01CE010E94A1
:10E40000ED7B800F911FDF91CF911F910F910895A8
:10E410008F929F92AF92BF92CF92DF92EF92FF9234
:10E420000F931F93CF93DF931F921F92CDB7DEB749
:10E43000082E000C990BAA0BBB0BFC013197EF3097
:10E44000F10508F066C28827E757FE4F8F4F0C94FE
:10E4500078B584E08093F4098AE08093F50986E238
:10E460008093F70981E08093FA098093FB098093F8
:10E47000F90944EC58E120E030E08091F40990E0A3
:10E48000281739070CF08CC1FA0185919491A0E00E
:10E49000B0E0880F991FAA1FBB1FF901EE0FFF1FE5
:10E4A000EE0FFF1FE557F64F80839183A283B3835E
:10E4B0002F5F3F4F4E5F5F4FE0CF84E08093F409C2
:10E4C0008AE08093F50986E28093F70981E08093E2
:10E4D000FA098093FB0982E08093F9094CEB58E13B
:10E4E00020E030E08091F40990E0281739070CF023
:10E4F00057C1FA0185919491A0E0B0E0880F991F6F
:10E50000AA1FBB1FF901EE0FFF1FEE0FFF1FE557FC
:10E51000F64F80839183A283B3832F5F3F4F4E5F7B
:10E520005F4FE0CF84E08093F50985E28093F7099F
:10E5300081E08093FA0988E08093FB0983E080936F
:10E54000F90980E090E0FC01EC54F74EE491DC0125
:10E55000A450B64FEC93019688309105A1F70E9424
:10E56000005A1EC188E08093F40986E08093F50983
:10E5700086E28093F70981E08093FA098093FB0992
:10E5800084E08093F90944EA58E120E030E080918A
:10E59000F40990E0281739070CF002C1FA018591BF
:10E5A0009491A0E0B0E0880F991FAA1FBB1FF9014A
:10E5B000EE0FFF1FEE0FFF1FE557F64F808391838D
:10E5C000A283B3832F5F3F4F4E5F5F4FE0CF88E062
:10E5D0008093F40981E08093F50997E29093F7091D
:10E5E0008093FA098093FB0985E08093F90944E957
:10E5F00058E120E030E08091F40990E028173907D5
:10E600000CF0CEC0FA0185919491A0E0B0E0880FA3
:10E61000991FAA1FBB1FF901EE0FFF1FEE0FFF1F6F
:10E62000E557F64F80839183A283B3832F5F3F4FDB
:10E630004E5F5F4FE0CF82E18093F40981E08093E9
:10E64000F50997E29093F7098093FA098093FB0903
:10E650008FE08093F90940E758E120E030E08091B5
:10E66000F40990E0281739070CF09AC0FA01859157
:10E670009491A0E0B0E0880F991FAA1FBB1FF90179
:10E68000EE0FFF1FEE0FFF1FE557F64F80839183BC
:10E69000A283B3832F5F3F4F4E5F5F4FE0CFE09188
:10E6A000550AF091560A74978081918140E550E0B7
:10E6B00060E070E08B5A954F0E94575B2AC182E15F
:10E6C0008093F40985E08093F50982E28093F7094D
:10E6D00081E08093FA098093FB0987E08093F90930
:10E6E00080E993E3A0E0B0E080938B0990938C09DC
:10E6F000A0938D09B0938E09F2E08F2E912C01E04A
:10E7000010E080E090E0A0E0BBE54CE454E060E085
:10E7100070E024EEC22E2CE0D22EE12CF12C9801D8
:10E72000220F331F220F331F5401AA0CBB1CAA0C4B
:10E73000BB1C2557364FF901B7FF0DC0C082D182EF
:10E74000E282F38295012557364FF90140835183C8
:10E75000628373830CC0408351836283738395010A
:10E760002557364FF901C082D182E282F382880FA9
:10E77000991FAA1FBB1F0E5F1F4FF2E08F0E911C47
:10E7800022E18216910459F688E79FEFA0E0B0E0FD
:10E790008093CF099093D009A093D109B093D20967
:10E7A0000E946F5AB6C0CE0101960E94EC5923E038
:10E7B00040E150E060E070E072C084E08093F409D2
:10E7C00082E38093F50986E28093F70981E08093E4
:10E7D000FA098093FB098AE08093F90948E658E139
:10E7E00020E030E08091F40990E028173907C4F662
:10E7F000FA0185919491A0E0B0E0880F991FAA1FBB
:10E80000BB1FF901EE0FFF1FEE0FFF1FE557F64F7D
:10E8100080839183A283B3832F5F3F4F4E5F5F4F0F
:10E82000E1CF84E08093F40980E28093F50986E2E9
:10E830008093F70981E08093FA098093FB098BE0CC
:10E840008093F90940E658E120E030E08091F40936
:10E8500090E0281739070CF0A3CFFA018591949125
:10E86000A0E0B0E0880F991FAA1FBB1FF901EE0FAF
:10E87000FF1FEE0FFF1FE557F64F80839183A283A2
:10E88000B3832F5F3F4F4E5F5F4FE0CFCE010196C6
:10E890000E94EC5921E040E154E060E070E0CE01DC
:10E8A00001960E94CB5A35C084E08093F40983E03E
:10E8B0008093F50986E28093F70981E08093FA0955
:10E8C0008093FB098DE08093F90948E558E120E049
:10E8D00030E08091F40990E0281739070CF060CF00
:10E8E000FA0185919491A0E0B0E0880F991FAA1FCA
:10E8F000BB1FF901EE0FFF1FEE0FFF1FE557F64F8D
:10E9000080839183A283B3832F5F3F4F4E5F5F4F1E
:10E91000E0CF0F900F90DF91CF911F910F91FF905B
:10E92000EF90DF90CF90BF90AF909F908F90089521
:10E930000F931F93CF93DF93EC01462F50E060E0DD
:10E9400070E02AE025D68C01CE0147D7800F911FB9
:10E95000DF91CF911F910F910895462F50E060E015
:10E9600070E02AE015C62FB7F894882381F08091D3
:10E970003D1290913E1290934C1280934B128091D5
:10E980004D1290914E1218161906ACF00FC08091DE
:10E990003F129091401290934C1280934B128091B1
:10E9A0004D1290914E12181619062CF480914D12AA
:10E9B00090914E1207C080914D1290914E129195F8
:10E9C0008195910990934E1280934D122FBF089517
:10E9D000AF92BF92CF92DF92EF92FF920F931F936D
:10E9E000CF93DF931F921F92CDB7DEB78C017A834E
:10E9F0006983CE0101966C01580192E0A90EB11C09
:10EA0000E12CF12CC8010E94BBBAF60161916F01A3
:10EA1000861731F0C8010E94CDBAFFEFEF1AFF0A46
:10EA20000F5F1F4F0A151B0569F781E0EF2809F4F6
:10EA300080E00F900F90DF91CF911F910F91FF9089
:10EA4000EF90DF90CF90BF90AF900895EF92FF923C
:10EA50000F931F93CF93DF931F921F92CDB7DEB713
:10EA60008C017B018AEA8A8341E050E0BE016E5F3F
:10EA70007F4FC8010E944F51D701ED91FC91028454
:10EA8000F385E02DC701199582E8898341E050E0C4
:10EA9000BE016F5F7F4FC8010E944F510F900F90D2
:10EAA000DF91CF911F910F91FF90EF900895CF923A
:10EAB000DF92EF92FF920F931F930E9400496B0128
:10EAC0007C016093B9127093BA128093BB12909339
:10EAD000BC128091020B0E94AE448093B8129091B8
:10EAE000040B992329F091E0811190E09093B812E2
:10EAF00080910C0B90910D0BA0910E0BB0910F0B10
:10EB000097018601081B190B2A0B3B0B4091100B38
:10EB10005091110B6091120B7091130B9091050B9A
:10EB2000041715072607370760F4C092080BD09228
:10EB3000090BE0920A0BF0920B0B1092070B892F36
:10EB40001EC09093060B8091B8128093050BC09263
:10EB5000080BD092090BE0920A0BF0920B0B89176D
:10EB600061F0C0920C0BD0920D0BE0920E0BF09264
:10EB70000F0B91E09093070B02C01092070B1F91AF
:10EB80000F91FF90EF90DF90CF9008950F931F9318
:10EB9000CF93DF93EC012AE0FBD48C01CE011DD68C
:10EBA000800F911FDF91CF911F910F910895CF9208
:10EBB000DF92EF92FF920F931F93CF93DF936B013E
:10EBC000770FEE08FF08F7FE19C0EC016DE2A0D444
:10EBD0008C0144275527BA014C195D096E097F093C
:10EBE0002AE0CE01D5D4800F911FDF91CF911F91E4
:10EBF0000F91FF90EF90DF90CF9008952AE0B7013A
:10EC0000A601DF91CF911F910F91FF90EF90DF90C0
:10EC1000CF90BEC4CF92DF92EF92FF920F931F93DB
:10EC2000CF93DF938C016B01770FEE08FF08F7FE9F
:10EC300010C06DE26DD4EC0144275527BA014C1980
:10EC40005D096E097F092AE0C801A2D4C80FD91F47
:10EC500005C02AE0B701A6019BD4EC01C801BDD5CF
:10EC60008C0F9D1FDF91CF911F910F91FF90EF901F
:10EC7000DF90CF9008950F931F93CF93DF931F9250
:10EC8000CDB7DEB78C0169830E94BBBA6981861754
:10EC900029F0C8010E94CDBA81E001C080E00F9048
:10ECA000DF91CF911F910F910895CF930E941F8202
:10ECB00084E090E09093FF0A8093FE0A84E09FE056
:10ECC0009093DC118093DB111092D6118091FD0A94
:10ECD0009091040F891718F091E09093D3112DE0D3
:10ECE0003FE03093E6112093E5111092E0119091EE
:10ECF0000D0F891718F091E09093DD1126E13FE0A8
:10ED00003093F0112093EF111092EA119091160FA9
:10ED1000891718F091E09093E7112FE13FE03093CD
:10ED2000FA112093F9111092F41190911F0F891785
:10ED300018F091E09093F1111092FC0A20E030E07D
:10ED4000F901E855F04F4081518141505109443259
:10ED5000510520F491E09093FC0A05C02D5F3F4FD0
:10ED60002837310569F79091FC0A992341F12091E8
:10ED7000170F3091180F2D5D3F4F3093180F2093D0
:10ED8000170F2091190F30911A0F23523109309328
:10ED90001A0F2093190F2091200F3091210F2D5D14
:10EDA0003F4F3093210F2093200F2091220F30915D
:10EDB000230F235231093093230F2093220F909178
:10EDC00021109F3049F4909122109F3029F4109225
:10EDD000D2111092D11108C0209175103091761087
:10EDE0003093D2112093D11122E130E03093CF1132
:10EDF0002093CE112091FE0A3091FF0AA8E2BFE0D5
:10EE0000EAE7F1E141E0B683A5839C91992329F0DB
:10EE1000891718F040832F5F3F4F1A96379691E17C
:10EE2000EE3CF90781F73093FF0A2093FE0A213167
:10EE3000310534F080E190E09093FF0A8093FE0A60
:10EE40000E940A8287ED91E19093DD108093DC109F
:10EE50008091DB119091DC119093DB108093DA109C
:10EE600084ED91E19093DF108093DE1085ED91E1C8
:10EE70009093E1108093E01083ED91E19093E31083
:10EE80008093E21081EE91E19093E7108093E61079
:10EE90008091E5119091E6119093E5108093E41034
:10EEA0008EED91E19093E9108093E8108FED91E160
:10EEB0009093EB108093EA108DED91E19093ED101B
:10EEC0008093EC108BEE91E19093F1108093F01011
:10EED0008091EF119091F0119093EF108093EE10CC
:10EEE00088EE91E19093F3108093F21089EE91E116
:10EEF0009093F5108093F41087EE91E19093F710C2
:10EF00008093F61085EF91E19093FB108093FA10B7
:10EF10008091F9119091FA119093F9108093F81063
:10EF200082EF91E19093FD108093FC1083EF91E1CB
:10EF30009093FF108093FE1081EF91E19093011167
:10EF4000809300112091FE0A3091FF0A245031096C
:10EF500060E07AE0C7E0462F50E04217530724F5FF
:10EF6000CA010496789FF001799FF00D1124E652B2
:10EF7000FF4EC49FC001C59F900D1124AC014458A1
:10EF80005E4E53834283DC01A658BE4E15964D91CA
:10EF90005C9116975183408385589E4E9583848358
:10EFA000B187A0876F5FD7CF81E08093000BCF91AF
:10EFB00008950F931F93CF93DF93FC012481358134
:10EFC0002115310519F4FB01108211C0EA012197C6
:10EFD0002C173D0708F4E9018B01FC016081718168
:10EFE000AE01C8010E94C2B8C00FD11F1882DF91C4
:10EFF000CF911F910F9108950895CF92DF92EF92D4
:10F00000FF920F931F93CF93DF936C017A018B01D3
:10F01000C0E0D0E0CE15DF0589F0D8016D918D01FB
:10F02000D601ED91FC910190F081E02DC60119957A
:10F03000892B11F47E0102C02196ECCFC701DF912C
:10F04000CF911F910F91FF90EF90DF90CF90089597
:10F05000FC01A089B1898C91A689B78982FD0FC076
:10F060009C91818D8F5F8F73228D821749F0218D46
:10F07000DF01A20FB11D5D969C93818F08958C9145
:10F080000895FC01918D828D981761F0828DDF01CA
:10F09000A80FB11D5D968C91928D9F5F9F73928F8B
:10F0A00090E008958FEF9FEF0895FC01918D828D80
:10F0B000981731F0828DE80FF11D858D90E008954D
:10F0C0008FEF9FEF0895FC01918D228D892F90E0A5
:10F0D000805C9F4F821B91098F739927089587E168
:10F0E00097E0F1DF21E0892B09F420E0822F0895D9
:10F0F00084EB97E0E8DF21E0892B09F420E0822F00
:10F10000089581E598E0DFDF21E0892B09F420E014
:10F11000822F08958EEE98E0D6DF21E0892B09F446
:10F1200020E0822F0895FC01848DDF01A80FB11D1E
:10F13000A35ABF4F2C91848D90E001968F7399272D
:10F14000848FA689B7892C93A089B1898C9180641A
:10F150008C93938D848D981306C00288F389E02DDB
:10F1600080818F7D80830895EF92FF920F931F938C
:10F17000CF93DF93EC0181E0888F9B8D8C8D98136A
:10F1800005C0E889F989808185FD23C0F62E0B8DA5
:10F1900010E00F5F1F4F0F731127E02E8C8DE812C8
:10F1A0000BC00FB607FCFACFE889F989808185FF8B
:10F1B000F5CFCE01B8DFF2CF8B8DFE01E80FF11D48
:10F1C000E35AFF4FF0820B8FEA89FB8980818062CE
:10F1D00007C0EE89FF896083E889F98980818064AE
:10F1E000808381E090E0DF91CF911F910F91FF909C
:10F1F000EF900895CF93DF93EC01888D8823C1F0C1
:10F20000EA89FB89808185FD05C0A889B9898C912F
:10F2100086FD0EC00FB607FCF5CF808185FFF2CFCB
:10F22000A889B9898C9185FFEDCFCE017CDFE8CF2D
:10F23000DF91CF91089580E090E0892B19F06ADF8B
:10F24000811116C080E090E0892B19F05ADF8111FE
:10F2500012C080E090E0892B19F04ADF81110EC0C6
:10F2600080E090E0892B79F03ADF81110AC008959F
:10F270000E940000E7CF0E940000EBCF0E94000038
:10F28000EFCF0C94000008950E94A3B80F931F9332
:10F29000CF93DF938C01EB01FC018081918100977A
:10F2A000B1F0688179816115710579F042815381EE
:10F2B0002C813D814217530740F00E94BBB88C81DE
:10F2C0009D81F8019583848313C00E9427B78881AC
:10F2D0009981F801918380838A819B8193838283C2
:10F2E0008C819D8195838483198218821B821A8266
:10F2F0001D821C82DF91CF911F910F9108950F9372
:10F300001F93CF93DF93EC0188819981009729F0B7
:10F310002A813B812617370788F48B016F5F7F4F67
:10F320000E94BFB7009761F0998388831B830A838B
:10F330002C813D81232B11F4FC01108281E001C05E
:10F3400080E0DF91CF911F910F910895EF92FF928E
:10F350000F931F93CF93DF93FB0124813581E080CE
:10F36000F180FC0104811581E114F10411F480E0C5
:10F3700016C02115310591F0EC01020F131FB801E1
:10F38000BEDF8823A1F3288139818C819D81B7015B
:10F39000820F931F0E94BBB81D830C8381E0DF9115
:10F3A000CF911F910F91FF90EF900895EF92FF92F0
:10F3B0000F931F93CF93DF93EC017B018A01BA0176
:10F3C0009EDF2881398181110DC02115310519F089
:10F3D000C9010E9427B7198218821D821C821B82D4
:10F3E0001A8206C01D830C83B701C9010E94BBB8F5
:10F3F000CE01DF91CF911F910F91FF90EF90089573
:10F40000CF93DF93EC016115710551F0FB01019081
:10F410000020E9F73197AF01461B570BC7DF0CC03F
:10F4200088819981009711F00E9427B7198218826C
:10F430001D821C821B821A82CE01DF91CF9108951A
:10F44000FC01808191810C9427B70F931F93CF9378
:10F45000DF93CDB7DEB762970FB6F894DEBF0FBE6D
:10F46000CDBF8C01CB01F801118210821382128270
:10F470001582148250E0BE016F5F7F4F0E9426B953
:10F48000BE016F5F7F4FC801BBDF62960FB6F89475
:10F49000DEBF0FBECDBFDF91CF911F910F910895B9
:10F4A000FC0111821082138212821582148261156E
:10F4B000710549F0FB0101900020E9F73197AF0198
:10F4C000461B570B73CF0895CF93DF9300D01F9245
:10F4D000CDB7DEB7611571058105910579F09B0106
:10F4E000AC0169833A834B835C830E941AB92981FA
:10F4F0003A814B815C810E94DBBA03C060E070E01E
:10F50000CB010F900F900F900F90DF91CF91089546
:10F51000DC01ED91FC910190F081E02D1994EF92C6
:10F52000FF920F931F93CF93DF938C017B01C0E079
:10F53000D0E0F701EC0FFD1F6491662361F0D80164
:10F54000ED91FC910190F081E02DC8011995892B76
:10F5500011F02196EECFCE01DF91CF911F910F9147
:10F56000FF90EF9008956115710579F0FB0101900E
:10F570000020E9F73197AF01461B570BDC01ED91F5
:10F58000FC910280F381E02D199480E090E00895D1
:10F590004F925F926F927F92EF92FF920F931F9321
:10F5A000CF93DF93CDB7DEB7A1970FB6F894DEBF48
:10F5B0000FBECDBF7C01FA01CB0119A2223008F4A5
:10F5C0002AE08E010F5D1F4F422E512C612C712CB1
:10F5D000BF01A30192010E9407BBF901CA010150BA
:10F5E00011096A3014F4605D01C0695CD8016C9344
:10F5F000232B242B252B61F7B801C701B4DFA1967B
:10F600000FB6F894DEBF0FBECDBFDF91CF911F9133
:10F610000F91FF90EF907F906F905F904F900895C3
:10F620004F925F926F927F928F929F92AF92BF9212
:10F63000CF92DF92EF92FF92CF93DF93EC016A01BA
:10F640007B01B22E9A01AB01C701B6010E948EB6B2
:10F65000882319F060E076E027C026013701E8949E
:10F6600077F82FEF3FEF4FE75FE7C301B2010E944A
:10F670008EB681110DC02FEF3FEF4FE75FE7C3015B
:10F68000B2010E9492B918161CF464E076E00CC036
:10F690002FEF3FEF4FE75FE4C701B6010E948AB644
:10F6A000181694F468E076E0CE01DF91CF91FF90D8
:10F6B000EF90DF90CF90BF90AF909F908F907F9012
:10F6C0006F905F904F904FCF2FEF3FEF4FE75FEC82
:10F6D000C701B6010E9492B987FDE4CF20E030E077
:10F6E000A901C701B6010E9492B987FF09C06DE266
:10F6F000CE010EDF4C01F7FAF094F7F8F09402C057
:10F70000812C912CA12C60E070E080E09FE3AB1491
:10F7100041F020E030E040E251E40E94F1B5A394D2
:10F72000F6CF9B01AC01C701B6010E948DB52B013C
:10F730003C010E945EB66B017C010E9496B99B0160
:10F74000AC01C301B2010E948CB52B013C012AE03F
:10F75000B701A601CE011CDF7C01E80CF91CBB201F
:10F7600029F06EE2CE01D4DEE80EF91EDB2CDD209E
:10F7700021F120E030E040E251E4C301B2010E94F7
:10F78000F7B92B013C010E945EB64B01A12CB12CB4
:10F790002AE0B501A401CE01FBDEE80EF91EC50189
:10F7A000B4010E9496B99B01AC01C301B2010E9451
:10F7B0008CB52B013C01DA94DACFC701DF91CF91F0
:10F7C000FF90EF90DF90CF90BF90AF909F908F9081
:10F7D0007F906F905F904F9008956CE076E0C3CE7D
:10F7E0000F931F93CF93DF93EC01BDDE8C01CE010D
:10F7F000F4DF800F911FDF91CF911F910F9108953A
:10F800000F931F93CF93DF93EC0189DE8C01CE0120
:10F81000E4DF800F911FDF91CF911F910F91089529
:10F820001F920F920FB60F9211240BB60F922F93C7
:10F830003F934F935F936F937F938F939F93AF9378
:10F84000BF93EF93FF9387E197E06DDCFF91EF911A
:10F85000BF91AF919F918F917F916F915F914F91E8
:10F860003F912F910F900BBE0F900FBE0F901F90E6
:10F8700018951F920F920FB60F9211240BB60F928C
:10F880002F933F934F935F936F937F938F939F93A8
:10F89000AF93BF93EF93FF9387E197E0D9DBFF919D
:10F8A000EF91BF91AF919F918F917F916F915F91F8
:10F8B0004F913F912F910F900BBE0F900FBE0F9065
:10F8C0001F9018951F920F920FB60F9211240BB62E
:10F8D0000F922F933F934F935F936F937F938F93E9
:10F8E0009F93AF93BF93EF93FF9384EB97E01BDC61
:10F8F000FF91EF91BF91AF919F918F917F916F9108
:10F900005F914F913F912F910F900BBE0F900FBEC3
:10F910000F901F9018951F920F920FB60F921124FF
:10F920000BB60F922F933F934F935F936F937F93F9
:10F930008F939F93AF93BF93EF93FF9384EB97E0E5
:10F9400087DBFF91EF91BF91AF919F918F917F9155
:10F950006F915F914F913F912F910F900BBE0F9040
:10F960000FBE0F901F9018951F920F920FB60F9217
:10F9700011240BB60F922F933F934F935F936F9386
:10F980007F938F939F93AF93BF93EF93FF9381E503
:10F9900098E0C9DBFF91EF91BF91AF919F918F915B
:10F9A0007F916F915F914F913F912F910F900BBE7F
:10F9B0000F900FBE0F901F9018951F920F920FB6C9
:10F9C0000F9211240BB60F922F933F934F935F9397
:10F9D0006F937F938F939F93AF93BF93EF93FF9317
:10F9E00081E598E035DBFF91EF91BF91AF919F9159
:10F9F0008F917F916F915F914F913F912F910F90D8
:10FA00000BBE0F900FBE0F901F9018951F920F9274
:10FA10000FB60F9211240BB60F922F933F934F9373
:10FA20005F936F937F938F939F93AF93BF93EF9366
:10FA3000FF938EEE98E077DBFF91EF91BF91AF914E
:10FA40009F918F917F916F915F914F913F912F91F6
:10FA50000F900BBE0F900FBE0F901F9018951F9226
:10FA60000F920FB60F9211240BB60F922F933F9364
:10FA70004F935F936F937F938F939F93AF93BF93B6
:10FA8000EF93FF938EEE98E0E3DAFF91EF91BF9151
:10FA9000AF919F918F917F916F915F914F913F9126
:10FAA0002F910F900BBE0F900FBE0F901F901895C7
:10FAB000CF93DF93EC01E881F9810284F385E02D97
:10FAC0001995EA89FB8980818F7E8083EA89FB8989
:10FAD0008081877F8083EA89FB8980818F7780831B
:10FAE000EA89FB8980818F7D80838A8D898FDF9170
:10FAF000CF910895CF92DF92EF92FF921F93CF9311
:10FB0000DF93EC016A017B01122FE889F98982E019
:10FB100080834115514E61057105B1F060E079E0D7
:10FB20008DE390E0A70196010E9407BBDA01C901AD
:10FB30000197A109B109B695A79597958795AC014D
:10FB4000411580E15807A8F0E889F989108260E83A
:10FB500074E88EE190E0A70196010E9407BBBA010C
:10FB6000A901415051096109710976956795579529
:10FB70004795EC85FD855083EE85FF854083188E83
:10FB8000EC89FD891083EA89FB898081806180830B
:10FB9000EA89FB89808188608083EA89FB8980818A
:10FBA00080688083EA89FB8980818F7D8083DF91F3
:10FBB000CF911F91FF90EF90DF90CF900895482F45
:10FBC00050E095E1899FF0011124E550FE4E21811E
:10FBD000328180859185280F391F83819481821716
:10FBE000930728F08581968128173907E8F485E185
:10FBF000849FF001859FF00D1124E550FE4E858114
:10FC000096812817390728F52581368185E1849F5B
:10FC1000F001859FF00D1124E550FE4E8285823063
:10FC200019F411861086128685E1849FF001859F64
:10FC3000F00D1124E550FE4E328321838091840023
:10FC400090918500280F391F3093890020938800F8
:10FC500008958381948182179307C0F623813481AC
:10FC6000D5CF8091FB0A811157C0E091DB11F09153
:10FC7000DC11858196819093D8118093D7111092D1
:10FC8000DA111092D911E091E511F091E611858118
:10FC900096819093E2118093E1111092E4111092F9
:10FCA000E311E091EF11F091F0118581968190932D
:10FCB000EC118093EB111092EE111092ED11E09186
:10FCC000F911F091FA11858196819093F611809344
:10FCD000F5111092F8111092F71182E190E09093D3
:10FCE000CF118093CE1181E08093D4118093DE11E7
:10FCF0008093E8118093F2118093D01180E090E01E
:10FD000021E0FC01E658FE4E2183079684359105DB
:10FD1000C1F781E08093FB0A08951092F4110895D1
:10FD20001092EA110895982F8FB7F89425E1929FC9
:10FD3000F0011124E550FE4E21E027838FBF41B131
:10FD400021E030E0B90102C0660F771F9A95E2F713
:10FD5000CB01842B81B908958A3058F49FB7F89469
:10FD600025E1829FF0011124E550FE4E1186108698
:10FD70009FBF08951F93CF93DF9325E1829FC0011A
:10FD80001124EC01C550DE4E8A8581110FC01FB7CA
:10FD9000F89481E08A8789899A899A8389830E9465
:10FDA00000496B877C878D879E871FBFDF91CF912E
:10FDB0001F910895CF93DF938A30D0F56233710598
:10FDC00038F061369DE6790728F060E67DE602C0EE
:10FDD00062E370E0D42FC82F80E090E00E9496B9D3
:10FDE00020E030E04AE754E40E94F1B520E030E042
:10FDF0004CE852E40E94F7B99B01AC0160E070E06E
:10FE00008AEF94E40E94F1B50E9459B69B01DD236C
:10FE100021F022273327261B370B8FB7F89495E163
:10FE2000C99FF0011124E550FE4E318720878FBF16
:10FE3000DF91CF9108958A3010F40C94423F0895D9
:10FE40008A3010F40C945D3F08958A3058F495E19F
:10FE5000899FF0011124E550FE4E81819281969593
:10FE60008795089580E090E008958A3010F40C940E
:10FE7000783F08951F920F920FB60F9211240BB680
:10FE80000F920F931F932F933F934F935F936F9313
:10FE90007F938F939F93AF93BF93CF93EF93FF93F2
:10FEA00080911113893048F0109211138091AA1299
:10FEB000882399F08091A3120DC0E0911113E150B5
:10FEC00025E1E29FF0011124E550FE4E8781882351
:10FED00021F0808192B1892782B9E091111385E1E7
:10FEE000E89FF0011124E550FE4E8781882321F020
:10FEF000808192B1892B82B9E0911113C5E1CE9F27
:10FF0000F0011124E550FE4E80859185892B09F082
:10FF10004DC0E0911113CE9FF0011124E550FE4E2B
:10FF20008285813009F060C00E940049E091111380
:10FF3000CE9FF0011124E550FE4E038514852585E2
:10FF40003685E0911113CE9FF0011124E550FE4E4D
:10FF50000784F089E02DAB01BC01401B510B620B03
:10FF6000730BCF01A0E0B0E084179507A607B70791
:10FF7000D8F5E0911113A0911113CA9FD00111245B
:10FF8000A550BE4E53968D919C915497CE9FF001F3
:10FF90001124E550FE4E91878087E0911113CE9F8A
:10FFA000F0011124E550FE4E82E08287809111130A
:10FFB00006DE809111138F5F80931113FF91EF91F3
:10FFC000CF91BF91AF919F918F917F916F915F91F1
:10FFD0004F913F912F911F910F910F900BBE0F905A
:10FFE0000FBE0F901F901895E0911113809184001F
:10FFF0009091850025E1E29FF0011124E550FE4E2D
:020000021000EC
:1000000021813281820F931F909389008093880011
:10001000D0CF1F93CF93DF9380911013811173C0C2
:10002000109211139FB7F89485E128EB3BE04CED5B
:1000300055E064E971E1A1E0B0E0E0911113E9302D
:1000400008F052C0E09111138E9FF0011124E55089
:10005000FE4E32832183E09111138E9FF001112413
:10006000E550FE4E56834583E09111138E9FF001BB
:100070001124E550FE4E74836383E0911113F091D7
:100080001113ED0101C0CC0FFA95EAF78E9FF00134
:100090001124E550FE4EC083E09111138E9FF001B4
:1000A0001124E550FE4E1782E09111138E9FF0014E
:1000B0001124E550FE4E11861086E09111138E9F9B
:1000C000F0011124E550FE4E1286E09111138E9F2F
:1000D000F0011124E550FE4E148A138AE0911113A9
:1000E000EF5FE0931113A9CF9FBF8FB7F89420EA79
:1000F0003FE03093A5122093A4121092A3128FBF59
:1001000081E080931013DF91CF911F9108950F9399
:100110001F93CF93DF938C01C62FD42FDC01119650
:100120008D919C911297DC01ED91FC910190F081F1
:10013000E02DD8016C911995F80181819281DC0143
:10014000ED91FC910190F081E02D6C2F1995F80153
:1001500081819281DC01ED91FC910190F081E02D93
:100160006D2F1995F80180816C2F70E0680F711D5B
:100170006D0F711D6F77772781819281DF91CF910C
:100180001F910F910C94DE710F931F93CF93DF9308
:100190008C01C62FD42FDC0111968D919C91129762
:1001A000DC01ED91FC910190F081E02DD8016C9182
:1001B0001995F80181819281DC01ED91FC9101900A
:1001C000F081E02D6C2F1995F80181819281DC017D
:1001D000ED91FC910190F081E02D6D2F1995F801C2
:1001E00080816C2F70E0680F711D6D0F711D6F772E
:1001F000772781819281DF91CF911F910F910C948C
:10020000DE714F925F926F927F92AF92BF92CF92C8
:10021000DF92EF92FF921F93CF93DF93DD24D3946D
:1002200045E0C42E52E0A52EB12CC3E0D0E0EE2470
:10023000E394F12C8091F4129091F512DC01ED9190
:10024000FC910480F581E02D1995892B09F4BEC03D
:10025000109130018091F4129091F512DC01ED9132
:10026000FC910680F781E02D199596B3B39A209101
:100270008400309185002059384E30938D002093B2
:100280008C00212F2C7139F010920F13D093F312A0
:10029000C093F212CFCF93FB992790F9E0910F13FF
:1002A000E11116C0992331F28F3021F6D0920F134D
:1002B0008093F6128091F2129091F312892B09F03B
:1002C000B9CFF092F312E092F2121092F112B2CF83
:1002D0009111DACF91E09E0F90930F13F0E0EA5066
:1002E000FD4E8083993109F0A5CF81116CC08091BA
:1002F0000D1382FF05C0D093F312C093F21263C0B6
:1003000083FDF9CF8091F2129091F312019739F4A5
:100310008091F1128F5F8093F112843020F0B092BF
:10032000F312A092F2128091F0128F5F8093F0127C
:100330009091EF12981708F044C0D092EE12AEECF4
:10034000B2E1E7EFF2E140E050E0BA0110E0CF01A6
:10035000FC011B3098F401964080512C612C712CCB
:10036000012E04C0440C551C661C771C0A94D2F75D
:100370004429552966297729185FEACF9A013770F1
:10038000205E3340C29EC001C39E900D112497FD94
:10039000079623E0959587952A95E1F784529A4F21
:1003A0008D939D931B503BE07695679557954795A8
:1003B0003A95D1F782E1AE3EB80749F61092F012B5
:1003C00002C01092EE1210920F1334CFDF91CF9132
:1003D0001F91FF90EF90DF90CF90BF90AF907F90F4
:1003E0006F905F904F9008958091010B833029F4B6
:1003F0008091CC129091CD129DC108958091010BF6
:10040000823029F48091CA129091CB12FACE0895CD
:10041000F5DFEACF1092D4111092DE111092E8119C
:100420001092F2111092D01180E090E0FC01E65899
:10043000FE4E1182079684359105C1F7089580918B
:10044000010B823039F0833049F0813049F48091DA
:10045000C71201C080E18093FD0A04C08EE0FBCF8B
:100460001092FD0A8091FD0A08958091010B82305F
:1004700039F0833049F0813059F48091C6120895E3
:10048000BDDF8091EE120895AFDF8091C51208950F
:1004900080E008958091010B823049F0833069F04B
:1004A000813089F48091C1129091C2120895A6DF23
:1004B0008091F2129091F312089596DF8091C31209
:1004C0009091C412089581E090E008958F929F92D8
:1004D000AF92BF92CF92DF92EF92FF921F93CF9392
:1004E000DF93EC0111E08E819F81892B09F410E0EC
:1004F0002C813D81E885F985C580D680878190E093
:10050000A601480F591F2417350764F180850D2C6B
:10051000000CEE08FF08A901330F660B770B038070
:10052000F481E02D9A01AB012C193D094E095F09B8
:10053000882329F0A1E0BFEF0E9403BB04C0AFEF06
:10054000B0E00E94F7BA4F01FF0FAA08BB08A5014F
:1005500094012C193D094E095F090E94DBBA3F83C3
:100560002E834BC0A601481B590B421753070CF4AE
:100570003FC080850D2C000CEE08FF08A901330F49
:10058000660B770B81809280092C000CAA08BB08AF
:100590009A01AB01281939094A095B09882399F0A6
:1005A000A1E0BFEF0E9403BBA701960128193909FA
:1005B0004A095B090E94DBBADA01C90181509F4FE9
:1005C000AF4FBF4F12C0AFEFB0E00E94F7BAA70124
:1005D0009601281939094A095B090E94DBBADA0138
:1005E000C9018F5F9109A109B1099F838E8305C05D
:1005F0001F821E82111101C019828E819F81009776
:1006000089F08F3F910519F014F08FEF90E0813061
:100610005FEF950714F481E09FEF9F838E8381E065
:1006200018271A83DF91CF911F91FF90EF90DF90F1
:10063000CF90BF90AF909F908F900895CF93DF930E
:10064000C091BD12D091BE126091BF127091C012C4
:10065000CE010E94DE3D81110DC021E33EE74CE258
:1006600051E060E070E0CE010E94453E9093C012E0
:100670008093BF12DF91CF910895CF93DF93CDB7D1
:10068000DEB7A0970FB6F894DEBF0FBECDBF8031A6
:100690000CF080E020E739E13A83298329E639E14B
:1006A0003C832B832BE539E13E832D832FE439E115
:1006B00038872F8325E439E13A8729872BE339E10D
:1006C0003C872B8727E339E13E872D8720E339E1FB
:1006D000388B2F8725E239E13A8B298B28E139E1E4
:1006E0003C8B2B8B2DE039E13E8B2D8B21E039E1CA
:1006F000388F2F8B2FEE38E13A8F298F2EED38E18E
:100700003C8F2B8F29ED38E13E8F2D8F2CEC38E17B
:1007100038A32F8FE82FEE0FFF0BEC0FFD1F818109
:100720009281A0960FB6F894DEBF0FBECDBFDF91C9
:10073000CF910895AF92BF92CF92DF92EF92FF9246
:100740000F931F93CF93DF938BE193E17EE1D72E3D
:10075000D80ECC24C39402E010E0C3E0D0E0E2E085
:10076000BE2EEE24E394F12C80912A0E90912B0E54
:10077000DC01ED91FC910480F581E02D1995892B28
:1007800009F4ADC0A090300180912A0E90912B0EFB
:10079000DC01ED91FC910680F781E02D199596B36F
:1007A000B39A2091840030918500285A344E3093BA
:1007B0008D0020938C002A2D2C7119F01092270E99
:1007C0004BC093FB992790F9E091270EE11116C0D9
:1007D000992351F2803241F6C092270E80931B1369
:1007E0008091C3129091C412892B09F0BDCFF09271
:1007F000C412E092C3121092290EB6CF9111DECF2F
:10080000E13041F4803409F0AFCFB092270E8093ED
:100810001C13E6CF91E09E0F9093270EF0E0E55E6B
:10082000FC4E8083903209F09FCF1092270EEBE1AF
:10083000F3E12FEF3FEF8191281B3109DE12FBCF4F
:100840004091391380913A1390E0982F8827840FB4
:10085000911D2817390729F0D093C412C093C312F1
:1008600083CF8091C3129091C412019739F4809183
:10087000290E8F5F8093290E843020F01093C412CC
:100880000093C3128091280E8F5F8093280E909161
:10089000260E981708F5C092C51220E030E0F90145
:1008A000E55EFC4E4281838190E0982F8827840F7B
:1008B000911DAC014F5E52404B3D554028F4F9016B
:1008C000E45DF14F918380832E5F3F4F2C313105E2
:1008D00031F71092280E48CF1092C51245CFDF9104
:1008E000CF911F910F91FF90EF90DF90CF90BF902D
:1008F000AF900895EF92FF920F931F93CF93DF93E2
:100900001092030F82E08093040F68EE73E07093FF
:10091000060F6093050F40ED57E05093080F40938A
:10092000070F2CED35E030930A0F2093090F8FE06D
:1009300080930B0F10920C0F94E090930D0F709317
:100940000F0F60930E0F5093110F4093100F3093C1
:10095000130F2093120F8093140F1092150F93E032
:100960009093160F7093180F6093170F50931A0FF0
:100970004093190F30931C0F20931B0F80931D0F72
:1009800010921E0F91E090931F0F7093210F6093B0
:10099000200F5093230F4093220F3093250F209365
:1009A000240F8093260F1092270FE8E2FFE0A1E3C7
:1009B000BFE080E008EE13E060ED77E04CED55E03D
:1009C00031E022E095E0980F9083128301837483D5
:1009D000638356834583ED01229791E03883219606
:1009E00028831C928F5F3A961A968C3059F7109292
:1009F000A00F9093A10F1092A20F9093A30F8AE8DB
:100A000092E09093A50F8093A40F9093A70F8093EB
:100A1000A60F80E090E09C012D5F304FF901EB556F
:100A2000FF4F11821082329610820396883791050B
:100A300091F784E290E09093A90F8093A80F81E052
:100A40008093AA0F2CE030E03093AC0F2093AB0FD3
:100A500094E09093AD0F21E230E03093AF0F2093FC
:100A6000AE0F27E02093B00F29E030E03093B20FB3
:100A70002093B10F20E12093B30F7AE07093201000
:100A80002BE0209321102093221048EE53E0509346
:100A900024104093231020ED37E03093261020934C
:100AA00025101092271064E6609328106093291097
:100AB00050932B1040932A1030932D1020932C101C
:100AC00010922E105093301040932F10309332100C
:100AD00020933110109233101092341080933510FF
:100AE000109237101092361080933810809339107E
:100AF000E8ECF0E0F0933B10E0933A10E0E2F3E032
:100B0000F0933D10E0933C1050933F1040933E1003
:100B1000309341102093401080934210E9E5F0E0BB
:100B2000F0934410E0934310E0E8F0E0F0934610B7
:100B3000E0934510EFEFF0E0F0934810E09347109A
:100B4000F0934A10E093491080934B1090934C100F
:100B500010924D1080934E1090934F1010925010A1
:100B60001092511080935210109253101092541002
:100B7000809355101092561098E29093571050930E
:100B800059104093581050935B1040935A10309373
:100B90005D1020935C1080935E1092E390935F1041
:100BA000E2E0E09360108093611060936210E6E4ED
:100BB000E093631090936410109265101092661089
:100BC00010926710109268101092691010926A10BB
:100BD000EAEFF0E0F0936C10E0936B1010926D1060
:100BE00010926E1060936F1061E460937010109219
:100BF0007110909372101092731090937410EEE530
:100C0000F1E0F0937610E093751010927710ACED50
:100C1000B5E0B0937910A093781000EA1FE010932C
:100C20007B1000937A1030937D1020937C10C8E8DD
:100C3000D3E1D0937F10C0937E1068EBE62E6BE07B
:100C4000F62EF0928110E0928010E0E4FFE1F09344
:100C50008310E093821010928410109285101092ED
:100C6000861069E1609387108093881080938910C3
:100C700080938A1050938C1040938B1030938E1079
:100C800020938D10F0929010E0928F10109392109C
:100C900000939110D0939410C093931020E737E104
:100CA00030939610209395101092971010929810F0
:100CB0001092991090939A1090939B1090939C107F
:100CC00010929D1010929E1010929F108093A01071
:100CD0001092B0101092A11099E09093A21010926F
:100CE000A3101092A4101092A5101092A610B09309
:100CF000A810A093A710F093AA10E093A9108093D6
:100D0000AB107093AC101092AD1021E030E0309336
:100D1000AF102093AE1040E052EC61E070E04093E1
:100D2000B1105093B2106093B3107093B41040930D
:100D3000B5105093B6106093B7107093B81040E0A0
:100D400056E960E070E04093B9105093BA10609398
:100D5000BB107093BC104093BD105093BE106093B5
:100D6000BF107093C0101092C11020E039E1309391
:100D7000C3102093C2101092C4109EE19093C5102E
:100D80001092C6102EE130E03093C8102093C710A7
:100D90003093CA102093C9103093CC102093CB10FD
:100DA0009093CD109093CE108093CF108093D0105D
:100DB0001092D1109093D2108093D3109CE0909316
:100DC000D4108093D51083E891EFA0E0B0E0809339
:100DD000D6109093D710A093D810B093D91003E0F9
:100DE0001FE0C0E0D0E0CE010E94BBBAF8016191E3
:100DF0008F01861719F0CE010E94CDBA2196C73D0A
:100E0000F1E0DF0781F7DF91CF911F910F91FF9004
:100E1000EF9008954F925F926F927F928F929F9280
:100E2000AF92BF92CF92DF92EF92FF92CF93DF9378
:100E3000EB01A0911913B0911A139D012F5F3F4F41
:100E400045E0429F2001439F500C1124052C000CCB
:100E500066087708812C912C54012434E1E03E0788
:100E6000ECF44FE851E961E0772775016401C40CA7
:100E7000D51CE61CF71C4C0D5D1D6E1D7F1D6BBF48
:100E8000FA014791569165E0860E911CA11CB11C98
:100E9000C417D50729F12F5F3F4FDFCF25E0822E02
:100EA000912CA12CB12C21E030E0A217B30708F45B
:100EB0004CC04FE851E961E07727480D591D6A1D84
:100EC0007B1D6BBFFA0147915691F5E08F0E911C87
:100ED000A11CB11CC417D50719F02F5F3F4FE5CFF8
:100EE0004FE851E961E07727E5E0E29F6001E39F89
:100EF000D00C11240D2C000CEE08FF084E5F5F4F44
:100F00006F4F7F4F4C0D5D1D6E1D7F1D6BBFFA0136
:100F100047915691FC01538342834FE851E961E0C8
:100F200077274C5F5F4F6F4F7F4FC40ED51EE61E75
:100F3000F71EEBBEF601C790FC01C48230931A1372
:100F400020931913C901019606C010921A1310922A
:100F5000191380E090E0DF91CF91FF90EF90DF9048
:100F6000CF90BF90AF909F908F907F906F905F9049
:100F70004F9008950F931F938091141381111EC0F9
:100F80000E94004900911513109116132091171318
:100F900030911813AB01BC01401B510B620B730B5A
:100FA0008091121390911313A0E0B0E0841795077D
:100FB000A607B70718F481E0809314131F910F91CF
:100FC00008958091121390911313892B89F08091C9
:100FD0001413882381F00E940049609315137093C5
:100FE00016138093171390931813109214130895E7
:100FF00081E08093141308951F920F920FB60F9201
:1010000011242F938F939F93109295001092940028
:101010008091F50A8F5F8093F50A90914D1389179F
:1010200084F01092F50A2091F70A8091581390915C
:101030005913820F911D27FD9A9590935913809310
:1010400058138091F40A8F5F8093F40A90915D1396
:10105000891784F01092F40A2091F60A80915B13AC
:1010600090915C13820F911D27FD9A9590935C13CC
:1010700080935B139F918F912F910F900FBE0F90D4
:101080001F9018958091F30A811104C08091F20A93
:10109000882321F080917100826003C080917100EB
:1010A0008D7F809371000895CF93DF93EC011C86B0
:1010B0001D861E86188A1F860E94004968837983D0
:1010C0008A839B83198618861C86DF91CF910895A9
:1010D000CF92DF92EF92FF920F931F93CF93DF9304
:1010E000CDB7DEB765970FB6F894DEBF0FBECDBFA4
:1010F0008C016B017A01D8DFF801118ADA82C9828A
:10110000FC82EB82FF24F394FD8A85E1FE01319697
:10111000D801529601900D928A95E1F7F801D08A94
:10112000C78682E08687C8010E9459950E940049BF
:10113000F8016083718382839383F48665960FB68A
:10114000F894DEBF0FBECDBFDF91CF911F910F91FD
:10115000FF90EF90DF90CF900895FC018385882366
:1011600011F061E001C060E082850C94D6440F93D9
:101170001F93CF93DF93EC0188859985892BE9F044
:101180000E9400490C811D812E813F81AB01BC0171
:10119000401B510B620B730B88859985A0E0B0E072
:1011A00084179507A607B70740F4CE01D6DFCE0116
:1011B000DF91CF911F910F9177CF8F859889892BE0
:1011C00009F445C00E940049088119812A813B81A8
:1011D000AB01BC01401B510B620B730B8F859889CF
:1011E000A0E0B0E084179507A607B70780F58D85C6
:1011F0008F5F8D879E858917C0F480FF03C0CE0165
:10120000ACDF03C0CE010E9459958989811119C0B4
:101210008D858B3050F6FE01E80FF11DE80FF11DB2
:1012200082899389988B8F870CC08EA1882309F4BB
:10123000BCCF8A899B89988B8F871D86CE010E949F
:1012400059950E940049688379838A839B83DF9143
:10125000CF911F910F91089560E089E30E94D644D9
:1012600060E08AE30E94D64460E085E30E94D644B1
:1012700060E085E00E94D64460E084E00E94D644AD
:1012800060E087E00E94D64472980895CF93C091A1
:1012900012026C2F89E30E94D64481E0C8276C2F8C
:1012A0008AE30E94D644C0931202CF910895CF934F
:1012B000DF93C09111026C2F89E30E94D644D1E0E4
:1012C000DC276D2F8AE30E94D6446C2F85E30E94B1
:1012D000D6446D2F85E00E94D6446D2F84E00E9495
:1012E000D6446C2F87E00E94D644CC2311F072982C
:1012F00001C0729A9091110281E0892780931102B6
:10130000DF91CF910895CF93DF9380914C1381119A
:101310000DC010924B1310924A1381E090E090930D
:1013200049138093481380934C1336C080914A131D
:1013300090914B13863191057CF18F38910534F4EF
:101340008091481390914913019609C08D3521E091
:10135000920754F480914813909149130296909308
:1013600049138093481318C0863222E0920734F460
:1013700080914813909149130496F1CF883E934091
:101380003CF480914813909149138A5B9F4FE7CFBB
:1013900010924913109248138ADFC0914A13D091DA
:1013A0004B13C93E83E0D80754F010924C1354DF1E
:1013B0002BEF39E848EE53E060E070E007C023E827
:1013C00039E8AE010D2E000C660B770B84E69BE02E
:1013D0000E94453E90934713809346138091481393
:1013E000909149138C0F9D1F90934B1380934A1338
:1013F000DF91CF910895CF93DF938091B906882331
:1014000019F0DF91CF917FCFC0914613D091471350
:10141000BE0184E69BE00E94DE3D882329F0BE01E8
:1014200084E69BE00E94F63DDF91CF9115CFCF93EC
:10143000C09143136C2F70E088E00E94784689E1E8
:101440008093421390911002992311F0CD5F01C057
:10145000C350C093431380914313873970F099238D
:1014600021F08FEF8093431308C08D3D30F086E963
:101470008093431388E780934213809143138F3FF7
:1014800019F41092100205C08A3118F481E080939B
:1014900010024091421350E060E070E027E13AE82A
:1014A00084E69BE00E94453E9093921380939113B3
:1014B000CF910895CF92DF92EF92FF92CF93DF9377
:1014C000EC019C01AFEFB0E00E9429BBCC24CA9490
:1014D00023E0D22EE12CF12CA70196010E94DBBA69
:1014E000B90188E00E9478469E01A4E6B0E00E941F
:1014F00029BBA70196010E94DBBA8091CD1082130F
:101500002093CD10DF91CF91FF90EF90DF90CF909F
:101510000895CF93DF93C0919113D0919213BE01A0
:1015200084E69BE00E94DE3D882329F0BE0184E62C
:101530009BE00E94F63D60E088E00E94D6448091E6
:10154000B6068823D1F080919313882319F06FE0B9
:101550007AE10DC080919013882319F066EF79E14C
:1015600006C080919613811108C067EE79E18091E1
:10157000B4069091B5060E94007C109293131092CD
:101580009013DF91CF91089561E088E00E94D644E6
:101590008091B606882361F080919313811108C071
:1015A00069ED79E18091B4069091B5060C94007CC8
:1015B000089580919313811110C0ABDF81E0809377
:1015C00093138091B606882341F06EE37AE180910F
:1015D000B4069091B5060E94007C80914113882347
:1015E00029F060E088E00E94D64401C0CDDF9091F0
:1015F000411381E0892780934113882329F040918A
:10160000C9105091CA1004C04091CB105091CC1019
:1016100060E070E029ED3AE884E69BE00E94453EF8
:1016200090939213809391130895CF9380913F13D9
:1016300081110FC081E080933F138091B60688230B
:1016400041F067EA79E18091B4069091B5060E9475
:10165000007CC0913E136C2F85E00E94D6444091DF
:10166000D21050E060E070E025E13BE884E69BE0CA
:101670000E94453E90933D1380933C1381E06C2F74
:10168000682760933E13CF910895CF93DF93C09165
:101690004413D0914513BE0184E69BE00E94DE3DD9
:1016A000882361F0BE0184E69BE00E94F63D109223
:1016B000451310924413DF91CF91CECDDF91CF919E
:1016C0000895609144137091451384E69BE00E9455
:1016D000DE3D81112EC060E089E30E94D64460E0C7
:1016E0008AE30E94D64460E085E30E94D64460E02D
:1016F00085E00E94D64460E084E00E94D64460E029
:1017000087E00E94D64472988091CF10882319F008
:1017100027E539E802C026E439E842E350E060E01A
:1017200070E084E69BE00E945F3E909345138093B7
:101730004413089560E08AE30C94D64461E08AE3A0
:101740000C94D6440F931F93CF93DF938C01C1E089
:10175000D0E00C171D079CF0F1DF64E670E080E03C
:1017600090E00E94C848E6DFC017D10734F46AE56C
:1017700070E080E090E00E94C8482196EACFDF91B7
:10178000CF911F910F91089583E090E0DBCF82E02D
:1017900090E0D8CF81E090E0D5CF60E089E30C9471
:1017A000D64461E089E30C94D6440F931F93CF9302
:1017B000DF938C01C1E0D0E00C171D079CF0F1DF36
:1017C00064E670E080E090E00E94C848E6DFC01761
:1017D000D10734F46AE570E080E090E00E94C848E8
:1017E0002196EACFDF91CF911F910F91089583E069
:1017F00090E0DBCF82E090E0D8CF81E090E0D5CFE1
:101800006091CD1070E088E00E9478468091B60625
:10181000882341F068E27AE18091B4069091B506A0
:101820000C94007C0895109240138091A2068111BF
:1018300004C060E084E00E94D6448091B60688230C
:1018400041F066EC79E18091B4069091B5060C9474
:10185000007C089581E0809340138091A20681115D
:1018600006C060913B1370E084E00E94784680914E
:10187000B606882341F064EB79E18091B40690913B
:10188000B5060C94007C08951092A2068091401336
:10189000811104C060E084E00C94D64460913B1355
:1018A00070E084E00C947846CF93DF9360E085E0AD
:1018B0000E94D64480913F1381110BC08091B006E5
:1018C0009091B106DC01ED91FC9102ACF3ADE02DFD
:1018D0001995C0913C13D0913D13BE0184E69BE065
:1018E0000E94DE3D882329F0BE0184E69BE00E9431
:1018F000F63D8091B606882379F020913F138091C0
:10190000B4069091B506222319F06BE979E102C083
:101910006FE879E10E94007C10923F13DF91CF9134
:10192000089561E085E00E94D6448091B0069091D0
:10193000B106DC01ED91FC9102ACF3ADE02D1995FF
:101940008091B606882341F064E879E18091B4067D
:101950009091B5060C94007C089560E085E30E94A8
:10196000D6448091B0069091B106DC01ED91FC91D6
:1019700006A8F7A9E02D19958091B606882341F0B5
:1019800068E779E18091B4069091B5060C94007CEB
:1019900008954115510529F06115710511F00C9458
:1019A000D9770895EF92FF920F931F93CF93DF9310
:1019B0001F921F92CDB7DEB78C018CE789831A8204
:1019C000F801E480F580FFEFEF1AFF0AB701C801C4
:1019D0000E947F79882381F0F80120813181848100
:1019E0009581BE016F5F7F4F820F931F0E94BBB82E
:1019F000F801F582E48281E00F900F90DF91CF91A2
:101A00001F910F91FF90EF900895AF92BF92CF92E8
:101A1000DF92EF92FF920F931F93CF93DF9300D04B
:101A20001F92CDB7DEB78C0149835A836B837C83C9
:101A3000CE0101966C01580194E0A90EB11CE12C75
:101A4000F12CC8010E94BBBAF60161916F018617A3
:101A500031F0C8010E94CDBAFFEFEF1AFF0A0F5F05
:101A60001F4F0A151B0569F781E0EF2809F480E094
:101A70000F900F900F900F90DF91CF911F910F91CA
:101A8000FF90EF90DF90CF90BF90AF900895CF92EE
:101A9000DF92EF92FF920F931F93CF93DF93EC01AE
:101AA00000915E13E0E0F0E020E030E0A90110E0FA
:101AB000CE17DF071CF1309711F40D32E1F0DF0192
:101AC000A25ABC4EFC9080ED8F0D8A30A8F4AAE09B
:101AD000B0E00E94F7BA2F2DFF0C330B20533109D1
:101AE0006901330FEE08FF089B01AC012C0D3D1D71
:101AF0004E1D5F1D01C011E03196DACFCA01B90158
:101B0000112339F090958095709561957F4F8F4F97
:101B10009F4FDF91CF911F910F91FF90EF90DF903A
:101B2000CF9008958091050B811105C081E09091BF
:101B3000070B911101C080E00895CF93DF932091AE
:101B40002C0A30912D0AE9012697A881B981A45D5C
:101B5000B54F12961C92082E000C990BAA0BBB0BCA
:101B6000FC013197EF30F10508F06EC18827E85687
:101B7000FE4F8F4F0C9478B5F9013A97808191818F
:101B8000845D954F0E9443B3882309F462C1E091BC
:101B90002C0AF0912D0A36970190F081E02DE45D3A
:101BA000F54F81E0EDC0F9013C9780819181845D22
:101BB000954F0E9480B2882309F44BC1E0912C0A12
:101BC000F0912D0A36970190F081E02DE45DF54FFC
:101BD00082E0D6C0F9013E9780819181845D954F66
:101BE0000E94C3B1882309F434C1E0912C0AF0911A
:101BF0002D0A36970190F081E02DE45DF54F83E0EA
:101C0000BFC0F901709780819181845D954F0E94DA
